:020000040800F2
:10000000005000208955010829560108713F010858
:100010002956010829560108295601080000000048
:100020000000000000000000000000002956010848
:10003000295601080000000029560108BF240108C4
:100040002956010829560108295601082956010890
:100050002956010829560108CD9F0008C99F0008AC
:100060002956010829560108295601082956010870
:10007000295601082956010879D200082956010895
:1000800011EE0008295601082956010829560108D1
:10009000295601082956010829560108C59F00085C
:1000A00029560108A9E1000829560108B9E100080C
:1000B00099E1000889E1000879E10008C1640008BD
:1000C000C5640008B9640008BD6400082956010829
:1000D0002956010871D2000869D2000861D20008CF
:1000E000CD24010829560108295601080000000006
:1000F0000000000000000000000000000000000000
:0C01000000000000000000005FF808F1A3
:100110002DE9F04F764B774FA1B03B6000237B6019
:1001200011F00DFC18B911F02BFC08F0B9FF09F023
:1001300081F8714A714D1378714E43F001031370C9
:100140000023089309930A934FF4E0130B932B6851
:10015000307B43F480332B60AB6943F01003AB6119
:100160002B6803F400330993089B01330893099B20
:100170001BB9089BB3F5A06FF2D12B685F4913F44C
:10018000003301D0022315E00A6842F001020A6040
:1001900008932B6803F002030993089B013308932B
:1001A000099B1BB9089BB3F5A06FF2D12B689A0786
:1001B00039D501230A93534B53491A6842F0100270
:1001C0001A601A6822F003021A601A6842F00202EA
:1001D0001A606B686B606B686B606B6843F480637C
:1001E0006B604A4B1A68043B22F070425A60484ADE
:1001F0001160696821F47C116960596841F000411F
:100200005960D96821F40041D9609B681B0449BF3B
:10021000404B4FF4E01313604FF480130B930A9B91
:10022000012B01D117E0FEE7022B18D168B10B9B1F
:10023000B3F5801F02D14FF4A01305E00B9BB3F57B
:10024000E01F02D14FF400130B930B996B680B4323
:1002500043F4803302E06B6843F460136B602B68F7
:1002600043F080732B602968244B8C01FBD55968BF
:1002700021F003015960596841F0020159606B682F
:100280001E4903F00C03082BF9D14B68DFF890905E
:1002900003F00C03042B03D0082B03D01A4B12E0FD
:1002A000136810E04B684868C3F38343C00303F14D
:1002B000020301D4184905E0496811F4003F1168B0
:1002C00018BF49084B43C9F800306B681349C3F3A2
:1002D00003130B44187ED9F800308846C340C9F890
:1002E00000301368084A93421CD101221EE000BF6F
:1002F00007890008C8000020A03300200010024039
:10030000E81000200020024000127A000410014092
:100310002C000020001BB70000093D00B892010826
:1003200054000020AB4A934202D10222AA4B1A7019
:10033000DFF808C3A94B20ACCCF80C30AB69CDF882
:100340000CC043F00103AB616B6ADFF8B8A2BB607D
:100350006B6A4FF0000B43F080736B62AB69A0488F
:1003600043F01C03AB614FF6FF7324F82C3D21468C
:100370008DF856B00EF057FE504621460EF053FE53
:10038000214698480EF04FFE974A2046536843F0A6
:10039000007353600CF0D4F9944A159B5946B3FB93
:1003A000F2F3934A934813600C2217F0D8FAD9F865
:1003B00000304FF47A72B3FBF2F38F4ADDF80CC0D1
:1003C000013B5360F0238CF823300723C2F808B0B8
:1003D0001360B368DFF86892DFF868C2C9F80030CC
:1003E0009CE80F0084E80F00AB69CDF80CC043F027
:1003F0000803AB61AB69159843F00803AB610823B0
:10040000CAF810301023CAF8103016A90EF00BFEEF
:10041000179818A90EF007FED9F80030DFF828B2B7
:1004200013F0080FDDF80CC051D09BF89031012B70
:100430004DD8DCF810002146206050469BF891B161
:100440000EF0F1FD0A2012F025F8DAF8083003F07A
:1004500020039BB2002B3AD1684A9268D20040F147
:100460000286DB0733D5664ADFF898B11068DFF8FB
:1004700070A11023CBF814302146159050460393F9
:100480000EF0D1FD0822CAF810203C2012F00DF821
:10049000039BCBF81030002396F89121934216DA93
:1004A000584A4FF0080B04937820C2F810B003921A
:1004B000CAF814B011F0EEFF039A7820C2F814B015
:1004C000CAF810B011F0E6FF049B0133E4E76420A2
:1004D00011F0EBFFA0224C48002117F040FAEB6925
:1004E000002243F00703EB61AB6943F4006343F080
:1004F0000C03AB61414B4FF0000A03F10C0102F811
:1005000001A001320E2AF5D1FF229A76DA761A7707
:100510005A773E4B3E4A51461A603E483C22D9F833
:10052000005017F01CFA5146C5F3801905233A4ACA
:10053000DFF8E0E0885C0C224A4302F80E00B9F1D3
:10054000000F08D11E3801289FBFFF2003F1FF33A1
:1005500002F80E00DBB201310529E8D12F4A3048FC
:10056000137073792F4A254913702F4A3A62C032AB
:1005700002602E4AA80602EBC302527848BF01224D
:100580004A62002240F2DC50294921F8120001326F
:10059000082AF7D10EA800211C22039317F0DFF9D7
:1005A00015F4007B05F4006A039B4FD0AA040BD41A
:1005B000BAF1000F0AD01F4A96F88401A2F10C018B
:1005C000012808BF0A4602E01B4A00E0194A0392CC
:1005D00014943DE0001BB700CB3300200005FA0562
:1005E00000080140001001400000014040420F009F
:1005F000B42F0020C821002010E000E0C800002037
:10060000F4920108000C0140FC2F00201022002071
:10061000DA12002014220020CDBD01089D10002018
:100620001831002018090020F810002044BB0108F0
:1006300008100020C4920108B892010800ED00E003
:100640007C310020E0920108E8100020CDF80CB0C9
:100650000E2B03D003F0EF03082B02D101238DF8FA
:100660004A30012011F0E2FD18B14088003018BF77
:100670000120C5F340038DF83E30C5F3403300F050
:1006800001008DF83830C5F3C0338DF83D008DF88A
:1006900040908DF83B30BAF1000F07D096F884A156
:1006A0000AF1FF3EDEF1000A4AEB0E0AC5F30043F1
:1006B0008DF841307B6A1BF1000B18BF4FF0010B26
:1006C000003318BF01238DF84330C5F30053B6F84B
:1006D00044018DF84430B6F84631ADF84E00ADF81F
:1006E0004830E804B6F8523148BFBD48ADF846304E
:1006F000C5F3804348BFB0F84C018DF83F30B6F8E1
:10070000503148BFADF84E00B3F5FA7FADF84C302C
:1007100084BF0023ADF84E3096F8D431B14887F845
:100720002830002387F8293043709DF84A3005F0BF
:100730000101002BC5F3C0028DF83CA08DF83910E3
:100740008DF83A208DF842B00CBF0023022301B986
:1007500002B1013308EB8308D8F840304FF00009AC
:10076000A3F1020A1A3304934FF6FF733AF8022FEB
:100770009A4200F094819DF83D10D3B2120AD6B28D
:1007800019B1991E012940F286819DF8401031B1BE
:100790009548190140589549884200F07C819DF8A0
:1007A00041E0BEF1000F06D08F48190140588F4933
:1007B000884200F070819DF83E1051B18A488C4DFE
:1007C00000EB03104168A94203D10189102900F010
:1007D00062819DF83B1051B18348854D00EB0310B9
:1007E0004168A94203D10189022900F054819DF892
:1007F0003C1051B17C487F4D00EB03104168A94289
:1008000003D10189022900F04681149F7FB1764D02
:10081000396805EB03156868884208D12989B888CA
:10082000884200F03881F888884200F03481022A3A
:1008300002D19DF8382003E0012A04D19DF8392027
:10084000002A00F028819DF84320674D1F015AB10E
:100850009DF84A2042B9A3F10802012A04D8EA59B6
:1008600065498A4208BF04269DF844203D4462B190
:100870009DF84A204AB9BEF1000F02D00C3B012B73
:1008800001E0043B032B40F2EE80012E4AD1564A90
:10089000DFF87081D119FF2391F80DE088F87030EE
:1008A00088F87130486801F1080309894FF0000B9E
:1008B000ADF8541002218DF8571088F874B015A9BE
:1008C000C8F880508DF856E00692059388F82CB051
:1008D000C8F830B0C8F834B0C8F838B0C8F86CB050
:1008E00088F872B088F873B00EF09DFB059B069AED
:1008F0009978D0595A4609F0B6F9284659463246F1
:100900000CF00AFC3D4BC8F88CB0C8F884303C4B66
:100910002846C8F8883008F1840108F188020CF0F4
:1009200043FCB8E0022E4BD15FFA89F31C2101FB96
:1009300003FC344B4FF0000803EB0C0B01238BF846
:1009400074300693284B8BF87590D91991F80DE007
:1009500001F10802486809898BF87680ADF85410D7
:100960008BF87E8015A9CBF88050CDF81CC08DF88F
:1009700056E005928DF857600EF055FB1A4B059A1C
:10098000D8599178424609F06EF9069B28461A46D6
:1009900041460CF0C1FB1C4A1A4BDDF81CC0CBF8D9
:1009A000842003EB0C01194A8431CBF88820CBF862
:1009B0008C8028460A1D0CF0F7FB09F101096AE05A
:1009C000032E4ED19DF83F300E4E114F13B396F8C3
:1009D0002A80284608214FF6FF72002335E000BF29
:1009E000E8100020F1000020C4B501080004004018
:1009F00000080140000C0140002C0140D596000881
:100A0000B5970008C8000020A19C0008AB9600081C
:100A1000C82F0020BDF84C2096F82A80B2F5FA7F46
:100A2000BDF84E300BD987492846B1FBF2F20821B8
:100A300092B209F06DF9844B47F828000AE0834927
:100A40002846B1FBF2F2012192B209F061F9804B24
:100A500047F82800C36096F82A30013386F82A3018
:100A600019E0042E17D1BDF84620784B794E93FB40
:100A7000F2F22846BDF84830012192B296F829706A
:100A800009F046F996F8293006EB87070133C7F8D5
:100A9000540186F82930049B9A457FF465AE6D4B6E
:100AA0006D4F93F82920002583F874216B4A3D701F
:100AB00016789846A6F11702022A1AD8D8F82030DC
:100AC0000021585903EB050913F016FF18B1D8F8A7
:100AD00024306BBB25E0624B05EB030E99E80F0059
:100AE0008EE80F003B7810350133C02D3B70E5D107
:100AF000EDE75C4B13F836C003EBC603D3F8049064
:100B000087F800C0B9F1000FE1D06545DFDA544A3B
:100B10002B0103EB020E4B440FCB01358EE80F0087
:100B2000F3E7514B1A68984612F4805F26D11FE014
:100B30004E4B4F4A13F8360003EBC6035D68107046
:100B4000002DEED000238342EBDAC3EBC3016A1819
:100B5000D2F80080DFF840C1013341F80C8001EB8E
:100B60000C0E9188AEF8041092798EF80620EAE710
:100B700006F0EF03082B3F4B24D125E03B78012BF7
:100B8000F6D93D4D05EB031303F110071035BD42B7
:100B9000EED055F8100C4FF07C5113F019FD4FF0CA
:100BA0007C5145F8100C55F8140C13F011FD4FF062
:100BB0007C5145F8140C55F80C0C13F009FD45F860
:100BC0000C0CE3E70E2E08D11A78182E42F0100212
:100BD0001A7008D111F00CFF05E01A78192E22F0D6
:100BE00010021A70F5E711F0E7FED8F80030234F35
:100BF0005E035EBF224B01221A70224A224E1378F6
:100C0000224843F0040313703B784FF48052022BC8
:100C100034BF142310238DF856304FF002038DF8A3
:100C20005730B369ADF8542043F00403B36134BFC7
:100C30000025012515A90EF0F6F9154B75B3154AD7
:100C40002DE000BF00127A00D597000840420F0047
:100C5000C5970008C8000020F82F002018090020C0
:100C60005408002044BB01087C31002004A5010881
:100C7000A4300020E01800205C080020CB330020C6
:100C8000800D0020A0330020001002400008014029
:100C9000B033002005220108A5300020BD4A002005
:100CA0001A6011F021FCBC4BBC4D93E80300B36902
:100CB00084E8030043F00803B361159816A90EF009
:100CC000B2F9F3694FF0030A43F48043F3613369E7
:100CD000284643F48043336118238DF8563021466B
:100CE0004FF42043ADF854304FF0040B8DF857A06B
:100CF0000EF099F94FF48043284621464FF480596D
:100D0000ADF854308DF856B00EF08DF9102328460A
:100D100021468DF85630ADF854900EF084F93369C1
:100D2000322043F480433361336923F480433361D9
:100D30009B4B1A8802F4415242F4457242EA0A027D
:100D40001A80998B072221F400610904090C998308
:100D50001A821A8892B242F040021A809F23C5F884
:100D600010908DF8343000238DF835308DF8363002
:100D70008DF8373011F099FB5A46C5F8149020468B
:100D80000DA912F069FCC5F810909DF856309DF839
:100D900055201B0243EA02439DF857201343814A22
:100DA000934214D0322011F080FBC5F81490F52046
:100DB00012F088FCFF2012F085FC7028C5F8109016
:100DC00005D13B78022B04BF774B83F800A03B781A
:100DD000032B0CBF1F20022006F025FF3B78032BBE
:100DE00003D001200EF070FB07E0022011F01EFA84
:100DF0000028F6D04388002BF3D06C4D4FF0100B39
:100E0000284600215A46D8F800403F7816F0A7FD42
:100E10004FF6FF73ADF83430022304F4004904F4B4
:100E200000684FF0000A1C408DF836308DF837A06E
:100E30000DD05F480DA9ADF834B00BF02DFE0423A2
:100E40002B700124072385F801A0AC70EB70012FF3
:100E50000FD9202356480DA9ADF834300BF01CFEF5
:100E6000052301222B72AA72631C07226C72EA729C
:100E7000DCB2B9F1000F0ED002234D480DA9ADF838
:100E800034300BF009FE0123E2182B71AB710723FC
:100E90006C71EB71D4B2B8F1000F0FD002233F4850
:100EA0000DA9ADF834300BF0F7FD092301222B73A7
:100EB000AA73631C07226C73EA73DCB273683D4843
:100EC00043F44043736073693A4F43F00103736125
:100ED000B36943F40073B3610BF0BAFB364B0026E1
:100EE0001593364B012C169394BF334680231A93E7
:100EF0004FF480731B934FF480631C93202315A938
:100F00001D9338464FF4005318941E931796199664
:100F10001F960BF085F93B68294A43F001033B60BB
:100F20005368012C23F4702394BF0021012123F482
:100F3000807343EA012353609168224B013C0B40CC
:100F4000314643F4602343F002039360D36AE4B272
:100F500023F4700343EA0454D46201236A1890789E
:100F600000286BD06C5C581C092CC0B2D278144F8E
:100F70002AD9A4F10A06D7F80CC006EB46064FF0B2
:100F8000070E0EFA06FE2CEA0E0EB2404EEA0202E0
:100F9000FA6026E01922010808930108000C0140BC
:100FA0000038004015202000CB33002020240020F2
:100FB00000080140080002404C2401403024002079
:100FC00000240140FDF7F1FF3E6904EB440C4FF0B3
:100FD000070E0EFA0CFE26EA0E0602FA0CF2324357
:100FE0003A61062B244E0CD85A1E776B02EB820214
:100FF0001F23934027EA030704FA02F33B4373637A
:101000001BE00C2B0CD8DA1F376B02EB82021F237C
:10101000934027EA030704FA02F33B4333630CE0EF
:10102000A3F10D02F76A02EB82021F23934027EA25
:10103000030704FA02F33B43F36203460431102929
:101040008CD10D4B9A6842F480729A609A6842F093
:1010500001029A609A6842F008029A609968064A0A
:101060000D070BD5FAE70BF1FF33092B8CBF0023DB
:101070000123FFF7F6B900BF00240140936843F055
:1010800004039360AC4B9A6812F004020492F9D105
:101090009A6842F4A0029A60A84BB3F8580100285D
:1010A00040F0A286B3F95A21002A40F09D86B3F998
:1010B0005C31002B40F09886A14D2B689C0320D515
:1010C000C82011F0F2F9AE200EF069F908B10EF067
:1010D0006BF99C4C84F87501C82011F0E6F99A4B25
:1010E0000021C4F87831994C0C22204616F037FCC8
:1010F0000223E3700DF077FA11F0B0F9944B03443A
:10110000A360944E8D4C336894F85F0194F8691194
:1011100094F86A21B3F956300AF00CFC059610B920
:10112000012011F035FA8C4A0A26137843F00203A5
:1011300013708A4B10225A6108221A61874F1920B6
:10114000FB68013E83F01003FB60FB6883F008033B
:10115000FB6011F0AAF9012011F0C6F9192011F075
:10116000A4F9002011F0C0F916F0FF06E6D108231B
:101170003B6110267A4B3E611B68180707D5794BF7
:101180007E611B689847784B01223E611A70774B4D
:1011900000271E68DFF80C82307B13F0C5F9744914
:1011A00013F016FA07F018FF724B1860724B18888C
:1011B00013F0BAF901464FF07E5013F0BDFA6F4BB1
:1011C0006B4918606E4B186913F002FA6D4B18608A
:1011D000307813F0A9F901464FF07E5013F0ACFAC5
:1011E000694B014618604FF07E5013F0E7F8674BEB
:1011F0004FF07E521860664B38469A601F605F6001
:10120000644B9A601F605F6007F0E6FE0646384652
:1012100007F070FE31460746304613F0D9F93946DB
:101220008246384613F0D4F931468146504613F0D1
:10123000CFF939468346484613F0CAF90146584665
:1012400013F0BEF83146C8F80000384613F0C0F974
:101250003146069013F0BCF9069B83463946184682
:1012600013F0B6F9034658461946069313F0A6F84C
:10127000069BC8F804001946584613F0A1F83946F1
:10128000C8F80800504613F0A3F93146074648460F
:1012900013F09EF90146384613F090F83E4F3F4B4D
:1012A0000026C8F80C00FF2138461B221E7016F0DD
:1012B00056FB38463E702A4E394B3268012112F0F7
:1012C000020F18BF797019701FBF03211970022116
:1012D000B970510741BF19784F1C1F70032748BFD1
:1012E000475412F00A0F0CD01A7804218154511C73
:1012F000C9B205274754D11C02321970D2B2062157
:1013000081542A68970641BF19784F1C1F70072720
:1013100048BF4754110608D51978092747548F1C30
:1013200001311F70C9B20A2747546779082F3BD093
:101330000E2F42D138E000BF00240140E810002009
:101340007C310020C800002070120020CC2D00202D
:10135000404B4C0018100020A0330020000C01402E
:10136000DC18002000220020E80500206820002072
:1013700035FA8E3C642000201C0000201C20002038
:1013800058210020202000207C2000206C200020FC
:101390008020002070200020E10F0020DB1F0020B3
:1013A000E00F002054200020197801F1010E83F88D
:1013B00000E04FF00B0E00F801E0197812F4803FC6
:1013C0004FF00C0C00F801C001F1010E1CBFDFF85A
:1013D00070C202315FFA8EFE83F800E01FBF8CF806
:1013E000001096494FF00E0C01F80EC0510748BF8F
:1013F00019784FF0120C41BF01F1010E83F800E0A3
:10140000102343548E4912F4806F0B7803F1010EC0
:101410005FFA8EFE81F800E000F803C00BD094F86C
:101420001CC2BCF1000F06D002330B70834B4FF08F
:10143000130C03F80EC00B7812F4007F4FF0140C5D
:1014400000F803C003F1010E1CBFDFF8F4C1023342
:101450005FFA8EFE81F800E01FBF8CF80030774BFA
:101460004FF0150C03F80EC0182F13D10B784FF066
:10147000160E00F803E003F1010E5FFA8EFE4FF046
:10148000170C00F80EC003F1030E0233DBB281F833
:1014900000E0C754130341BF69490B785F1C0F700C
:1014A00044BF1921C154D70541BF654A1378591C5F
:1014B000117044BF1A22C25400219822614816F0CC
:1014C0004EFA0AF06AF9604A604BB4F84E111A609D
:1014D0005F4BB4F8960119805E4900230B808B7036
:1014E0005D490A6081B25D4A22F813100133122B64
:1014F000F9D12B68D9045CBFB4F89C1111801B078B
:1015000040F1008194F89031062B00F2F580DFE87D
:1015100003F004070E395576760045F2F05201E0EB
:1015200042F6F8224E4B1A800AF0C0F9E3E042F688
:10153000F8224B4B1A8012F0F7FF4A4913F048F893
:10154000494912F03BFF13F02FFA0023474A42F8B3
:1015500023000133122BF9D1454A4649402011603E
:10156000454A137010F09AFE002800F0C580012350
:101570004FF0070990F9000040218DE808023F4A2A
:101580003F4BB3E042F6F822354B40201A803D4AEB
:10159000374B1A60384B10221A7010F07FFE00286B
:1015A00000F0AA8001234FF0000890F900004021CC
:1015B0008DE80801344A4FF4E13397E042F6F8220F
:1015C000274B40201A80314A294B1A602A4B0822A7
:1015D0001A7010F063FE002800F08E8001234FF097
:1015E000000C90F9000040218DE80810284A4FF4C3
:1015F000E13306F045FB274BC3F87C0178E042F667
:10160000F821174A062B11801B494FF00C02DFF816
:101610009CE0214F21480A704AD000233B708EF88D
:10162000003003701E4B1B2119701E4B4FF4E13725
:101630001A701D4B05221A7047E000BFE10F002011
:10164000E00F0020A820002070120020BC0E002017
:10165000C00E0020D4240020C8240020B83100206F
:10166000C2070020CDCCCC3F0000B044FC220020BB
:101670002400002089C300084421002001C600087E
:10168000A086010075C3000855C500085DC30008A9
:1016900009C50008C800002065230020642300203D
:1016A0006623002089220020672300208A22002050
:1016B0000021397001708EF800103C49212008701B
:1016C0003B493C4F0A703C4A13703C4A3C4B40201B
:1016D0001A6010F0E3FD78B101234FF0000E90F98D
:1016E00000008DE808403B46364A402106F0C8FA23
:1016F000003018BF012028B9082007F097FC324AB3
:101700002F4B1A602B68314A13F4804F1FBF0821FA
:1017100011702F482A4918BF086042F20101194090
:1017200099B144F620602B490880980441BF0821F4
:1017300011702948224948BF0860D90741BF0C21D0
:10174000117026481E4948BF086011781F06A1F194
:101750000401517040F185802148DFF890A04FF0DE
:101760000008204F41461522C0F880A1DFF8809084
:1017700000F5C27087F80180C7F80480C7F80880B8
:1017800016F0EDF8AAF105034046C9F800300CF058
:1017900034FA154B02201B68FB6010F07FFDCE462B
:1017A00040BB802007F042FC53E000BF66230020CE
:1017B0008922002090D003006723002085C2000802
:1017C00024000020E9C30008E5C3000844210020EC
:1017D000B9C30008C2070020D5C30008C5C300086C
:1017E000C80000201C070020A0310020DA120020D1
:1017F0003C07002090F805C07B78C5490C2202FB0D
:1018000003125278624504D00133DBB2042BF4D9C1
:1018100000237B70DEF800307A781B7890F90000A6
:10182000002B4FF00C0303FB021314BF4FF0030E09
:101830004FF0010E00225B78CDF800E0019202210A
:1018400006F01EFAB34B18600028AAD001200CF055
:10185000D4F9059B1868B04B00F5C5721A600CF0FE
:1018600073FA2B68980553D5AC4AAD4F039B4FF0E4
:1018700010083B609369AB4843F001039361039BFD
:101880000CA91B888DF83280ADF8303002238DF81A
:1018900033300DF0C8FB3B68A2485B880CA9ADF85B
:1018A000303004238DF832300DF0BDFB3B68012051
:1018B000197A0DF0A3FB3B689B4A5B684FF0000967
:1018C000536115A88DF859804FF0010815938DF8D4
:1018D00058908DF85A800BF0A1F83B680DA85B7A00
:1018E0008DF836908DF8343003238DF835308DF82F
:1018F000378011F093FE8D4B8D4A1B683C3B136083
:1019000033684FF0FF3243F010033360894B1A60A5
:10191000894B8A4A8A4E13608A4A803313602B6847
:101920000027D903377040F1B28040F22A39DFF83E
:101930004CA2DFF8E8B10FF02BFC4FF001084A464B
:101940005046394686F8008016F009F8DBF8183062
:101950007D4843F00403CBF818304023ADF8303015
:1019600018238DF833300CA903238DF832300BF097
:1019700093F8DBF81C30754A43F00203CBF81C30B7
:10198000734B744E1B68ABF6947BB3FBF2F3328857
:10199000013B22F45C721204120C32809BB21D22B5
:1019A000B2853385A6F81480338C23F001031B0421
:1019B0001B0C3384338CB188328B23F0020322F06A
:1019C000730212041B04120C1B0C89B242F0600259
:1019D00043EA0803B1803283B7863384338B23F024
:1019E00008031B041B0C43F008033383B6F8443090
:1019F0006FEA43436FEA53439BB2A6F84430DBF8E7
:101A0000A83F43EA0803CBF8A83F58460AF020FE57
:101A1000514BCDF858A0159380231A934FF480733F
:101A20004FF0100A1B9358464FF4005315A91E930C
:101A300019971C971D971F97CDF85CA0CDF8609063
:101A40000AF0EEFBB3890DA89BB243F40073B38197
:101A5000DBF8003043F00203CBF800308DF834A0FF
:101A60008DF835808DF836708DF8378011F0D6FD01
:101A70003A4B04991A683A4B43F821200B4601333C
:101A8000202B0493F4D10DF0DBF90DF0D9F92B687C
:101A90005A0540F19080334E334BD6F8C48404206D
:101AA000C3F8008010F0FAFB0421C6F8C80410F057
:101AB000D1FB2E4B86F8CC040820C3F8008010F030
:101AC000EDFB2B4B0821186010F0C4FB294F86F862
:101AD000CD04002138462C2215F041FF8E237B7067
:101AE0004FF07C0AE0234FF07D09FB7087F800A0DF
:101AF00087F82B90204F2C220021384615F02FFF1D
:101B00008A237B701020A023FB7087F800A037E0A9
:101B100080930108C82D0020100F00200010024003
:101B200018070020000C014000040140A0310020F3
:101B3000140700203810002014130020A8190020DA
:101B4000810D00200C2E00200008014000366E019F
:101B500054000020000400403404004010930108A9
:101B6000820D0020C8000020D01800202819002075
:101B700074190020F81800202D190020610200209F
:101B800087F82B90C6F8D08410F088FB1021C6F897
:101B9000D40410F05FFB86F8D8042020C6F8DC845B
:101BA00010F07CFB2021C6F8E00410F053FB86F80F
:101BB000E4040CF0EFFB734B734E1B78022B67D1E0
:101BC000724A00271388322023F040031B041B0CA9
:101BD000138013884FF4805823F038031B041B0C28
:101BE000138013889BB243F0400313809F238DF82A
:101BF00034308DF835708DF836708DF8377010F000
:101C000054FC8DF85570624F0422C7F8148015A853
:101C10000DA911F021FDC7F810809DF856309DF8F0
:101C200055201B0243EA02429DF857301343594A9C
:101C3000934219D00AD8A2F51A42033A93420CD023
:101C400002F51A420232934209D01CE0524A9342F2
:101C500005D00132934207D015E0202300E0802315
:101C600033804FF4807302E04FF4807333807380CD
:101C7000B38832881B02B3605343F360474B0122A1
:101C800083F8E52404E0002333807380B360F360BD
:101C9000F66826B3F60AB0464FF00009B1450BDAF4
:101CA00009EB06077F100DF1540AF8025146102285
:101CB0000DF026FB0F2807DC0CF0F8F9374B4FEA44
:101CC000C822C3F8E8240AE000235AF8232001328E
:101CD00054D10133042BF8D1B8463E46DEE72B68D9
:101CE0002F4A13F4002318BF0123137010F0B6FB22
:101CF0002C4B2D4918606379052B02BF2B4B4FF4F9
:101D0000C8721A802A4B4FF47A721A80294BC82263
:101D10001A80294A137843F008031370274A13786E
:101D200023F00203137040F602030A6813406BB1FC
:101D30002348244B1860244B03201870234B0120A8
:101D4000187023480023038022480380930341BF77
:101D5000214B04221A71DA7844BF42F00102DA7092
:101D60001E4B01229B680B601D4B1A701D4A137895
:101D700063F07F03137021B0BDE8F08F07F1010914
:101D80003746AAE7CB3300200C0000200038004083
:101D9000000C014018BA20001740EF00C8000020D6
:101DA000DC310020940700207C310020EE1F002051
:101DB000C2330020C0330020E0180020C9330020C7
:101DC00062120020C81800202C19002048000020B2
:101DD000B00F0020B20F0020CC2D0020E810002012
:101DE000800D0020A0330020424B00221A7000B268
:101DF00012F09AFB404912F0EBFB404C0646B4F956
:101E00005A0112F091FB3C4912F0E2FB0546B4F98D
:101E10005C0112F089FB384912F0DAFB04463046C7
:101E200007F0DAF88046304607F064F806462846A0
:101E300007F0D2F80746284607F05CF8054620462A
:101E400007F0CAF88246204607F054F8414681461A
:101E5000504612F0BDFB41468346484612F0B8FB9F
:101E600051460590304612F0B3FB49460690304685
:101E700012F0AEFB39460790504612F0A9FB204CF9
:101E80004946206007F1004012F0A2FB294660603D
:101E9000A560069812F09CFB0146059812F090FA96
:101EA0002946E060079812F093FB0146584612F06D
:101EB00085FA3946206106F1004012F089FB294677
:101EC0006061584612F084FB0146079812F076FADA
:101ED0002946A061059812F07BFB0146069812F096
:101EE0006FFA4146E061384612F072FB2062FFF75C
:101EF000E3B800BF3000002035FA8E3CE810002027
:101F0000FC230020954A2DE9F04F1568944C05F507
:101F10009C43944E20332360336889B013F4804F80
:101F2000059205D10AF096FF10B923790133237188
:101F30008D4A13784BB18D4909688D4240F2E58096
:101F400003F1FF3882F80080DFE09846884B5FFAA3
:101F500088F51F78DFF83892AF4231D9D9F80030D0
:101F6000072D98BF595D834B88BF29461B68804861
:101F70009847032D1ED8D9F8002005F10E0302EB77
:101F800083039988DA88A8B14FF47A73401A5843CA
:101F9000531A90FBF3F040F6C90300F57A709842AB
:101FA00005DC40F2EE239842B8BF184601E040F647
:101FB000CA0080B204EB4505E88008F10108C5E7D6
:101FC00094F804800325B8FBF5F50F2384F82A3034
:101FD00094F82B3005EB4505019394F82C30C5EBB4
:101FE00008050393D9F80030DFF8ACA10293EBB2F7
:101FF00004930025BD4255DA5F4B4FEA450933F89B
:1020000015B0019B53B90AF025FF28B1039B002BA3
:1020100008BF4FF0000B01E0DDF804B0029B988A86
:10202000584502D8D88A58450ED2E8B20AF0BCFE0C
:10203000032D8346DFBF94F82AE00120A8402EEA52
:102040000000D8BF84F82A000AF004FF18B14B48FA
:1020500029F800B022E0049B94F876002AF813B027
:1020600030B9B8F1020F15D93D4B012083F8760045
:10207000BAF80000BAF802300344BAF80400034486
:102080003F489BB229F800301BB2032093FBF0F3CA
:102090009BB200E05B46394829F8003001350AF16F
:1020A000060AA7E794F82A203648A2F10F014A420F
:1020B0004A4184F89020344B6AB1344A1268520184
:1020C00009D40268D9689A60521AC82A1DD9012217
:1020D00083F8212019E002689868DA605B68121AB8
:1020E0009A4288BF284B4FF0000184F82B1088BF1C
:1020F00083F821100025BD4207DAE8B20AF054FE49
:102100001E4B23F815000135F5E73368DD0405D5CE
:102110001E4B1B68D80701D411F0F6FE059B1F6803
:102120001B4B1A68907A002838D01449137B013869
:1021300031F810001BB1C0F53B60083080B200B22E
:10214000A0F57A70B0F57A7FA8BF4FF47A7020EAD4
:10215000E07012F0E9F90F4955E000BFAC33002000
:10216000100E00207C310020D0240020CC24002040
:102170004421002024000020160E0020B831002049
:10218000880E0020A0310020D4240020DC0F002085
:10219000C824002000007A443E0E00203368190451
:1021A0003AD5D4F89430934DFB1A002B34DB07F565
:1021B0009C432033C5F894308F4BD27A59798F4B9A
:1021C00033F8113095F898109BB293FBF2F301317C
:1021D00001F00F0285F898202A4482F899300346CE
:1021E000874A825C0130134410289BB2F8D11BB29D
:1021F00093FBF0F000B26428A8BF642020EAE070EE
:1022000012F092F97F4912F097FA7F4912F0E0F943
:1022100012F0CAFB7D4B188033687D4D13F4807F2C
:1022200000F00F817B4BDFF8F0919F4205D999F8C0
:10223000022012B9012289F8022099F80220002A0E
:1022400000F0FF80744A95F8008092F82170C8F37E
:1022500080087A1E57425741704A002F92461168F3
:1022600018BF4FF0000BC1F38063019308BF4FF01C
:10227000030B99F82020052A00F2DD80DFE802F048
:10228000034E537988A5B8F1000F3AD0D4F8AC00CA
:10229000B4F8B01010F09FF8012809D16049614AE4
:1022A00009681268C988642000FB0122C9F810205F
:1022B000019B6BB15A4A126812794AB10EF0DAFEEC
:1022C000032289F820204FF47A72C9F81C20D0E745
:1022D000002F40F0B080534AD9F8101010684E4AD1
:1022E00088420AD902920EF0C5FE029A032182F8B2
:1022F000201040F6B831D161BBE7012182F82010EF
:10230000B7E7019B4FF4806013B106F07FFE01E058
:1023100006F06CFE0022C9F810208CE0002F49D195
:102320000EF0A8FEA5E727B1052289F8202001209C
:1023300000E03846B8F1000F0CD0D4F8AC204FF0D4
:10234000020BD189384A1180518091803449096843
:102350004988D180334A1168D9F81420914202D8B3
:10236000B8F1000F64D147F23052C9F81C200322A3
:1023700021E02A7842F002022A7011F0C5FD294AB4
:10238000D9F81C1012680A44C9F81820042212E077
:10239000244A9FB11168D9F8182091424BD9234A99
:1023A00012781AB9DAF80020D30744D42A7822F038
:1023B00002022A70052289F820205AE71268D9F80B
:1023C0001C100A44C9F8182035E01549154A096857
:1023D0001268C988642000FB01224FF48060C9F8AC
:1023E0001020002289F8202089F8032006F0FEFD45
:1023F0003FE700BF100E00202024002030240020E2
:10240000A90E00200000C84200C07F443C100020FC
:10241000C9330020404B4C00D4240020DC0F0020A6
:10242000382E0020A0310020B83100200800002004
:1024300000287FF41EAFBBF1000F02D0584610F009
:102440006DF8924F07F5C470B7F84E110FF0C3FF47
:102450000197834668B90EF0FFFD8D4B0022C3F84B
:1024600000B0C3F804B0C3F808B08A4B1A605A60D1
:102470009A602B785F0736D53368D80633D5864BFC
:102480001B78D9062FD4854B1B789BB1019B93F801
:10249000E031BBF1000F15D17BB1814B1A68D4F844
:1024A000B4309B1A002B08DA11F02EFD7D4B83F817
:1024B000B8B018E0BBF1000F0DD1102010F02EF8CD
:1024C00001230EE03BB1764A4FF47A71126801FBAA
:1024D0000323C4F8B43094F8B83023B110F00AF8EC
:1024E000002384F8B830019B93F8DEA193F8DF1144
:1024F000B3F898E1B3F89AC1002318466A4F8008F0
:1025000037F9132001337245C4BF60F07F00C0B2B9
:102510006245B8BF40F04000042BB946EED194F8B4
:10252000B930604A834205D192F8BA30F92B04D809
:10253000013300E0002382F8BA30584B84F8B90028
:102540001A785A4F9846E2B93B68DA0708D5BBF1CA
:10255000000F16D12B78DB0713D511F025FB10E007
:102560002B7858070DD54F4B93F82B304BB1504B70
:10257000DB7833B911B111F0C7FC02E0BBF1000FF9
:10258000F9D094F8BA30474A142BDFF840B140F044
:10259000AF8098F800301AF1000A18BF4FF0010A16
:1025A0006BB392F8B9305F2B11D12B7803F0040391
:1025B00003F0FF0113B111F0A7FC08E00B20039119
:1025C00002920FF0ABFF029A039982F8BA10BAF1A7
:1025D000000F14D094F8B9307D2B10D12B7803F074
:1025E000040303F0FF0213B111F08EFC07E00B208F
:1025F00002920FF093FF2B4B029A83F8BA202B78AC
:1026000003F0040303F0FF01002B71D194F8B930FB
:10261000244A572B15D1274B4FF47A721A8033680E
:10262000190601D50BF0E0FB234B1B685A0742BF8C
:10263000224A0A21118013F0080359D1204A13803D
:1026400056E03068400716D55A2B14D11D4B187828
:1026500020B119701C4B01221A7049E092F8BB306E
:1026600083F0010382F8BB300BB10C2000E00D2099
:102670000FF054FF3CE05D2B00F01D855B2B00F05C
:102680001C855E2B24D1032000F018BDE81000202B
:10269000541F0020B81F0020E01800200800002070
:1026A000A0310020100E0020B8310020DC0F0020E7
:1026B000D4240020C2330020DC180020C0330020C6
:1026C000D8100020192000201A2000201810002007
:1026D000562B01D106F07EFF98F80030002B00F059
:1026E000038594F8B9306F2B40F0F88411F05CFA50
:1026F0003368580732D594F8BB30A3B12B7859070B
:1027000011D5019BB9F90620B3F898319A420ADD38
:102710003B6813F0010301BFAC4A32211180AC4A7F
:1027200008BF82F8BB303B68DA030AD5A94B1A7898
:102730002AB9A94A127812B9A44A32211180012279
:102740000BE0A54A13784BB12B7803F0040303F098
:10275000FF011BB9A14B117001221A70DBF8009028
:1027600000233B6009F17B0809F1CB0A98F80020AF
:1027700098F8013018F8010C9A420BD241460FF03C
:10278000F5FD38B118F8022C012303FA02F23B6878
:1027900013433B6008F10408D045E7D1904B1B7808
:1027A00053B1904B904F1A68984612F0020FDFF821
:1027B000509240F0388330E309F1CA0709F589786F
:1027C0003A787B7817F8010C9A4225D239460FF0F7
:1027D000CDFD08B397F804E00C21BB7801FB0E4156
:1027E000824A013B03EB43031344D1F8C02097F81E
:1027F00003909A4276480FD0C1F8C030002390F879
:10280000EC20C1F8C430012303FA0EF322EA0303DB
:1028100081F8BC9080F8EC3006374745D0D1744B36
:10282000DFF8E0A1D3F80080724B4FF0000B1B687B
:10283000029394F82B300393DAF80030002B00F069
:10284000E38293F80090B9F1000F00F0DD82DAF82E
:10285000042002998A1A002A0CDB01F5FA72CAF8E0
:10286000042094F8EC10012202FA0BF221EA020291
:1028700084F8EC20039A002A00F0C6821AF8042C8F
:1028800059780432D2B2002940F07F825A4931F996
:1028900012105A4AB2F8962102F1C800814201DDB5
:1028A0009F7814E0C83A914202DA99784F420EE0DC
:1028B00094F8EC20012303FA0BF322EA030384F8D3
:1028C000EC30029B03F5FA73CAF804309CE294F8EA
:1028D000EC3043FA0BF3DB0700F19682002FCCBFFC
:1028E000022001200FF03CFE09F1FF32384B132A81
:1028F00000F28282DFE812F014002300320044006C
:1029000061008800ED005201B701EA01190280025E
:10291000440055008800ED005201BF0024018901E8
:1029200098F8001040460F44FA2FA8BFFA2727EA6C
:10293000E77788F800700FF0FFFC01201EE098F8A0
:10294000011040460F44642FA8BF642727EAE777A9
:1029500088F801700FF0F0FC02200FE098F80310E7
:1029600040460F44642FA8BF642727EAE77788F81A
:102970000370D3F8F0100FF097FC03203946D1E133
:1029800098F805100D2039446429A8BF642121EA74
:10299000E17188F805100FF04DFDB9F10D0F00F051
:1029A0002B8298F804100E2039446429A8BF6421B2
:1029B00021EAE17188F80410B4E198F806100520C6
:1029C000394481F3080188F80610ABE100200020AB
:1029D000100E002018200020192000201A200020AE
:1029E000CE330020DC0F0020DC180020889701087F
:1029F00040100020A0310020B8310020E810002055
:102A0000A4190020D00E0020D3F8F4301A78022A3E
:102A100022D13846049311F087FDA94911F08CFEAC
:102A2000049B596A059311F0CBFC0021049011F02E
:102A30006DFF059B48B9049AA149104611F084FF27
:102A4000049A059B10B19E4A00E000225A620F20B2
:102A500011460FF0DBFC0AE099780F203944C829B1
:102A6000A8BFC82121EAE17199700FF0E3FCB9F128
:102A70000F0F00F0C181934BD3F8F49099F8003018
:102A8000022B1AD1384611F04FFD8D4911F054FE3A
:102A9000D9F8201011F094FC0021074611F036FF00
:102AA00030B93846864911F04FFF10B1844F00E02D
:102AB0000027C9F82070122057E199F80110122060
:102AC0003944C829A8BFC82121EAE17189F8011059
:102AD00028E1D3F8F4301A78022A22D13846049338
:102AE00011F022FD764911F027FE049B196B059326
:102AF00011F066FC0021049011F008FF059B48B915
:102B0000049A6F49104611F01FFF049A059B10B1FB
:102B10006B4A00E000221A63102011460FF076FC89
:102B20000AE0197B10203944C829A8BFC82121EA2E
:102B3000E17119730FF07EFCB9F1100F00F05C81A8
:102B4000604BD3F8F49099F80030022B1AD1384634
:102B500011F0EAFC5A4911F0EFFDD9F82C1011F0F0
:102B60002FFC0021074611F0D1FE30B938465449F8
:102B700011F0EAFE10B1524F00E00027C9F82C70A6
:102B80001320F2E099F80B1013203944C829A8BF8C
:102B9000C82121EAE17189F80B10C3E0D3F8F430C1
:102BA0001A78022A22D13846049311F0BDFC464916
:102BB00011F0C2FD049BD96B059311F001FC0021BB
:102BC000049011F0A3FE059B48B9049A3C491046B5
:102BD00011F0BAFE049A059B10B1394A00E00022B8
:102BE000DA63112011460FF011FC0AE0997D1120E3
:102BF0003944C829A8BFC82121EAE17199750FF0AD
:102C000019FCB9F1110F00F0F7802E4BD3F8F490B6
:102C100099F80030022B1AD1384611F085FC2A4968
:102C200011F08AFDD9F8381011F0CAFB00210746CF
:102C300011F06CFE30B93846214911F085FE10B113
:102C40001F4F00E00027C9F8387014208DE099F874
:102C5000151014203944C829A8BFC82121EAE17100
:102C600089F815105EE0D3F8F49099F80030022B43
:102C70001AD1384611F058FC114911F05DFDD9F810
:102C8000281011F09DFB0021074611F03FFE30B9DE
:102C900038460B4911F058FE10B1094F00E00027EB
:102CA000C9F82870092060E099F803100920394418
:102CB000C829A8BFC82121EAE17189F8031031E0D1
:102CC0000000C842100E002000007A44D3F8F490AF
:102CD00099F80030022B1AD1384611F025FCB4497E
:102CE00011F02AFDD9F8341011F06AFB00210746D3
:102CF00011F00CFE30B93846AD4911F025FE10B187
:102D0000AB4F00E00027C9F834700A202DE099F895
:102D10000D100A203944C829A8BFC82121EAE17151
:102D200089F80D100FF086FB66E0D3F8F49099F85F
:102D30000030022B1DD1384611F0F6FB9D4911F0F1
:102D4000FBFCD9F8401011F03BFB0021074611F0C5
:102D5000DDFD30B93846964911F0F6FD10B1944FBB
:102D600000E00027C9F840700B2039460FF04EFBF9
:102D700042E099F817100B203944C829A8BFC82190
:102D800021EAE17189F81710CCE7012934D198784C
:102D9000894B33F91230B3F5617F05DB40F633021E
:102DA0009342A8BF134601E04FF46173B9F10C0FD1
:102DB00022D14FF4966292FBF0F0A3F5617393FB7E
:102DC000F0F37E4ADFB21378BB4215D0042F34BF34
:102DD0003B4602231370019A09FB0323784A03F24E
:102DE000B673136006F002FA484639460FF022FB2C
:102DF000781CC0B20FF0B4FB94F8EC20012303FA66
:102E00000BF3134384F8EC300BF1010BBBF1040F0F
:102E10000AF10C0A7FF410ADC3E43368D80510D56D
:102E2000684BDB786BB13B6899070AD5B9F800307D
:102E300013F0010A0AD10EF00FF9012006F0E6F8AE
:102E400004E0012006F0D2F8012300E00023D8F8C6
:102E5000002052070DD563B1012006F0C7F8B9F87C
:102E600000309B0708D40EF0F7F8022006F0CEF8E9
:102E700002E0022006F0BAF8B9F80030524A13F026
:102E8000030F4FF0100114BF516111613A6812F045
:102E90000A0F27D0D8F80020D00609D559070AD440
:102EA000042006F0B3F8494B1B88A4F8F83002E080
:102EB000042006F09BF8D8F800309A0607D5B9F838
:102EC00000305B0606D4402006F0A0F802E0402067
:102ED00006F08CF8D8F80030580642BF3B4B1B88F0
:102EE000A4F8FA303B68990609D4D8F800301A05DE
:102EF00040F1B0804FF4807006F088F8AEE0344BBB
:102F00001B789B076ED5334B1B78042B6AD9D8F8F6
:102F1000003013F4007A0FD0B9F80030DF063AD44D
:102F2000102006F073F8202006F060F82A48011DF2
:102F30000AF0C4FE02232AE0B9F8007007F0100777
:102F4000BFB22FB1102006F051F8012784F8FCA081
:102F5000D8F80030580512D5D4F800311F495A89E5
:102F6000B1F90030002BB8BF5B42934207DAB1F9E8
:102F70000230002BB8BF5B429342C0F20781B9F820
:102F80000030990608D5202006F030F8002384F898
:102F9000FC30012700E0002794F804319BBB0E2091
:102FA0000FF0BCFA0E4B012283F804212BE000BF86
:102FB0000000C84200007A44B831002034310020BB
:102FC00040100020D4240020000C0140D810002024
:102FD000E0180020E618002048100020E010002033
:102FE000100E0020B9F8003003F03003002B3FF43E
:102FF0007CAF102005F0FAFF202005F0F7FF00233A
:1030000084F8FC3002E0002F3FF46FAF002214463A
:103010006B4B002023F814006A4B191D03F10A07BB
:1030200021F814000021D15117447860B96023F8C9
:10303000140003F132075A33D151D15017441344CD
:103040007860B960586099601432002C7FF44DAFFD
:103050000124DDE74FF4807005F0C8FF5A4B5A7920
:103060001C46082A01D00E2A02D1402005F0BEFFDE
:1030700033685A0540F1A08094F81C321BB92B78B4
:1030800013F0040F03E0D8F8003013F4002F0BD036
:103090004E4B00221A703C2009F090F8002800F0F6
:1030A0008B800FF0EFFFF6E70BF074F909B0BDE885
:1030B000F04F08F072BB012000E002205FFA80F8B8
:1030C000019A08F1FF3382F8B43705F0E9FF06F002
:1030D000B1F840460FF044FAFFF70ABBBAF1000F0F
:1030E00002D07E2B3FF402AB94F8B930972B05D178
:1030F000374B4FF4C8721A80FFF7FABAA72B06D1E4
:10310000344A137843F004031370FFF7F1BA002236
:10311000BB2B079201D1022303E0B72B04D14FF65A
:10312000FE73ADF81E3009E0BE2B01D1022303E08F
:10313000BD2B1AD14FF6FE73ADF81C30DBF8003012
:10314000BDF81C10B3F858200A44A3F85820BDF865
:103150001E10B3F85A200A44A3F85A2006F03AFA8F
:10316000002384F8BA30FFF7C3BA792B04D11A4A86
:10317000D37823F0010306E07A2B7FF4B9AA164A2C
:10318000D37843F00103D370FFF7B2BAB9F8003037
:103190009B063FF501AF202005F038FF0F4B10488C
:1031A0001A685B68011D436002600AF087FD0D4BE1
:1031B000012783F8FC70EFE609B0BDE8F08F00BF8F
:1031C000C4330020160F0020E81000200C2200203D
:1031D000EE1F0020E0180020CC2D0020E818002071
:1031E00050100020100E0020BA4B2DE9F04FB3F91B
:1031F0000610B94B89B01F6801937A8991420EDBA2
:10320000B1F5FA6FFC79BFBF8B1A6343A2F5FA647C
:1032100093FBF4F4ACBFC4F16404643400E06424B0
:10322000AE4BAF4A1868B2F896A1054692F95E21F6
:10323000049092B205920293002240F2E630A54B30
:103240004FEA420B33F912300393CAEB030303F244
:10325000F316864203D8002BB8BF5B4201E04FF45F
:10326000FA73022A049E4FF064002FD096F811E101
:10327000BEF1000F04D07345CCBFCEEB0303002397
:1032800093FBF0FCDFF8A0E26FF063093EF81C80CE
:1032900009FB0C390CF1010C3EF91CE00FFA88FC1B
:1032A000CCEB0E0E0EFB09FE9EFBF0FE8D4EC644CF
:1032B00026F80BE0BE18367973438B4E93FBF6F37A
:1032C00064339BB2634393FBF0F02DE096F812E178
:1032D000BEF1000F04D07345CCBFCEEB0303002337
:1032E00093FBF0F0DFF82C826FF0630C0CFB0039DD
:1032F00038F910E0013038F91000002BCEEB000057
:1033000000FB09F999FBFCF90598CEEB090909FBCB
:1033100000F97448B8BF5B42A0F80490B879434301
:10332000714893FBF0F064306B784FF0640E4343C8
:1033300093FBFEF36D4E022AB354EB7A6C4E00FB06
:1033400003F393FBFEF3B3546B7D664E00FB03F077
:1033500090FBFEF0674B9854674B0FD183F802E067
:10336000039B53450EDB5E4CB4F89821914215DB6C
:10337000B1F5FA6FA8BF4FF4FA6110E09C54039BBB
:10338000534504DA36F80B305B4226F80B30013235
:10339000032A05F101057FF450AFE4E71146891ACD
:1033A0004FF47A735943C2F5FA62B1FBF2F1642724
:1033B00091FBF7F2DFF874E16FF063033EF812005F
:1033C00003FB021101323EF9122003B2D21A51431B
:1033D00091FBF7F30344F380484B424D1B885F0693
:1033E0003BD5474A474B10881B88181A00B211F08A
:1033F0009BF8454911F0ECF8074605F0EDFD8046D5
:10340000384605F077FD0746B5F9020011F08CF853
:103410008146B5F9000011F087F84146824611F067
:10342000D7F839468346484611F0D2F80146584647
:1034300010F0C4FF11F092FA41462880484611F07E
:10344000C7F839468046504611F0C2F8014640465A
:1034500010F0B6FF11F082FA68802C4F3B68980795
:1034600040F19F8045F20721294B2A4D1A686B696C
:10347000D31A8B4240F395806A6109F07BFC264B9E
:10348000DFF8AC901A789846032AB9F8003051D189
:103490000A2B59D90023282088F800300FF005F8AE
:1034A00009F068FC1D4B188809F04EFC1C4B1A688B
:1034B000D37890FBF3F0013008281A4BA8BF0820FE
:1034C0001870537980B243432B8313795843688330
:1034D0003AE000BFB8310020401000201810002052
:1034E000E8100020E01000200CFEFFFFC41F0020A9
:1034F000A60F0020D81F0020441F0020A419002080
:103500000A0F0020D810002035FA8E3C7C310020B4
:10351000AC330020980F00202C1900203824002004
:10352000C818002048000020A62F00208E2F002061
:10353000CC1800200A2B07D803239C4A88F80030B7
:10354000002313702B836B8398F80030984A012B6B
:103550000CD002D3022B1BD023E02A8BB9F8003009
:103560009A421EDD012388F800300FE0B9F8001000
:103570006B8B8B4202DD022313700FE08D4B1B8B94
:103580000133994202DD002313700AE0082006E0AF
:103590006B8BB9F8002001339A42E3DC07200EF070
:1035A000BDFF3D68290577D5834B824F1A68FB69BB
:1035B000C3EB020845F2072398456DDD7F4BB6F952
:1035C00006B0D3F800904FF47A7099F80A30FA6197
:1035D000012B98FBF0F8B4F84E11ABF57A7B784EDE
:1035E00003D042D3022B20D041E0764B396A5A7B7C
:1035F000754B4FF0080E33F8122091FBFEF392B298
:10360000C91A8B183B6293FBFEF3BA8440F6E4427E
:103610009BB25343B9F80820C2EB13335843B9F9AE
:10362000063090FBF3F0306021E0684BB9F808A059
:103630001B78C6F800A05A0719D565480EF0CBFED6
:1036400020B915F0100F18BF4FF0000B0BFB0BF358
:10365000322293FBF2F3B9F906205B445A434FF44C
:103660007A7392FBF3F3534400E000233360336832
:10367000D7E90A0103FB08F84FF47A7398FBF3F8D3
:1036800010EB080041EBE8710023C7E90A01514A39
:1036900011F0AAF9504B1860504E3368DB0427D55F
:1036A0002F0622D54E4B1B789D071ED54D4B187803
:1036B00004281AD900224C4B0521D718951C4FF02D
:1036C0000A0E122AD154E9B287F801E004D0B0EB17
:1036D000510F2A46EFD800E014215A18322002F880
:1036E000010CFF225A540F2000E00A200EF016FFB2
:1036F0003E4D2A68002A51D03D4B3E4F186839682C
:10370000984681424AD83C4BDFF8F89019785268C5
:10371000E1B94FF0010A83F800A0B9F80030D35C9A
:1037200023B350460EF0E0FE344B83F800A009F0BE
:103730009DFBB9F80030CBB92B681B78053B53458E
:1037400014D80EF08BFE2E4B18600FE04FF0000ADD
:1037500083F800A0B9F80030D35C3BB150460EF0BE
:10376000C3FE264B83F800A009F080FB2B68B9F854
:1037700000205B6823499B5CFE2B02D100230B8059
:103780000CE0FF2B02D10EF0B5FE07E0D8F80000E8
:103790000A2505FB030301323B600A800B4D2B78A1
:1037A000580733D5184B08225A616DE048000020B5
:1037B0002C190020980F0020AC330020C8180020DE
:1037C000D41800202024002030240020C9330020F9
:1037D00070120020407E0500D8180020DC0F002069
:1037E000E0180020E618002054310020C42F0020EB
:1037F000A0310020BC2F0020B82F0020F82400208A
:1038000090330020C02F0020000C01403268D10707
:103810005CBF43F001032B709A4B1B781F075EBF00
:103820002B7823F001032B70D60248BF2B78964AE1
:1038300044BF23F001032B70944B1B6813F0040F5B
:1038400002D09349098851B99249098809B198076A
:1038500005D4914B1B88003318BF012333B10223D9
:1038600013702B7823F001032B7004E02978C9072B
:1038700058BF022313700EF0F1FD884B1B68C01A6D
:10388000002801DB09F0F2FA854F0AF083FD3E784B
:10389000002E00F0AD80834B1A689846002A00F095
:1038A0003887D8F800000EF0DBFE002800F03187E2
:1038B0007C4B7D4C18680EF0D0FE092801D03F28C3
:1038C00052D14FF0000A55462668DFF8FC9136B118
:1038D0007648D9F80010324614F08EF810B9CA466E
:1038E00005B94D46724B09F110099945EFD3EDB179
:1038F000D5F800C0DAF8009023681CF803E019F846
:103900000300704512D15A1C684958B92D2B09D8AB
:10391000DFF894E1CEF800204FF0200E01F803E02C
:10392000885403E001F803E02260E5E723680BB167
:10393000554510D05F480FF09BFC554507D855F80A
:10394000100B0FF095FC09200FF08AFCF5E75A48A0
:103950000FF08EFC002623689E42A2D2534B985D46
:103960000FF07EFC0136F6E72368002B40F0B786A7
:10397000042840F0F2864D480CF03CF800F0C9BE37
:10398000D8F80000DFF83CA10EF06AFE30B3DAF898
:1039900000000EF062FEDBF80030024693F848109B
:1039A000B1BB242840F09480012283F84820DBF842
:1039B0000030DFF818A193F84820062AE0D193F8E8
:1039C000490000F057FF8346002800F0AB800FF05D
:1039D000A7FBD9F80030002283F84820374B93F832
:1039E0003530002B40F069864C36982E00F09186D9
:1039F000334BF21892F84A100129F5D1DFF8CC9038
:103A0000F358C9F800202F4ACB4613609046B7E719
:103A1000012904D14D2814BF00220222C5E7022942
:103A200004D13C2814BF00220322BEE703290CD195
:103A300040284FF0000102D983F84810B7E75871C9
:103A40001971D97198710422AFE7042906D19979C7
:103A500083F849004A409A710522A6E70529A6D1B4
:103A6000587919798842987906D950409871481C3C
:103A700018710B441A729AE790420CBF062200227A
:103A800093E700BFE0180020F8240020DC18002095
:103A9000C0330020EE1F0020C2330020FC24002091
:103AA000CE33002050310020082E0020D82D0020D9
:103AB00044A40108D0B90108D5B90108980F002025
:103AC000A82000208819002064A201088419002081
:103AD0002B78CC4958073FF56AAF232ADAF8003033
:103AE00013D101203870C84804910360C74803927D
:103AF0000363C7480FF0BCFBC6480FF0B9FB04993D
:103B0000039A0B7843F002030B70C34B1B681B78BE
:103B1000934201BFC14AC24B1A60C24A04BFC24BA2
:103B2000DA6044E7DAF8002092F849304C2B00F0D4
:103B30007B845CD8332B00F0B28421D8292B00F091
:103B40003F8409D8252B00F01784272B00F01A8416
:103B5000232B40F0FE8503E22D2B00F0428407D892
:103B60002B2B40F0F6850FF0ADFA607100F0A0BD90
:103B70002F2B00F00085312B00F02A8500F0E9BDE5
:103B80003E2B00F0BD801DD8372B00F0BB8404D83D
:103B9000352B00F01E8200F0DCBD392B00F0FF83D6
:103BA0003C2B40F0D685DFF89082D8F800A00FF0CB
:103BB00089FA8AF80000D8F80030187807F0CEFAB1
:103BC00000F076BD432B00F07B8406D8412B40F0FB
:103BD000C0854FF0000800F067BC442B00F02D8535
:103BE000482B40F0B6850AF09FFA00F061BDD12B5A
:103BF00000F083831FD8CC2B00F013820ED8C82B83
:103C000061D004D84E2B00F01C8400F0A2BDC92B5B
:103C100000F04C83CA2B7DD000F09BBDCE2B00F072
:103C20003883C0F02D83CF2B00F04F82D02B00F0D3
:103C30001C8300F08EBDD82B00F024810BD8D32B31
:103C40003BD027D3D42B00F08482D62B40F0818543
:103C50004FF0000872E2F22B00F0DC8212D8EF2B5A
:103C600040F07785DFF8D081D8F800A00FF034FA63
:103C7000AAF85A00D8F800800FF02EFAA8F85800D9
:103C800000F016BDF32B00F0DD84FA2B00F00A8360
:103C900000F05FBD2B7803F0040303F0FF08002B56
:103CA00040F006850FF00EFA022884F8B40740F2BF
:103CB000E2825E4B83F8B487DDE20FF00DFA5C4BD5
:103CC000188000F0F5BC92F805804FEA5808B8F16A
:103CD000120F03D908F06EFA00F0EABC4FF0000AA8
:103CE000C24507D20FF0F8F9524B23F81A000AF137
:103CF000010AF5E7454B012283F8342000F0D8BCD7
:103D00000FF0E0F984F8E0010FF0DCF984F8DF014E
:103D100000F0CEBC484B1A6898461278022A40F050
:103D200093804FF00008DFF810A108F1080BDAF8D3
:103D3000003003930FF0C6F910F0F2FB3F4910F08A
:103D4000FBFC039B43F82B00DAF800B00FF0BAF944
:103D500008F10A030BEB830B10F0E2FB384910F07B
:103D6000EBFCDAF80030CBF8040003930FF0AAF96B
:103D700010F0D6FB334910F0DFFC08F10E0B039B6B
:103D800008F10108B8F1030F43F82B00CBD1B8F1CB
:103D9000070FDAF800B01AD10FF094F910F0C0FB59
:103DA000264910F0C9FCCBF84400DAF800B00FF057
:103DB00089F910F0B5FB214910F0BEFCCBF84800A2
:103DC000DAF800B00FF07EF98BF84C0012E00FF03B
:103DD00079F9C3448BF80100DAF800B00FF072F9FA
:103DE000C3448BF80B00DAF800B00FF06BF9C34452
:103DF0008BF8150008F10108B8F10A0FC7D100F0DF
:103E000057BC00BFC933002050310020980F00205C
:103E100005BA0108D5B9010810220020EFBEADDEB9
:103E2000F04F00200400FA0500ED00E0E81000204B
:103E3000080F0020B8310020181000200000204199
:103E40000000C84200007A444FF0000AD8F800B0E1
:103E50000FF038F9D3448BF80100D8F800B00FF018
:103E600031F9D3448BF80B00D8F800B00FF02AF9E1
:103E7000D3440AF1010ABAF10A0F8BF81500E5D113
:103E800000F016BC8046DFF880A308F1080BDAF8D2
:103E9000003003930FF020F910F042FBD44910F0EA
:103EA0004BFC039B43F82B00DAF800B00FF014F939
:103EB00008F10A030BEB830B10F032FBCC4910F036
:103EC0003BFCDAF80030CBF8040003930FF004F960
:103ED00010F026FBC64910F02FFC08F10E0B039BD7
:103EE00008F10108B8F1030F43F82B00CBD1B8F16A
:103EF000070FDAF800B01AD10FF0EEF810F010FB4F
:103F0000BB4910F019FCCBF84400DAF800B00FF010
:103F1000E3F810F005FBB64910F00EFCCBF84800B2
:103F2000DAF800B00FF0D8F88BF84C0012E00FF080
:103F3000D3F8C3448BF80100DAF800B00FF0CCF8E6
:103F4000C3448BF80B00DAF800B00FF0C5F8C34497
:103F50008BF8150008F10108B8F10A0FC7D1A7E3E3
:103F60000FF0B0F8132883463FF6B4AEDFF898A2FE
:103F7000DAF800800FF0A6F800239E490C2202FB1D
:103F80000312117A814220D1137808EB8B0888F84C
:103F900079300FF097F888F87A000FF093F888F8E6
:103FA0007B000FF08FF8944A944B88F87C001A60DD
:103FB000DAF80000924B0021186079300EF0FAF91F
:103FC000904B80F00100187072E301331C2BD4D1A8
:103FD00080E60FF077F80B2882463FF67BAE8A4BDF
:103FE000D3F800800FF06EF803283FF673AE062377
:103FF00003FB0A8888F8CE000FF064F888F8C9003F
:104000000FF060F888F8CA000FF05CF888F8CB0071
:104010000FF058F888F8CC000FF054F888F8CD006D
:1040200046E35379092B7FF655AE019BD3F8008008
:104030000FF048F8019B88F80000D3F800800FF0DB
:1040400041F888F801000FF03DF8019B64281B68D7
:10405000A8BF642018710FF035F8019B64281B6815
:10406000A8BF642058710FF02DF8019BFF281B6832
:10407000A8BFFF2098710FF025F8019B6428D3F8A2
:10408000008028BF642088F807000FF01BF8019B10
:1040900088F80200D3F800800FF014F8019B88F82C
:1040A0000300D3F800800FF017F8DAF80030A8F812
:1040B0000A005B790A2B40F2FB82544BD3F8008054
:1040C0000FF000F888F80800F2E20FF005F86FF43E
:1040D000AF6283189BB2C62B98BFA4F896010EF06E
:1040E000FBFFA4F840010EF0F7FFA4F842010EF028
:1040F000F3FFA4F844010EF0EFFFA4F8D8010EF08E
:10410000E1FF84F8ED010EF0DDFF0EF0DBFF84F837
:10411000EE010EF0D7FF84F885010EF0D3FF84F88E
:1041200092010EF0CFFF384BD3F800800EF0D4FF91
:1041300000EB80004000A8F8560030E10EF0CCFF04
:10414000334B23F8180008F10108B8F1080FF5D136
:10415000AEE253790F2B7FF4BDAD0EF0B3FF07280D
:1041600080463FF6B7AD029BD3F800A00EF0B4FF37
:104170000E2303FB08F8029BC244AAF81901D3F8E6
:1041800000A00EF0A9FFC244029BAAF81B01D3F8BD
:1041900000A00EF0A1FFC244029BAAF81D01D3F8B3
:1041A00000A00EF08FFFC244029B8AF81F01D3F8D3
:1041B00000A00EF087FFC244029B8AF82001D3F8CA
:1041C00000A00EF07FFFC244029B8AF82101D3F8C1
:1041D00000A00EF077FFC244029B8AF82201D3F8B8
:1041E00000A00EF083FFD044C8F8230160E200BFB6
:1041F00000007A44F497010828120020000F0020E4
:10420000040F00200800002018100020401000209B
:10421000363100200EF056FF0F2880463FF65AAD8B
:104220000EF050FFC8EBC80804EB080383F8D00079
:1042300003F1D0080EF046FF88F801000EF042FFAF
:1042400088F802000EF03EFF88F803000EF03AFFF7
:1042500088F804000EF036FF88F805000EF032FFF3
:1042600088F806000EF0C4FB22E22B785B0700F111
:104270001F820DF085FB04F013FF04F0DBFF17E253
:104280002B78580700F11482C54B4FF4C8721A807E
:104290000EE22B78590700F10B82C24A137843F0E3
:1042A000040328E02B785A07E5D552E20EF00AFF06
:1042B000BC4B1A7810B142F0020201E022F0020277
:1042C0001A700EF0FFFEB84BDFF8FC8218700EF08B
:1042D0000DFFC8F800000EF009FFC8F804000EF04A
:1042E000FBFEB24B18800EF0F7FEB14BB14A1880BE
:1042F000137843F002031370DAE10EF0E3FE03904B
:104300000EF0F4FE83460EF0F1FE82460EF0EEFE55
:1043100080460EF0E1FE0EF0DFFE0EF0D3FE039BB2
:10432000A3B9A54B1020C3F800B0C3F804A004F053
:104330005DFE9C4A137843F001031370B8F1000F3F
:1043400000F0B6819D4BC3F80080B1E1102B40F026
:10435000AF819B4BC3F800B0C3F804A0B8F1000FC5
:1043600002D0964BC3F800809548964B0222011D5F
:104370001A7009F0A3FC9BE1A0600EF0B7FE04F0F8
:104380005DFE95E10EF0A8FEA4F858010EF0A4FE23
:10439000A4F85A010EF0A0FEA4F85C0188E10EF02A
:1043A00091FE84F87A010EF08DFE84F87E010EF005
:1043B00089FE84F87D010EF085FE84F87F0177E1A7
:1043C0000EF08AFEA4F880010EF086FEA4F88201A9
:1043D0000EF078FE84F884010EF07EFEA4F88601CB
:1043E00066E10EF06FFE84F890010EF075FEA4F801
:1043F0009A010EF071FEA4F896010EF06DFEA4F87D
:1044000098010EF05FFEDAF8003084F891015B79D4
:10441000082B40F24D810EF05FFEA4F89C010EF0D7
:104420005BFEA4F89E0143E10EF04CFE84F8D60139
:104430000EF048FE84F8D7010EF04EFEA4F8D80125
:1044400036E192F805800323B8FBF3F8B8F1120FB8
:104450003FF640ACDFF874A14FF0000BC34580F08D
:1044600027810EF02FFE8AF8A0010EF035FE40F2F3
:10447000ED23984205DD40F6CA039842A8BF1846CE
:1044800001E040F2EE20A0F2EE20192390FBF3F0C1
:104490000BF1010B8AF8A1010AF1020ADEE70EF026
:1044A00011FE84F8920103E10EF00CFE04EB080308
:1044B00008F10108B8F1080F83F88801F4D1F7E09A
:1044C0000EF000FEC4F808B060710EF00FFE04F0AC
:1044D000B5FD0EF0F7FD84F890010EF0FDFDA4F897
:1044E00058010EF0F9FDA4F85A010EF0F5FDA4F8FC
:1044F0005C010EF0F1FDA4F880010EF0EDFDA4F8D2
:104500008201D5E053794FF0070AB3FBFAF2C2EB10
:10451000C2029A1A12F0FF0F7FF4DCABB3FBFAFA77
:104520000AF1FF3A5FFA8AFABAF1FF0F00F0C08091
:104530000EF0C8FD5FFA80FB4FFA8BF00DF076FEAF
:10454000804600283FF4C6AB80F800B00EF0C4FDF2
:10455000A8F802000EF0B6FD88F804000EF0B2FDD7
:1045600088F805000EF0AEFD88F807000EF0AAFDF1
:1045700088F80600D4E7DFF8548008F1400A0EF00E
:10458000ABFDA8F8AC020EF09DFD88F8AE020EF06F
:1045900099FD08F1040888F8AB02D045EFD187E017
:1045A000EE1F0020E0180020E6180020E41800208C
:1045B000E21800204610002048100020581000206B
:1045C000501000200C0F0020E8180020E8100020F8
:1045D0000EF078FD1F2880463FF67CABD9F80030FE
:1045E0005B79082B7FF476AB0EF076FD08F18A0834
:1045F00004EB880800F03F00A8F806000EF06CFD00
:10460000B8F80630800100F4FE501843A8F8060000
:104610000EF058FD000188F804000EF053FD98F8E4
:10462000043000F00F00184388F804000EF04AFD33
:1046300088F805000CF0ACFD3AE07A4B012283F8D3
:10464000352035E00EF03EFDFF2882461BD10023C9
:104650008DF81F309DF81F30052B29D89DF81F00BD
:10466000714A9DF81F30012102EBC3035B6852F8C9
:104670003000994089B2482203F00CFA9DF81F30AF
:104680000133DBB2E4E705283FF624AB00200EF04F
:104690006BFD0EF045FDD8F800000DF0D8FF18B9FD
:1046A00032200DF002FFF6E74FFA8AF003F000FA2D
:1046B00000200EF059FDFFF78AB95C4B98590DF0B8
:1046C000C6FF18B932200DF0F0FEF6E70EF050F9F3
:1046D00004F0BCFC564A574BDA60FFF785B90C284A
:1046E0003DD00A2844D1544D54480EF0C1FD28460F
:1046F000232113F06AF908B1401B20602368002BC6
:1047000059D14D4800213022236013F028F93B781D
:1047100043BB4B4B1B689B0614D54A4B41491B6856
:104720008A6B9A1A002A0DDB474A1278042A09D9A3
:1047300003F5123303F5F873444A8B63D36883F0AF
:104740001003D360424B9B68002B67D041489847C9
:1047500064E007F02FFDFFF73AB90C2804D13E487A
:104760000EF086FD3D480DE07F2812D1FFF799B885
:104770000D28B8D07F2809D12F4A013B00213848A5
:104780002360D1540EF074FDFFF78BB82F2B3FF64A
:1047900088A8A0F12002D2B25E2A3FF682A813B9FF
:1047A00020283FF47EA85A1C2260234AD0540EF0E1
:1047B00057FDFFF776B85A1EA95C202901D1134690
:1047C0009DE71D4A00212360D154264B264DD3F886
:1047D00000A0D5F800B0DFF86090584613F003F958
:1047E000064659463246484613F006F91F4A28B98C
:1047F00019F8063053445B785B0703D010359542B7
:10480000E7D306E0954204D2701CEB684844984711
:1048100002E017480EF02CFD002372E709B0BDE856
:10482000F08F00BF980F002038BD0108A82000209D
:104830000400FA0500ED00E0D82D002031C9010880
:10484000DC180020AC330020E6180020000C0140EA
:1048500058210020D40F0020DAB90108D5B9010889
:1048600001BA01085C00002064A2010844A4010808
:10487000E5B901082DE9F0474D28A0B0044600F045
:10488000488600F2BD80302800F0A98651D8222841
:1048900000F0938423D8032800F00A8214D801285A
:1048A00000F0FA81022840F01E8704200EF05CFC24
:1048B00043200EF024FC4C200EF021FC46200EF08C
:1048C0001EFC4C2000F04ABE042800F0FA810528A6
:1048D00040F009871A200EF047FC002403E2282844
:1048E00000F0E58515D8242800F0CC85262840F076
:1048F000FA86DD4C06200EF037FCB4F858010EF0B5
:1049000036FCB4F85A010EF032FCB4F85C0100F049
:10491000B6BD2C2800F0DE852E2800F04A862A2815
:1049200040F0E18601200EF01FFCCF4B587900F0DB
:1049300015BE3D2800F0FF821ED8362800F01F86E5
:104940000BD8322800F00486342840F0CC8648206A
:104950000EF00AFC002500F052BC3A2800F0C0829C
:104960003B2800F02384382840F0BD8604200EF058
:10497000FBFBBD4C00F08CBD452800F0A18627D87C
:10498000402800F0EE85422840F0AD86B64C10205D
:104990000EF0EAFB60790EF0B2FBA0680EF0F0FBBF
:1049A00094F890010EF0ABFBB4F858010EF0DFFB69
:1049B000B4F85A010EF0DBFBB4F85C010EF0D7FB43
:1049C000B4F880010EF0D3FBB4F8820100F057BDBB
:1049D000472800F05386C0F027864B2840F0838696
:1049E000A14C04200EF0C0FB94F8D6010EF087FB1A
:1049F00094F8D7010EF083FBB4F8D80100F03FBD66
:104A0000702800F0EF8200F2E180692800F048820F
:104A100000F2B280662800F0A28100F2A280642831
:104A200000F07A81652840F05E86904C0B200EF0F5
:104A30009BFB20880EF09BFB608880B20EF097FBFA
:104A40008B4B1B68C3F3C000C3F38002800040EAB5
:104A50004200C3F340021043C3F3401240EAC200D5
:104A600003F0100318430EF082FB824B1A88636830
:104A700002F0080103F4475949EA010903F48041AF
:104A800049EA010903F4004149EA010903F48031CC
:104A900049EA010903F4003149EA010903F48021DC
:104AA00049EA010903F4002149EA010903F48011EC
:104AB00049EA010903F0007349EA0303DFF8D491DE
:104AC00012F0010F99F8009018BF4FF00208C9F3D7
:104AD000800908BF4FF0000843EA090312F0020FF3
:104AE00043EA080314BF4FF0040C4FF0000C12F01F
:104AF000040F43EA0C0C14BF4FF0100E4FF0000EE1
:104B000012F0400F14BF202700274CEA0E0E12F0BF
:104B1000100F14BF4FF4007600264EEA070712F07C
:104B2000200F14BF4FF4806500253E4312F4807FB0
:104B300014BF4FF400600020354312F4007F14BF0F
:104B40004FF400110021284312F4806F41EA000164
:104B500014BF4FF08063002300201943247A0346DA
:104B6000EAE0672800F02381682840F0BC85102027
:104B70000EF0FAFA00248AE16C2800F0A48117D81C
:104B80006A2800F002846B2840F0AD8505200EF005
:104B9000EBFA394B18880EF0EAFA384B18880EF009
:104BA000E6FA324B93F86E0000F0010000F0D6BC3C
:104BB0006E282E4D00F09A8100F2C88106200EF07A
:104BC000D3FAE86D0EF0DCFA2D4B87E1782800F07F
:104BD000FB8018D8742800F033830AD8722800F0BC
:104BE0009483732840F07F8508200EF0BDFA0124DD
:104BF000C4E3762800F0E98300F25B832F200EF0F7
:104C0000B3FA204CCAE2A42800F0058414D87B280B
:104C100000F06A82A02840F066850C200EF0A4FA0D
:104C2000194B18680EF0ACFA184B18680EF0A8FA79
:104C3000174B186800F053BDF12800F00181FE28E1
:104C400000F01084F02840F04E85084C04200EF04F
:104C50008BFA236CB3F85A000EF089FA236CB3F880
:104C6000580000F00CBC00BFE8100020D80F002056
:104C7000DC180020A41900205A1900205C1900201B
:104C8000D0100020C3970108E8F7FF1FECF7FF1FC3
:104C9000F0F7FF1FC933002003200EF065FA002053
:104CA0000EF02DFA20460EF02AFA0D2000F056BC28
:104CB0000EF05AFA01200EF022FA0A200EF01FFA26
:104CC000A7E306200EF050FA41200EF018FA572004
:104CD0000EF015FA46200EF012FA31200EF00FFAFF
:104CE000AE4B1878CBE3AE4B185D01340EF007FAEB
:104CF0000B2CF8D10024AB4B185D01340EF0FFF9FA
:104D0000082CF8D10024A84B185D01340EF0F7F9F7
:104D1000072CF8D100F0E5BC07200EF025FAE720BB
:104D20000EF0EDF9A14B58790EF0E9F900200EF0E4
:104D3000E6F9042000F0D3BCA3420AD29C4A9D5C51
:104D4000012202FA05F50D421CBF9A4010430133BF
:104D5000F2E70EF015FA954B93F8B407FEE3122034
:104D60000EF002FA934B00241B88B3F5806F8CBFC2
:104D700008250125904B33F91400013490FBF5F020
:104D800080B20EF0F4F9032CF4D18C4CA08C0EF010
:104D9000EEF9E08C0EF0EBF9208D0EF0E8F9608D65
:104DA0000EF0E5F9A08D0EF0E2F9E08D67E310203A
:104DB0000EF0DAF90024824B185D01340EF09FF9F1
:104DC000102CF8D100F08DBC70200EF0CDF900262B
:104DD0000E247443794D01362B6C2344B3F819012A
:104DE0000EF0C5F92B6C2344B3F81B010EF0BFF98C
:104DF0002B6C2344B3F81D010EF0B9F92B6C23443E
:104E000093F81F010EF07BF92B6C234493F82001DB
:104E10000EF075F92B6C234493F821010EF06FF915
:104E20002B6C234493F822010EF069F92B6C1C447F
:104E3000D4F823010EF0A4F9082EC9D100F051BC1A
:104E400070200EF091F9594C04F1700594F8D000DF
:104E50000EF055F994F8D1000EF051F994F8D20003
:104E60000EF04DF994F8D3000EF049F994F8D400FF
:104E70000EF045F994F8D5000EF041F9073494F896
:104E8000CF000EF03CF9AC42E0D100F02ABC4D4B13
:104E9000185D01340EF033F9102CF8D100F021BC6C
:104EA000494D00242878400000F0FE000EF05CF927
:104EB0002B789C4280F01584444B33F814000EF09C
:104EC00056F90134F4E7424C06200EF04DF92088E3
:104ED0000EF04DF960880EF04AF93E4B1888CEE28C
:104EE00004200EF041F9354B186EF8E307200EF060
:104EF0003BF9394B1888FF28A8BFFF20C0B20EF03D
:104F0000FEF8364B186880F3100080B20EF02FF9CF
:104F1000B5F864000EF02BF9244B93F88521304B43
:104F2000186822B10A23584380F3100001E000F30F
:104F30000F0080B2A3E21D4C02200EF015F994F888
:104F4000E0010EF0DCF894F8DF0107E30B200EF02F
:104F50000BF9AB6E002618780EF0D1F8AB6E5878CE
:104F60000EF0CDF8AB6E154C3344187901360EF0C7
:104F7000C6F8032EF6D1A36ED8790EF0C0F8A36E52
:104F800098780EF0BCF8A36ED8780EF0B8F8A36E3F
:104F900058890EF0ECF8A36E187ADFE2CB330020CC
:104FA000FCB6010808B70108DDB60108E8100020CA
:104FB000E10F00201C000020CA100020D80F0020A4
:104FC000081000201C10002044210020B8310020CF
:104FD00074310020D8100020CC180020D8180020F0
:104FE000D4180020C04C1E200EF0BEF8236C002503
:104FF0001B78022B65D1236C05F1080253F82200BF
:10500000BA490FF0E5FA12F0B7FE80F30800C0B21B
:105010000EF075F8236CB64903EB8503D86A0FF0E0
:10502000D7FA12F0A9FE80F30800C0B20EF067F8BC
:10503000236C05F10E0253F82200AE490FF0C8FAB6
:1050400012F09AFE80F30800C0B201350EF057F856
:10505000032DD0D1072D236C21D1586CA3490FF01B
:10506000B7FA12F089FE80F30800C0B20EF047F8DC
:10507000236C9E49986C0FF0ABFA12F07DFE80F322
:105080000800C0B20EF03BF8236C93F84C000FF010
:1050900047FA12F071FE80F30800C0B20BE02B4417
:1050A00058780EF02CF8236C2B44D87A0EF027F8A1
:1050B000236C2B44587D01350EF021F80A2DC9D1FF
:1050C0000FE3236C2B4458780EF019F8236C2B4413
:1050D000D87A0EF014F8236C2B44587D01350EF06D
:1050E0000EF80A2DEDD1FCE23C200EF03DF8002434
:1050F0007D4D04F108022B6C7E4953F822000FF01D
:1051000067FA12F039FE80B20EF031F82B6C794953
:1051100003EB8403D86A0FF05BFA12F02DFE80B225
:105120000EF025F82B6C04F10E0253F822007149A1
:105130000FF04EFA12F020FE013480B20EF017F894
:10514000032CD5D1072C2B6C16D1586C69490FF064
:105150003FFA12F011FE80B20EF009F82B6C65498F
:10516000986C0FF035FA12F007FE80B20DF0FFFFD9
:105170002B6C93F84C000BE0234458780DF0F7FFAC
:105180002B6C2344D87A0DF0F2FF2B6C2344587D0E
:1051900001340DF0ECFF0A2CD4D1A2E214F8010F77
:1051A000002800F09E820DF0AAFFF7E701200DF025
:1051B000DBFF4D4B1B6C1878D0E150200DF0D4FF75
:1051C0000025494B0C211C6C4B4B04EB850494F8D7
:1051D0007920013501FB023393F838000DF08FFF81
:1051E00094F87A000DF08BFF94F87B000DF087FFA8
:1051F00094F87C000DF083FF142DE2D171E23A4B5C
:105200001C6C062303FB054494F8CE000DF077FFD9
:1052100094F8C9000DF073FF94F8CA000DF06FFF09
:1052200094F8CB000DF06BFF94F8CC000DF067FF05
:10523000013594F8CD000DF062FF0C2DDFD150E266
:105240004FF0000801260027274B1A7A974227DAE9
:105250000933FA5C00240C236343274D05F1300128
:10526000595C914207D12B44586B12F0BCFB82462B
:105270002EB9B14605E001341C2CECD10EE080447F
:105280000CE0D1450ADA0C2303FB04535B6B13F8E3
:1052900009000DF034FF09F10109F2E70137D3E706
:1052A000002E00F01E825FFA88F00DF05DFF0026F0
:1052B000C9E70D4D0024287A0DF056FF2B7A9C4249
:1052C00080F00F820D4B0021E65C0C2202FB01F303
:1052D000094800F13007DA5DB24211D1034493F876
:1052E00038000DF00CFF0EE0D80F00200000204128
:1052F0000000C84200007A44C4970108E10F002072
:1053000001311C29E1D10134D8E7D04C16200DF031
:105310002BFFB4F896010DF02AFFB4F840010DF010
:1053200026FFB4F842010DF022FFB4F844010DF05D
:105330001EFFB4F8D8010DF01AFF94F8ED010DF03E
:10534000DEFE00200DF0DBFE94F8EE010DF0D7FE3E
:1053500094F885010DF0D3FE94F892010DF0CFFE84
:1053600000200DF0CCFEBA4B0A201B6CB3F956306E
:1053700093FBF0F080B20DF0FAFE89E0E0B2013468
:105380000DF0BDFE092CF9D1ABE110200DF0ECFEC3
:10539000B04BB14C187800F002000DF0B0FEAF4BEE
:1053A00018780DF0ACFE20680DF0EAFE60680DF094
:1053B000E7FEAB4B18880DF0DAFEAA4B18880DF00B
:1053C000D6FEA34BB3F86C0059E00DF07BFE074608
:1053D00012200DF0C9FE9E4C17B9266F656F05E0CF
:1053E000102F19BF00252E46A66FE56F38460DF029
:1053F00086FE30460DF0C4FE28460DF0C1FED4F8FE
:1054000080000DF0BDFE00200DF0B1FE00200DF07B
:10541000AEFE0020A2E08E4D002495F884002E46BA
:1054200080000130C0B20DF09FFE95F884000DF0B1
:1054300066FE96F884309C4280F053818A4D285D48
:105440000DF05DFE05F11003185D0DF058FE05F13D
:105450002003185D30350DF052FE285D0DF04FFE33
:105460000134E6E708200DF07FFE00200DF07FFEFE
:1054700000200DF07CFE00200DF079FE00200DF0E4
:1054800076FE2EE104200DF06FFE704B986826E149
:1054900094F87A010DF033FE94F87E010DF02FFEA2
:1054A00094F87D010DF02BFE94F87F0156E0674CD7
:1054B00007200DF059FEB4F880010DF058FEB4F845
:1054C00082010DF054FE94F884010DF018FEB4F83A
:1054D0008601D4E75D4C0C200DF046FE94F8900157
:1054E0000DF00DFEB4F89A010DF041FEB4F89601EE
:1054F0000DF03DFEB4F898010DF039FE94F89101DD
:105500000DF0FDFDB4F89C010DF031FEB4F89E01E4
:10551000B5E7564C564D2078002600EB4000C0B24F
:105520000DF022FE237802359E4280F0DA8015F8D5
:10553000020C0DF0E4FD15F8010C013600EB8000C3
:1055400000EB800000F2EE2080B20DF010FEE9E7E3
:1055500001200DF009FE3D4B93F892010DF0CFFDB7
:10556000BFE008200DF000FE0024384B234493F8E0
:10557000880101340DF0C3FD082CF6D1B1E0344BA5
:10558000324C93F8C50004F12805C0EBC000C0B24E
:105590000DF0EAFD94F8F4010023364AD25C904203
:1055A00000F0A3800C333C2BF7D10834AC42F1D18E
:1055B00097E040200DF0D8FD244C04F14005B4F8EC
:1055C000AC020DF0D4FD94F8AE020DF098FD043459
:1055D00094F8AB020DF093FDAC42F0D181E0E020F5
:1055E0000DF0C2FD194C04F18005B4F82E0204340C
:1055F00000F03F000DF0BBFDB4F82A02C0F38610A6
:105600000DF0B5FD94F8280200090DF078FD94F82E
:10561000280200F00F000DF072FD94F829020DF041
:105620006EFDAC42E1D15CE0134C0D200DF09CFD11
:1056300009F032FE0DF063FD20880DF0A1FDE06859
:105640000DF09EFD08F078FC49E000BFE810002056
:10565000D80F0020E0180020E8180020E6180020ED
:10566000E4180020E21800205D10002044210020F2
:1056700088120020142200200C0000200DF036FDBE
:10568000054684200DF070FD28460DF079FD244B71
:10569000DC6805F18003A3428CBF641B802408F002
:1056A00005FD28462246694609F02AFE05460024E3
:1056B000AC4216DA1DF804000DF021FD0134F7E7C5
:1056C00013200DF051FD0024164B185D01340DF030
:1056D00016FD0B2CF8D100200DF052FD00200DF02E
:1056E0004FFD012018E0002016E00DF008FDB4F891
:1056F000F6010DF03CFD94F8F8010DF000FD94F872
:10570000F9010DF0FCFC94F8FB010DF0F8FC94F8A5
:10571000FA010DF0F4FC48E720B0BDE8F08700BFC7
:105720000C000020FCB601086B4B6C4A2DE9F04FD1
:105730005E8914684FEA062AB4EB0A0A9C884FF087
:1057400000054FEA04481C894FF0000BA4FB0A67D0
:1057500065EB0B0B04FB0B77F40944EA476418EB89
:1057600004065C884FF000094FEAE7154FEAC43899
:10577000DC8849EB050787B0CDE90467A4FB0A671D
:1057800004FB0B77340A44EA076418EB04064FEA7B
:1057900027259C894FF0000949EB0507CDE90067F3
:1057A000AAFB046704FB0B77F40D44EA472414F5C5
:1057B000FA664FEAE75545F10007B6F5FA6F77F15B
:1057C0000003CDE90267964666DADDE90489A4FBA9
:1057D000046704FB05F34FF0050C07EB4307A6FB3A
:1057E0000C230CFB07335F104FEA3206B8EB0608B8
:1057F0004FEA920646EA837669EB07099F10DDE9D6
:105800000023921B63EB0703CDE90023DDE9026768
:10581000334A4FF0FF33964277EB0303CDE9048917
:1058200027DA40F6AC520023A4185D4104FB05F3CF
:10583000A4FB04456FF0060205EB4305664202FB3C
:105840000566A4FB0223334418EB020649EB030769
:10585000CDE904670B26A4FB062306FB0533DDE92F
:1058600000455B104FEA3202A41A65EB0305CDE94F
:105870000045DDE902450AFB0BF3AAFB0AAB0BEB83
:10588000430B4FEADA7242EA4B02A41A4FEAEB7377
:1058900065EB0305CDE90245DEF80440009B019D60
:1058A000A4FB032304FB05334FEA525848EAC328FC
:1058B0004FEA6359DDE90423B8EB020269EB030305
:1058C0009946D30B43EA494300B1036009B1029BF7
:1058D0000B6007B0BDE8F08F78210020A0100020F9
:1058E00024FAFFFF2DE9F04FDFF8589285B0074604
:1058F000D9F808000E460EF017FE8E4C8046208820
:105900000EF00EFE4FF05C51054640460EF060FE74
:105910004FF06451824628460EF05AFE014650462A
:105920000EF04CFD4FF06251824640460EF050FEA4
:105930004FF06A51804628460EF04AFE0146404626
:105940000EF03CFD0546B4F902000EF0EDFD0146F7
:1059500028460EF03DFE5146054650460EF038FEF4
:105960008046B4F904000EF0DFFD014640460EF01B
:105970002FFE014628460EF023FD80460EF0EEFF76
:105980006D490546A06140460EF0D6FED9F80C30B0
:105990008046284601930EF0C7FD4FF07C510EF073
:1059A00017FE66490EF00AFD0546E389B4F90A00C0
:1059B00002930EF0B9FD29460EF00AFE29460EF0BC
:1059C00007FE4FF058510EF003FE8146B4F908006F
:1059D000B4F810B0B4F80CA00EF0A6FD29460EF0F5
:1059E000F7FD014648460EF0EBFC4FF058510EF023
:1059F000EFFD4FF060510EF0EBFD4FF07E510EF0D9
:105A0000DFFC8146E0880EF08BFD014648460EF033
:105A1000DFFD002181460EF06FFF00287BD1294673
:105A200028460EF0D5FD03900FFA8BF00EF07CFDAA
:105A3000039B014618460EF0CBFD4FF060510EF06F
:105A4000C7FD8346BDF908000EF06EFD01462846ED
:105A50000EF0BEFD01460EF0B3FC014658460EF0B6
:105A6000AFFC4FF07A510EF0B3FD834601980EF073
:105A70005BFD01464FF093400EF0A0FC05460FFA87
:105A80008AF00EF051FD4FF08F410EF0A1FD01465E
:105A900058460EF095FC4FF066510EF099FD014608
:105AA00028460EF08BFC26490EF092FD49460EF07A
:105AB00043FE0546B4F916000EF036FD29460EF0F9
:105AC00087FD29460EF084FD4FF040510EF080FD19
:105AD0008146B4F914000EF027FD014628460EF069
:105AE00077FD4FF060510EF073FD014648460EF011
:105AF00067FC8146B4F912000EF016FD01464846D7
:105B00000EF05EFC4FF076510EF062FD0146284625
:105B10000EF056FC00E0002017B10EF01FFF3860B9
:105B20002EB140460EF01AFF64235843306005B092
:105B3000BDE8F08FD82100200000A04500007A4782
:105B40000050C345A0100020704770472DE9F04178
:105B5000324C334D62892B8AB4F904809A1A238916
:105B6000B4F902E05A43B4F91230D613B4F9142050
:105B7000DB02324493FBF2F232440A26E2615643DE
:105B8000A2F57A6202FB02F3B4F90EC002FB0EFE2C
:105B900002FB08F2B4F90C801B130CFB03FC03FBA3
:105BA00008F31B1403EB62320232E388921002F511
:105BB000004253434CF25032B4F920704FEAEE2EBB
:105BC000B4F900400EEBEC2C0CEB8404BC406D6986
:105BD0000234A5EBA4043A4162434FEAD3384EBFE6
:105BE000B2FBF8F35400B4FBF8F340F6DE3448BFE0
:105BF0005B001A12524362430A4C08365C43241479
:105C000004EB224202F6CF62361103EB221300B1FD
:105C1000036001B10E60BDE8F08100BF8C2100205F
:105C2000A010002043E3FFFF024B4FF480521A8084
:105C3000704700BF1C000020054B1A7E02F0FF01D8
:105C400022B10122027000221A767047017070475B
:105C5000A01000207720482101220DF0CFB8772036
:105C6000582101220DF0CAB87620F42131220DF01E
:105C7000C5B8074B002193F82020064B920134321F
:105C800059767720F42102F0FC020DF0B7B800BF7E
:105C90008C210020A0100020034B00225A76772090
:105CA000F4212E220DF0AAB8A010002008B50F2173
:105CB000082218200DF0A2F80E22182010210DF055
:105CC0009DF8024B4FF480521A8008BD1C00002042
:105CD00008B5134B53201B782D2108227BB10DF002
:105CE0008DF831210A2253200DF088F82C210C2246
:105CF00053200DF083F853203821902209E00DF055
:105D00007DF831210A2253200DF078F853202C2100
:105D10000A220DF073F840F20912024B1A8008BDF6
:105D2000742100201C00002007B5002101AB0322D4
:105D300077200DF023F89DF805309DF804001B0234
:105D400043EA00439DF80600184303B05DF804FBE6
:105D500008B5FFF7E9FF014B586008BDA01000200F
:105D600008B5FFF7E1FF014B186008BDA010002047
:105D700007B5F7216B46062276200CF0FFFF9DF851
:105D800000309DF801101B0343EA01139DF8021037
:105D9000094A43EA1113D3609DF803309DF80410BB
:105DA0001B0343EA01139DF8051043EA11139360A6
:105DB00003B05DF804FB00BFA01000200F4B13B52B
:105DC0001B780F4C0BB1637EB3B1032201AB77207C
:105DD000F6210CF0D3FF9DF805309DF804201B023E
:105DE00043EA02439DF806201343064AB2F92020F5
:105DF000C2F10802D340636102B010BD2B00002045
:105E0000A01000208C2100200A4B13B51B780A4CEF
:105E10000BB1637E63B1022201AB7720F6210CF057
:105E2000ADFF9DF804209DF8053043EA022323824C
:105E300002B010BD2B000020A010002013B50622D8
:105E40000446432168206B460CF098FFA8B19DF8EA
:105E500000209DF80130012043EA022323809DF8B1
:105E600002209DF8033043EA022363809DF804205A
:105E70009DF8053043EA0223A38002B010BD13B59C
:105E8000062204463B2168206B460CF077FFA8B140
:105E90009DF800209DF80130012043EA0223238071
:105EA0009DF802209DF8033043EA022363809DF8A9
:105EB00004209DF8053043EA0223A38002B010BD00
:105EC00013B501220DF1070304461A2168200CF0D6
:105ED00055FF9DF8073003B10123237002B010BDB8
:105EE00013B5022204461B21682001AB0CF046FFCB
:105EF00070B19DF804209DF8053043EA022303F5B4
:105F00004E5310334FF48C7293FBF2F32333238000
:105F100002B010BD13B5062204461D2168206B4651
:105F20000CF02CFFA0B19DF800209DF8013043EA51
:105F3000022323809DF802209DF8033043EA0223C8
:105F400063809DF804209DF8053043EA0223A38076
:105F500002B010BD13B50622044601211C206B4679
:105F60000CF00CFF08B39DF801309DF800200421CF
:105F700043EA022242F38D0292FBF1F29DF80230D5
:105F800022809DF8032042EA032242F38D0292FB15
:105F9000F1F29DF8043062809DF8052042EA032367
:105FA00043F38D0393FBF1F3A38002B010BD13B54F
:105FB00006220446022118206B460CF0DFFEB8B121
:105FC0009DF800309DF801209B0803EB02232380FD
:105FD0009DF802309DF803209B0803EB02236380A9
:105FE0009DF804309DF805209B0803EB0223A38055
:105FF00002B010BD314B2DE9F3411B780546002B53
:106000003BD0002426462746A046013453203221A7
:1060100008226B46E4B20CF0B1FE08B9002049E05A
:106020009DF801209DF80030202C03EB02231BB2C9
:106030009DF8032098449DF8023003EB02231BB225
:106040001F449DF805209DF8043003EB02231BB28A
:106050001E449DF8073003F07F0301D0002BD4D1FC
:1060600098FBF4F897FBF4F796FBF4F6144BA5F8BD
:1060700000806F80AE809C761CE053203221062287
:106080006B460CF07BFE0028C8D09DF801209DF8DF
:10609000003003EB02232B809DF803209DF8023093
:1060A00003EB02236B809DF805209DF8043003EB81
:1060B0000223AB8002B0BDE8F08100BF7421002054
:1060C000A010002008B54FF4804006F0D7FC01284E
:1060D00001BF044B4FF480425A61034B08BF58760E
:1060E00008BD00BF00040140A010002010B5074CFF
:1060F0002368186906F0C2FC30B123681A69044BA2
:106100005A61044B01221A7610BD00BF7021002095
:1061100000040140A010002013B500222A211C20F9
:106120000CF06CFE0E2102221C200CF067FE0F21E9
:1061300003221C200CF062FE2B2112221C200CF0EA
:106140005DFE164A02249369154843F004039361E7
:106150002023ADF8043004230DEB03018DF8063045
:106160008DF8074008F05FFF22462C211C200CF020
:1061700045FE2D2101221C200CF040FE2E21002284
:106180001C200CF03BFE2A2105221C200CF036FEC0
:10619000044B4FF480721A8002B010BD0010024010
:1061A000000801401C000020F8B50F461646074CB9
:1061B0004FF48055656140F080000DF083FA384659
:1061C000002132460DF048FA2561F8BD000C01406F
:1061D00013B5012204460DF107013A20FFF7E4FF51
:1061E0009DF8073003B10123237002B010BD13B531
:1061F0000446694643200622FFF7D6FF9DF800209B
:106200009DF80130012043EA022323809DF80220FB
:106210009DF8033043EA022363809DF804209DF833
:10622000053043EA0223A38002B010BD13B5044633
:1062300069463B200622FFF7B7FF9DF800209DF836
:106240000130012043EA022323809DF802209DF8BB
:10625000033043EA022363809DF804209DF8053053
:1062600043EA0223A38002B010BD70B50E46054C70
:106270004FF4805565610DF025FA30460DF022FA95
:10628000256170BD000C01401F4B07B51A681F4BFC
:106290009A420ED14FF40053ADF8043002238DF82A
:1062A000073004231A480DEB03018DF8063008F07F
:1062B000BAFE80216B20FFF7D8FF64200CF0F5F8C0
:1062C00000216B20FFF7D1FF64200CF0EEF86B206B
:1062D0000121FFF7CAFF1B201821FFF7C6FF1C2072
:1062E0001021FFF7C2FF0B4B1A201978FFF7BDFFF3
:1062F000094B19201978FFF7B8FF38200121FFF763
:10630000B4FF03B05DF804FB2C000020001BB700B5
:10631000001001402A000020F4210020F0B5254D96
:1063200085B0EB7E002B43D1234C2368002B3FD05C
:106330001A68224E12B1B1690A43B2619A8898680C
:10634000ADF8002002228DF80320694604228DF862
:10635000022008F068FEB369002743F00103B3612F
:1063600023680126197D187B08F048FE14480CF0BC
:1063700059F92368134A1B695361029308230DEBF3
:1063800003008DF80D308DF80C708DF80E6006F05E
:1063900045FB236801A85B7D8DF806708DF80430FD
:1063A00003238DF805308DF807600DF037F9EE7690
:1063B00005B0F0BDA01000207021002000100240A8
:1063C000ED6000080004014008B5FFF7A7FF6B214E
:1063D000802268200CF012FD64200CF066F86B211E
:1063E000032268200CF00AFD124B19211A7868204C
:1063F0000CF004FD0F200CF058F80F4B1A211A78FE
:1064000068200CF0FBFC1B21182268200CF0F6FC25
:106410001C21102268200CF0F1FC3721002268209A
:106420000CF0ECFCBDE808406820382101220CF09B
:10643000E5BC00BFF42100202800002008B5FFF7CC
:106440006DFF074B1B7813B1012B03D008BD4FF430
:10645000006201E04FF48052024B1A8008BD00BF79
:10646000752100201C00002008B519200CF01DF833
:106470006820152100220CF0C1FC10B902200CF09C
:1064800087F80C4B16211A78682042F018020CF09D
:10649000B5FC1721002268200CF0B0FC3D21012240
:1064A00068200CF0ABFCBDE8084068203E210122CA
:1064B0000CF0A4BC290000200CF0ECBA0CF012BCCB
:1064C0000CF0E8BA0CF00EBC73B51D4C237F53BB27
:1064D0001C4A1D4D93694FF4805643F008039361A5
:1064E00010238DF806302846032301A98DF80730C4
:1064F000ADF8046008F097FD144A2E61138823F06C
:1065000040031B041B0C1380138823F038031B0467
:106510001B0C43F00803138013889BB243F0400325
:10652000138001232377752001A90122FFF73CFE88
:106530009DF80400A0F170035842584102B070BDAC
:10654000A010002000100240000C01400038004064
:1065500007B523200BF0A9FF6820752101220DF15A
:1065600007030CF00BFC28B19DF80700A0F16803AD
:106570005842584103B05DF804FB00BF2DE9FF47C6
:10658000CB4C07462378CB4E002B00F0E7813268D6
:106590006368D31A7C2B40F2E181237A6260013375
:1065A00023724FF0000808F12400C14DC0B207F07B
:1065B000A5FE05F10A0333F918000DF0B5FFBE4B37
:1065C000814618880DF0B0FF014648460EF0B4F839
:1065D000BA490DF0FDFF0EF0C1F908F1010800B253
:1065E00007F07AFEB8F1030FDDD1302007F086FE08
:1065F000B5F9100007F070FE07F078FE2B7A9A07C5
:106600002CD141F288336A689A4218D9102007F0D9
:1066100075FE68694FF0640890FBF8F000B207F06F
:106620005BFE212007F06AFE686990FBF8F308FB27
:1066300013000028B8BF404200B207F04DFE1420FE
:1066400007F05CFEB4F9180007F046FE1C2007F0C6
:1066500055FE002007F040FE07F048FE237ADFF8E1
:1066600050825B0740F05781022007F047FED8F8C0
:106670001C006423323090FBF3F000B207F02CFED4
:10668000B8F926504FF0050A95FBFAF5032007F0FC
:1066900035FE8B4BADB21B78DFF8389213F0040F48
:1066A0000DD008F5D87039460BF095FE28B9D9F809
:1066B000003013F0100F18BF002528B205E0D8F8FD
:1066C00008389889B0FBFAF000B207F005FED9F857
:1066D00000309F076ED5DFF80092B4F80C2899F8C7
:1066E00000304FF0640808FB02325B00B2FBF3F3AA
:1066F000B4F80E7806203F01BFB247EA0327BFB2C5
:10670000C3F303231F4307F0F9FD38B207F0E4FD9C
:10671000B4F80E3899F8001001339BB293FBF1F2F4
:1067200001FB1233A4F80E38D4F81038604D9B7B6F
:10673000012B05D1392007F0E1FDB5F90C081AE06D
:10674000B5F80C586E235D43152795FBF7F53A20F5
:10675000AFB207F0D3FDB7FBF8F528B208FB15750B
:1067600007F0BAFD3B2007F0C9FDA8B2451D0A207D
:1067700095FBF0F000B207F0AFFD282007F0BEFD5A
:10678000D4F814380A2093FBF0F000B207F0A4FD0F
:10679000042007F0B3FDD4F808389B8913B106F044
:1067A000ADFA04E0424BD3F8180880F3100000B2B1
:1067B00007F092FDD4F81C383D4F9D0640F1A080B3
:1067C00097F8203898071DD5112007F097FDB7F8E6
:1067D00022084FF4F36568433A4B90FBF3F000B2A4
:1067E00007F07AFD192007F089FDB7F82208454324
:1067F000642095FBF0F595FBF0F300FB135000B21D
:1068000007F06AFD94F82038B4F8245813F0020F0A
:1068100008BF0025012007F071FD28B207F05CFDDC
:10682000092007F06BFD002007F056FD264B94F879
:1068300026581A88B2F5967F0AD91D4B1B7A03F0A9
:106840000F03072B04D842F20F75954228BF154657
:10685000052007F053FDD4F810385B7B0BB928B244
:1068600016E0A5F120000DF05FFE18490DF064FF61
:10687000002105460EF04AF810B94FF07C5101E0B6
:106880004FF03F4128460DF09BFD0EF067F800B237
:1068900007F022FD94F82028054B910703D493F8C4
:1068A0002728012A1AD1012384F8273808482EE026
:1068B000C0100020A03100201C00002000007A44FD
:1068C000C9330020A08601004A0000206666E63F2A
:1068D000E81800207C31002048000020D3F8105830
:1068E000C04968680DF074FE0EF038F8BD4902909A
:1068F000A8680DF06DFE0EF031F8039002A806E0D6
:10690000B94A02AB92E8030083E80300184607F097
:1069100005FD07F0EBFC237A282B1FD1B34B002297
:106920001A7233684FF47A70B3FBF0F83C271720E3
:1069300007F0E4FCB8FBF7F5B5FBF7F007FB1050E8
:10694000000200B207F0C8FC182007F0D7FC07FBD4
:10695000158000B207F0C0FC07F0C8FC94F830388E
:10696000A24D002B00F061810BF078FDD5F8343892
:106970009F4AC31A9342074640F2C780002385F816
:106980003A3885F83C38B5F80C38DAB21B0A85F885
:10699000562885F8573885F84C2885F84D38D5F8AD
:1069A000642833689A1AD5F86838D97B4FF47A731B
:1069B0004B439A420ED38F4B1B68C5F8643895F849
:1069C0006C38013B012B9FBF102385F83A38022316
:1069D00085F83C38D4F814280A20D4F8183892FBEB
:1069E000F0F293FBF0F384F85428121284F855283F
:1069F00084F8583894F820281B1284F8593894F8F1
:106A000026389207794984F8873803D42D2381F8F2
:106A1000883878E0D4F828987748DFF8E8C199FBFF
:106A2000F0FA0CFB0A924FF0060E042B0EFB02F25A
:106A30008CBF3323322381F88838704BD4F82C680C
:106A400092FBF3F196FBF0F003FB1122642592FB1D
:106A5000F5F20CFB006C0EFB0CFE84F87928121288
:106A600084F87A289EFBF3F203FB12E393FBF5F321
:106A70000AEB8A0A4FFA81F80AEB8A0A08EB8A01C4
:106A800089B284F8771800EB8000090A84F8781836
:106A900000EB800051B201EB800292B284F87C28B6
:106AA000120A84F87D2884F87E38B4F822281B1254
:106AB00084F87F382423534393FBF5F5B4F89A38D0
:106AC0000A2284F880381B0A84F88138B4F8243804
:106AD0004FEAD979B3FBF2F303F5FA739BB284F86A
:106AE00082381B0A84F88338B4F89C38F60F84F88F
:106AF0007458C5F3072584F8769884F87B6884F881
:106B0000755884F88938C4F8347894F89E88374DDD
:106B1000B8F1000F0DD1D5F8A4080BF0A1FD0128A4
:106B200007D90228364E00F05C8207F0C7FB01232C
:106B3000B370D4F8A8282D4D002A76D095F89E6819
:106B40003EB140F6B731D5F8B038FB1A8B4219D8B0
:106B50006BE00123D5F8A40885F89E3801F07CF895
:106B6000D5F8B438082193F9000002238DE84800D5
:106B700032464FF4964301F083F885F8B868C5F8BB
:106B8000A40850E095F8AC68CEB9D5F8A408C5F8CB
:106B9000A86885F89E6801F05FF8D5F8B438082138
:106BA00093F9000001238DE8480032464FF49643E4
:106BB00001F066F8C5F8A40807F080FB33E0013E59
:106BC000F6B285F8AC6895F8B81895F8B938DEB91A
:106BD0004A1C013385F8B82885F8B938D5F8A408D7
:106BE0001FE000BF8096184B50990108C01000208C
:106BF0003F0D0300A03100208096980040420F0016
:106C00001C000020806967FF12F8016B01337018C7
:106C1000314685F8B808D5F8A408C5F8A82885F83D
:106C2000B9380BF020FDC4F8B07894F8BA38A04D0C
:106C3000DBB1D5F8BC38C3B1D5F8C038ABB1C5F8B5
:106C4000C4381B689B4AC5F8C838D5F8CC381344FB
:106C5000187AFDF70FFE0CF063FAD5F8CC38013343
:106C6000092B88BF0023C5F8CC38934D94F8D02861
:106C70002E688F4B002A00F0EF81D3F8D428002A29
:106C800000F0EA8193F8D838013B012B00F2E4814F
:106C9000D4F8D408864F0BF0E3FCE0B1D7F8D40861
:106CA0000BF0DBFC97F8D93880467E2BD5F80090A6
:106CB0000ED102231B2887F8D83809D1D7F8D40879
:106CC0000BF0CEFC20B90123C7F8DC9887F8E03838
:106CD00084F8D988DCE7D7F8DC282B689B1A41F6C2
:106CE000583293421ED9032387F8D838B4E1734A47
:106CF00032F8130010B903464FF403600133B0F5C6
:106D0000C06FDBB279D01ED9B0F5006F7FD032D919
:106D1000B0F5036F3FD184F8E138D4F81C38644FE4
:106D200099063FD494F8E01894F8E138002900F06F
:106D300055812A68921B012AD9D984F8E1380023A9
:106D400084F8E03888E1B0F5007F43D007D8B0F58B
:106D5000807F49D0B0F5887F00F08B80E6E7B0F502
:106D6000806F00F0AF80B0F5826F00F0F480B0F576
:106D7000047FDBD123E0B0F5E26F00F08B80B0F54B
:106D8000E46F00F08C80B0F5E06FCFD184F8E1388B
:106D9000B4F90A1087E0B0F5046F74D0B0F5026F53
:106DA000C4D104E197F820389A07BBD5B7F8221868
:106DB00024234B436421123393FBF1F108E184F85F
:106DC000E1383F4B3A4F1B689B07ABD5B7F80C38FF
:106DD0000A21FCE084F8E138394B354F1B6819056E
:106DE000A0D5D7F81418F3E084F8E138D4F81C38AB
:106DF0002F4F5A0796D57969EAE084F8E138304B8D
:106E00002B4F1B681B058DD5D7F81818E0E0D4F878
:106E10001C18274A8F0684F8E13883D592F8201889
:106E200088077FF57FAFD90711D5D2F82C38192202
:106E300083EAE371A1EBE37101EB5101B1FBF2F1E4
:106E4000002BACBF41F0004141F040410EE0D2F8D0
:106E50002838192283EAE371A1EBE37101EB5101B8
:106E6000B1FBF2F1002BB8BF41F080414FF400605C
:106E70008CE084F8E138D4F81C380D4F5B077FF5BF
:106E800051AF3969A4E084F8E138B4F918306421CD
:106E900059437BE084F8E138B4F90C1003E0B4F90D
:106EA0000E1084F8E1382C2391FBF3F16EE000BF63
:106EB000C010002050990108A031002022BB010819
:106EC0007C31002084F8E13894F8E238644A0133D8
:106ED000DBB2032B88BF012382F8E23842F2107341
:106EE00094F8E21859435F4B1B78D80748BF01312B
:106EF0009A0748BF02315F07B4F8E43848BF04314D
:106F0000D80748BF0A319A0748BF14311F0648BF47
:106F10002831D80548BF28315A0748BF64311F07B8
:106F200048BFC831980548BF01F5C8719A0648BFE7
:106F300001F57A71DF0648BF01F5FA61580648BFCE
:106F400001F57A614FF4806001F02CFC444B002283
:106F500083F8E028E6E6D4F81C18DFF8048111F085
:106F6000200784F8E13817D098F8202812F0020F93
:106F700014BF4FF47A71002112F0010F14BF4FF4C7
:106F8000FA6300230B4494F82618194401F00AFC14
:106F9000002384F8E038C5E6334B1B6819067FF5FB
:106FA000C1AE394601F0FEFB88F8E078BAE684F815
:106FB000E138D4F81C382A4F9A067FF5B3AE97F81B
:106FC00020389B077FF5AEAEB7F8243864215943CB
:106FD00001F0E8FB002387F8E038A3E684F8E13805
:106FE0003AE0B37823B1C5F8A07886F80280A0E52E
:106FF000D5F8A038FB1AB3F57A6FFFF49AAD0123E8
:10700000D5F8A408B3700BF028FB0646D5F8A40801
:107010000BF023FB76067FF48CAD8A2802D08E28F5
:107020000DD086E5D5F81C3898067FF582AD95F829
:107030009E38002B7FF47DAD05F66D0306E095F8D4
:107040009E38002B7FF475AD05F63803C5F8A838D7
:107050002D2385F8AC386CE504B0BDE8F08700BF9F
:10706000C0100020C93300207C310020F8B5044650
:107070000E46174600252046202110F0A6FC0446A7
:10708000D0B10134204610F003FDB0F5617F05DB7F
:1070900040F634039842A8BF184601E04FF46170EF
:1070A000A0F56170192390FBF3F00DB9307000E08A
:1070B00070703B7801333B700DB90125DBE720464A
:1070C000F8BD30B505460C46134629462246BDE8B4
:1070D0003040014801F05EBE14BC01087FB5047861
:1070E0000646E4B9354B1921186800EB840090F886
:1070F0007B5090F879204D4305F5617590F87A3012
:10710000009590F87C00414301F5617101912C4894
:107110002146013401F03EFE142CE3D14BE010F087
:10712000B7FC1328054641DC244B701C1C68202149
:1071300000238DF80F3010F048FC1E35064670B164
:107140000136304610F0A4FC1A289FBF04EB8503DB
:1071500058709DF80F30013398BF8DF80F303046CE
:10716000202110F032FC064670B10136304610F096
:107170008FFC0D289FBF04EB850398709DF80F309E
:10718000013398BF8DF80F3004EB85043046E11CC5
:107190000DF10F02FFF76AFF9DF80F30042B0AD0A4
:1071A000601C0021042210F0DAFB04E005480021F5
:1071B0001322FFF786FF04B070BD00BF1810002037
:1071C00033BC010848BC010801480CF051B800BFAD
:1071D0004EBC01082DE9F04304788FB00546002C21
:1071E00059D17B4B0021142209A807AED3F80080A7
:1071F00010F0B5FB07223046002110F0B0FB002351
:107200001A46A70005A8059308EB07058380714976
:10721000B5F802E031F813C01CEA0E0F0AD00E31A7
:107220000DF1380C595C02F1010E624402F81C1C8D
:107230005FFA8EF20133072BE9D100210B46664A33
:10724000B5F802E011F802C01CEA0E0F0AD00632AF
:107250000DF1380C8A5C03F1010E634403F8242C11
:107260005FFA8EF301310629E9D118F807308DE86D
:1072700041006A785949029209A81A0903F00F03DC
:1072800001F073FD2146564809AA013401F082FD40
:10729000202CA6D198E010F0FBFB1F28044600F339
:1072A000868028462021E4B210F08FFB1F2C02D9E3
:1072B000FFF78AFF88E0464B451C1B68002103EB63
:1072C00084042046042210F04AFB0027454B09AEF7
:1072D000304600210A2217F803905FFA87F810F071
:1072E0003EFB002315F8012B32B10A2B04D04A458E
:1072F00002D0F2540133F5E74A455ED108F1FF337D
:10730000032B09D8DFE803F01005023F0DF123013C
:1073100034E00DF123011EE0304610F0B9FB237874
:10732000C0B243EA001006E0304610F0B1FB23780B
:1073300000F00F001843207031E00133062B0AD013
:10734000244800F11B069E5D9642F6D103445A7D07
:1073500063881343638011F8012F02B30023EFE722
:107360000133072B0AD01B4800F10E069E5D9642A2
:10737000F6D130F8132063881343638011F8012F8E
:107380006AB10023EFE7304610F082FB0F2804DCDF
:10739000304610F07DFB607001E000236370013720
:1073A000052F93D1012409F0F3FE6CB980E70E4854
:1073B00000211F22FFF785FE06E02046002104225F
:1073C00010F0CDFA0024EEE70FB0BDE8F08300BF67
:1073D000A819002064990108799901085CBC01088A
:1073E0006BBC01088599010848BC0108F8B5047810
:1073F000064674B9304D2146B5F8C421B5F8C631FA
:107400002E48013401F0C6FC042C05F10405F2D12C
:10741000F8BD2B4910F0ACFAA8B9274B4FF47A719C
:107420004FF4FA62A3F8C411A3F8C621A3F8C81157
:10743000A3F8CA21A3F8CC11A3F8CE21A3F8D01148
:10744000A3F8D221F8BD304610F022FB03280546F0
:107450002BD83046202110F0B8FA044630B1013460
:10746000204610F015FB0126074600E006462046A0
:10747000202110F0AAFA10B9BDE8F840A4E60130C6
:1074800010F006FB012EF7D140F2DC53A7F2EE22FA
:107490009A42F1D8A0F2EE229A42EDD8064B70350E
:1074A00003EB85039F80D880F8BD064800210322A6
:1074B000BDE8F84005E600BFE810002077BC0108F1
:1074C0008ABC010851CA01082DE9FF41047805462C
:1074D000002C34D16D480BF0CBFE6D4D2869002196
:1074E0000DF00AFA002840F0CE802146694801F0EC
:1074F00051FC2869694601F0D3FA0146664801F05B
:1075000049FC6869694601F0CBFA0146624801F01E
:1075100041FCA869694601F0C3FA01465E4801F0E2
:1075200039FCE869694601F0BBFA013401465B4861
:1075300001F030FC0C2C05F11005CFD1A3E0584927
:10754000052210F059FA38B9514B0022034410308B
:10755000C0281A61F8D196E028465249042210F05A
:107560004BFA04462846002C3FD1202110F02DFA7A
:10757000002800F08880451C284610F034FA0746A1
:10758000494B53F824601EB948480BF071FE7AE06D
:1075900028463146FAB210F02FFA01340028EFD114
:1075A0003B4B0021C2181030C02811619E46F7D114
:1075B0003F4B03EBC402D2F804C09846BCF1000F65
:1075C00004D131463B4801F0E5FB53E0002718F8B1
:1075D00034309F42F5DA3B010EEB0305103563446E
:1075E0000FCB013785E80F00F1E710F051FA0B28B7
:1075F000064643DC2846202110F0E7F9054648B14D
:107600000135284601F0B6F9214B012403EB06139E
:10761000186100E004462846202110F0D6F90546FE
:1076200040B10135284601F0A5F9194B013403EBAF
:10763000061358612846202110F0C7F9054640B1CD
:107640000135284601F096F9114B013403EB06137E
:1076500098612846202110F0B8F910B9FFF7B4FD61
:1076600011E0013001F086F9094B032C03EB0616FB
:10767000F061F3D11048FFF727FF04E00F48012124
:107680000C22FFF71EFD04B0BDE8F08190BC01089C
:10769000E8100020ABBC0108B1BC0108D5C7010847
:1076A0008ABC0108B5BC010844A40108BABC0108A1
:1076B00044BB0108C9BC010804BA010848BC010860
:1076C000F0B5047887B0064614BB514B19201968F1
:1076D000062303FB041191F8CA5091F8CE204543CC
:1076E00005F5617591F8C930009591F8CB50C83116
:1076F000684300F561700190087902904979454826
:1077000003912146013401F045FB0C2CDDD17CE0D6
:1077100010F0BEF90B28044672DC3D4B701C1D684E
:10772000202100238DF8173010F04FF9064680B164
:107730000136304610F0ACF903289FBF062303FB47
:10774000045383F8CE009DF817309CBF01338DF8A9
:1077500017303046202110F038F9074680B1013744
:10776000384610F095F90D289FBF062303FB0453FC
:1077700083F8C9009DF817309CBF01338DF817308E
:1077800006266643A9193846CA310DF11702FFF7DC
:107790006DFC202110F019F9074670B10137384609
:1077A00010F076F914289FBF9DF817307619013331
:1077B00086F8CC0098BF8DF817303846202110F09D
:1077C00004F978B1013010F063F90D289FBF06234A
:1077D00003FB045383F8CD009DF817309CBF0133A1
:1077E0008DF817309DF81730062B0ED0062202FBBD
:1077F00004500021C93010F0B2F8FFF7E5FC04E0B6
:10780000054800210B22FFF75CFC07B0F0BD00BF6C
:1078100018100020D5BC010848BC0108F0B502785A
:1078200087B08AB94A4C04F1280694F8F421002361
:10783000484950B2595681426DD00C333C2BF7D198
:107840000834B442F1D180E0002204920592451C34
:1078500010F01EF9C4B260B20AF0E8FC074618B195
:107860008DF81040012400E004462846202110F045
:10787000ACF8054638B10135284610F009F9013455
:10788000ADF81200E4B200262846202110F09DF841
:10789000B0B3451C284610F0FBF800222E495FFAD1
:1078A00082FE51F82230834204D00132082AF5D1F9
:1078B000002300E0734651F82320824220D1022E9B
:1078C0000FD0032E12D05A1E012ED2B204D0042A99
:1078D00013D88DF814300EE0042A0ED88DF8153028
:1078E00009E0052B09D88DF8173004E09A1E052A07
:1078F00003D88DF816300134E4B20136042EC3D11A
:10790000052C03D807B0BDE8F0405DE404AB03CB21
:107910003860796019E094F8F9010F4B94F8F85148
:1079200053F82000B4F8F621009094F8FB0153F8C6
:107930002000019094F8FA0153F8200053F8253004
:107940000290064801F026FA7AE707B0F0BD00BFC2
:10795000E810002014220020C09E0108F5BC010898
:107960002DE9F347047807464CB9204601A90CF0ED
:1079700009F90134FFF7F4FF122CF6D17DE010F085
:1079800087F8C5B2112D73D8781C202110F01DF88E
:107990003B4C05F1D00614F816800346394F30B938
:1079A000A8F10202D2F1000848EB020846E007F114
:1079B000260800F1010A5978404610F006F868B12F
:1079C000032D8CBF03230023C8EB0000C0B23B444F
:1079D000184490F82A90B9F1030F02D1FFF7F4FB95
:1079E0004BE0A9F10203D3F1000850464FF020010B
:1079F00048EB03080FF0E9FFD8B1B8F1000FEDD064
:107A0000013010F045F840F2ED2380B2984205DDD8
:107A100040F6CA039842A8BF184601E040F2EE20A3
:107A2000A0F2EE20192290FBF2F004EB460358700E
:107A300002E0B8F1000FD1D104F8169014F8163016
:107A40001F4497F82620B8F1000F0CD00C4B0E48BD
:107A500003EB4606717819234B43294603F2EE23C4
:107A600001F098F909E02946084801F093F904E08B
:107A7000074800211122FFF724FB02B0BDE8F08780
:107A8000E81000206499010814BD010826BD010812
:107A900051CA010807B50123ADF8041001A98DF8FA
:107AA00006208DF8073007F0BEFA03B05DF804FB3E
:107AB0002DE9F047814672B6514C4FF400774FF4F0
:107AC00080616161204667614822FFF7E3FF394624
:107AD00020461022FFF7DEFF1FFA89F6494A4FEAD7
:107AE000C60802EB0803596852F83650464B4FEA75
:107AF000D10E05EB8E00586055F82E0001F00701FD
:107B000098608900D8600F208840C043D3F80CC02B
:107B100052F839A000EA0C0CC3F80CC0D3F808C026
:107B200002EBC90900EA0C009860D8684FF0080C15
:107B30000CFA01FC4CEA0000D860D3F808C0012020
:107B400000FA01F141EA0C019960996845F82E109C
:107B5000D9F80410994600FA01F5CAF810502761C7
:107B60001746A3685805FCD4D9F80830D9F8042082
:107B7000082113604FF40073CAF814506361234B5B
:107B800019611021596140F60553A16849051AD4BD
:107B9000013BFAD1D9F80C3057F83600136007EBE7
:107BA00008025268C168012393400B43C3604FF43D
:107BB000007113481822FFF76DFF62B6BDE8F04769
:107BC00032200AF072BC4822CAF810505046A9B2BE
:107BD000FFF760FF0D4B10221A61A268084B520597
:107BE000C2D5DAF808204FF400701542074A4FF06A
:107BF000080115BF1861586111615161EDE700BFBF
:107C00000008014038BD0108A8190020000C0140FF
:107C100010B5044620460AF01AFD18B90A200AF0E9
:107C200044FCF7E710BD30B5094900220B78094C38
:107C30001557854202BFFF25155503F1FF3302F1A9
:107C40000C0208BFDBB23C2AF1D10B7030BD00BF83
:107C50009D10002014220020002208490C2303FB61
:107C600002135968814204D10022C2621A725A601A
:107C700070470132052AF0D1704700BF142200205E
:107C80002DE9F743064689469DF8288011461A4695
:107C90009DF82C3000250C2068431D4FC419C05797
:107CA000B04202D1207A20B12BE00135052DF2D16E
:107CB00027E0022E0FD005DC56B1012E21D1009312
:107CC00014480AE01E2E0DD01F2E1AD1012009E003
:107CD0000093114801E011480093434605F0E8FA8B
:107CE000044605E001F004FF414604460AF0ACFCFE
:107CF0004CB10C2303FB0575267185F808906C6068
:107D000001E0002000E0204603B0BDE8F08300BFA2
:107D10001422002000440040003801400048004088
:107D2000344B354A1B68126810B51A60334A116823
:107D30005960516892689960DA60314A1168196136
:107D40005168926859619A612E4A1168D9615168E7
:107D5000926819625A622C4A11881985518859858E
:107D60009188D2889985DA85284A118819865188A0
:107D7000598692889A86264A1188D986518892888F
:107D80001987194621F83A2F224A10780022824298
:107D900006DA214C34F81240013221F8024FF6E79E
:107DA0001E4A1288A3F864201D4A1288A3F8662090
:107DB0001C4A1188A3F86C1051889288A3F86E10A1
:107DC000A3F87020184A3B2112689A66174A126875
:107DD00092FBF1F2B2F5967FC8BF4FF0FF325A67BF
:107DE000134A1288A3F87820124A5289A3F85E2019
:107DF00010BD00BFF8310020AC3300208C1F0020E4
:107E0000981F0020A41F0020E0100020FC0F00207D
:107E1000CA100020F82F00201C1000203824002059
:107E2000BC0F002002100020D41000200000002011
:107E30003C100020081000202DE9F84305460E46AE
:107E40000D4B002493E88003B44213DA7B1933F915
:107E5000140008EB050333F9142009EB050333F98B
:107E6000143001341344022293FBF2F3C01A0AF0D7
:107E700048F9E9E7BDE8F883F831002010B5134B65
:107E8000014693F8DC37012B19D1114B114C1878AE
:107E9000421CD2B21A70120644BF00221A700E4A57
:107EA0001B7812782154934236BFC2F180029B1A8C
:107EB0009B183F2B09D9BDE8104006F013B9074BBA
:107EC000BDE8104018680AF0CEBB10BDE8100020D5
:107ED000082F00200A2F0020092F0020E031002069
:107EE00070B54720FFF7CAFF174B1B681B0307D568
:107EF000164B174A5B6810681B68C01A0AF0F1F845
:107F0000144E154C154D30780AF0EBF823682868AC
:107F1000C01A0AF0F6F863686868C01A0AF0F1F847
:107F20000F4B18880AF0DDF80E4B18880AF0D9F8C4
:107F30000D4B18880AF0D5F8337823742B68A360AA
:107F40006B68E36070BD00BF7C330020F831002017
:107F5000AC330020E6180020E4310020E8180020AF
:107F6000E4180020E2180020441000207FB5264CC1
:107F7000264E274D2749284A284B20B128480088FB
:107F8000B0F5805F31D2308891F820101278ADF8CA
:107F9000040028781C4D1B788DF806008DF807101A
:107FA0008DF8082001A8294606228DF809300FF027
:107FB000BBFC30B30198BDF808302860AB8053207B
:107FC000FFF75CFF20880AF08CF8A0780AF089F8A7
:107FD000E37801A80193237902936379039309F06D
:107FE000E5FF0F4B00221A800BE0308891F820103B
:107FF0002080127828781B78A070E170227163715C
:10800000DDE704B070BD00BFB8190020A41900203E
:10801000E0180020D42400203B0E0020A00E0020F9
:108020009C3300200A4A138801331380094A1368DD
:1080300001331360084A138801339BB2202B01BF20
:1080400000231380054A138808BF0133138070474B
:108050009C33002084330020883300208A330020A2
:1080600038B5394B05461B780C46083B012B6AD8BE
:108070004520FFF703FF2846FFF700FF0C2D23D014
:1080800004D80A2D0AD014D835B138BD0E2D4BD0E6
:108090002ED3FF2D50D038BD206849E02078FFF75F
:1080A000EDFE62796378002A14BF80200020184317
:1080B00000E02078FFF7E2FEA078FFF7DFFEE0782F
:1080C000FFF7DCFE20793BE0B4F9000009F0FEFF89
:1080D000A078FFF7D3FEE078FFF7D0FEB4F90400F4
:1080E00009F0F4FFB4F90600BDE8384009F0EEBF2E
:1080F000637820788BB180F08000FFF7BFFEA46822
:10810000E0B2FFF7BBFEC4F30720FFF7B7FEC4F3EE
:108110000740FFF7B3FE200E12E0FFF7AFFE6068E6
:10812000BDE8384009F0EDBF206809F0DAFF60686B
:10813000BDE8384009F0D5BF044809F0E6FF00204B
:10814000BDE838409AE638BDDC31002068BD010842
:108150002DE9F04FBE4B8BB01A880193BD4F002A1A
:1081600040F0A98042F20103B7F8DA07BA4EC21A0A
:1081700050425041FFF7FAFEFFF7D2FD3468492024
:108180002546FFF77BFEB54B04F11C09186809F082
:10819000A8FF55F8040B09F0A4FF284603F0F0FAF5
:1081A00004F1100003F0ECFA4FF01008AC4D01237D
:1081B0002A6803FA08F3134203D0D9F8000009F043
:1081C000A0FF08F10108B8F1130F09F10409EDD17E
:1081D00004F1280003F0C4FAB7F84031B4F92E00D6
:1081E000C01A09F07EFF2B68DB0408D59D4BB4F85C
:1081F00064001B88181AC0F30D0009F072FF2B6889
:10820000980403D5B4F8660009F06BFF2B68590594
:1082100003D504F16C0003F0A3FA2B681A0502D50C
:10822000A06E09F06EFF2B685B0402D5606F09F049
:1082300068FF2B68180403D5B4F8780009F051FFE3
:10824000A04604F1300003F08BFA04F1360003F08D
:1082500087FAB7F8403138F93C0F0127C01A09F006
:1082600040FF814B1B789F4208DA38F9020FB4F9BE
:108270003C300137C01A09F044FFF2E72B6899053A
:1082800005D5B4F95E00A0F2DC5009F03AFF32687F
:1082900076487260B260121A9110754A4A43531CB4
:1082A000032293FBF2F202EB42029A1A7C2303FBB5
:1082B00002033360D6E16F4B6F4A1B6811688B4233
:1082C00006D00AA941F8203D00201360FFF7C8FE40
:1082D000019B97F8DA171B8897F8DB070B44013BE3
:1082E000B3FBF0F200FB12338B4280F086815A4FD1
:1082F0000120FFF73BFEFFF713FD50203E687D682D
:10830000FFF7BCFDBA683B6810681B687A680344D5
:10831000106806F11C0BA3EB400009F0F2FE6A683E
:10832000736802A89B1A0293AA68B36805F11C0837
:108330009B1A0393EA68F36810249B1A049303F0D2
:108340001FFA2A69336902A89B1A02936A69736942
:108350009B1A0393B369AA699B1A049309F026FE3A
:108360003F4901220B68A2401A428A4606D0DBF838
:108370000000D8F80030C01A09F0C3FE0134132CF5
:108380000BF1040B08F10408EAD106F1260005F10F
:108390002601002331F9024F30F9022F121B02ACE3
:1083A00044F823200133042BF4D103214FF00009BA
:1083B0004FEA89035FFA83F902AB53F821206AB1CF
:1083C00002F108000F2802D849F0010906E08032C6
:1083D000FF2A94BF49F0020949F0030911F1FF3166
:1083E000E6D248460024FFF749FDA0460DF1080BF0
:1083F00009F00302022A16D0032A1DD0012A4ED109
:10840000B8F1000F05D1DBF8004090462401E4B23A
:1084100045E0DBF800004FF0000800F00F002043BB
:10842000FFF72CFD3BE0B8F1000F0CD0DBF80000AB
:10843000C0F3031020432CE0B8F1000F1ED19BF8CD
:108440000100FFF71BFD9BF80000FFF717FD26E07A
:1084500088330020E8100020F83100208433002009
:108460007C33002078330020F82F002004320020D5
:10847000DF7BEFBD903300208C330020DBF8000061
:10848000C0F303302043FFF7F9FCDBF80000C0F332
:108490000710FFF7F3FCDBF800402401E4B20BF116
:1084A000040B06AB9B454FEA9909A1D1B8F1010F26
:1084B00002D12046FFF7E2FCDAF8003013F48054D2
:1084C0001FBFB6F86420B5F864100124521A18BF13
:1084D00002929A040AD50AAA02EB8401B5F8660052
:1084E000B6F866200134121A41F8202C580513D52D
:1084F00002AA02EB840C06F16A0E05F16A00002262
:108500003EF9021F30F9028FC8EB01014CF822102E
:108510000132032AF4D10334190508D50AAA02EB63
:108520008400A96EB26E0134521A40F8202C5A040D
:1085300008D50AAA02EB8400696F726F0134521ADF
:1085400040F8202C18040BD50AAB03EB8402B5F8D5
:108550007810B6F8783001345B1A42F8203C00E01D
:10856000FCB1012C03D1029809F0CBFD19E0631E88
:10857000002002AA52F823204000C0B20AB140F005
:108580000100013BF5D5FFF779FC4FF0000802AB85
:1085900053F8280008B109F0B4FD08F10108A0451E
:1085A000F5DB30200321FFF747FC36200321FFF7DE
:1085B00043FC2F4B3C201978FFF73EFCDAF80030E3
:1085C000990506D5B6F95E00B5F95E30C01A09F016
:1085D00098FD3A6827487B687A60121A9110264AFB
:1085E000BB604A43531C032293FBF2F202EB4202AC
:1085F0009A1A7C2303FB02033B60204B1B681A067C
:1086000030D51F4C1F4D22682B689A420BD16268EF
:108610006B689A4207D1019B1B88102B11D11A4B12
:108620001B885B060DD14820FFF728FC206809F065
:1086300068FD606809F065FD23682B6063686B6006
:108640000EE0124A0F4B11782A7C914208D1104A51
:1086500099681068884203D15268DB689A4201D059
:10866000FFF73EFC09F090FC0BB0BDE8F08F00BFB7
:10867000F82F002004320020DF7BEFBD7C3100208A
:1086800048100020E43100208A330020E618002042
:10869000E81800202DE9F84F0C9EC2EB030B394C73
:1086A0000B9B002914BF4FF0060A4FF0040AF61A7C
:1086B000636805460133904613D1236853455ED263
:1086C000314A032B98BF294652F823202F4809F03E
:1086D00087FD63680022013363602D4B05469A7164
:1086E00013E0002511E02B4A1278954240DA0B9BEB
:1086F000E3B109FB06F2995C01228A402649096828
:108700000A4213D1636801336360D4F804900A9B72
:108710001C4F9945E7DB2BD10A20FFF7AFFB3B68E5
:1087200001333B604FF0FF337B6021E0184A9179C1
:1087300021B12C20FFF7A2FB013501E0012191714D
:1087400009FB0BF3226808EB030752B958F8030042
:1087500009F0DBFC97F9041005444B1CD2D00F48FC
:1087600002E03A440E48117909F03AFD0544C9E7A0
:10877000206850452CBF00200120BDE8F88F002064
:10878000BDE8F88F94330020549E010873BD0108A2
:10879000B8190020580000207C33002082BD010859
:1087A000BFBE010830B585B004AC002524F8025DD9
:1087B0000091ADF806002146102005F061FD9DF8FE
:1087C0000600214605F05CFD9DF80700214605F0F6
:1087D00057FD9DF80000214605F052FD9DF801006F
:1087E000214605F04DFD9DF80200214605F048FDAB
:1087F0009DF80300214605F043FD9DF80E00294633
:10880000C043C0B205F03CFD05B030BDF0B5012459
:10881000B0FBF4F58D4201D34C43F9E70026D4B107
:10882000B0FBF4F504FB1500B4FBF1F41EB9002D08
:1088300001DC002CF3D1092D03F1010EEFB204DDB0
:10884000002A14BF3725572500E030253D441D7010
:1088500001367346E3E71C70F0BDF0B50124B0FBB0
:10886000F4F58D4201D34C43F9E70026D4B1B0FBB7
:10887000F4F504FB1500B4FBF1F41EB9002D01DC86
:10888000002CF3D1092D03F1010EEFB204DD002A13
:1088900014BF3725572500E030253D441D700136B3
:1088A0007346E3E71C70F0BD03685A1C0260197040
:1088B00070472DE9F843089E002B0746884614466A
:1088C000334614BF4FF030094FF0200913F8012B45
:1088D0000AB9254603E0002CFBDD013CF6E7002D3C
:1088E00004DD38464946C047013DF8E7354624EAED
:1088F000E474A01B284415F8011B11B13846C04789
:10890000F7E7BDE8F883024B186809F0ACBE00BF7A
:10891000C80F0020F8B507460C46486800211546E8
:108920001E460BF0E9FF58B128460BF0FDFD10493B
:108930000BF04EFE01464FF07E500BF0FDFE6060E6
:10894000616830460BF03CFD014630460BF0F4FE0A
:1089500025680646294638460BF030FD014630466C
:108960000BF036FE014628460BF02AFD2060F8BDCC
:10897000DB0FC9402DE9F04102780346202A00F1BF
:108980000100F9D0092AF7D02D2A02D10346414D22
:1089900004E02B2A08BF03464FF07E551C460026F4
:1089A000234614F8012BA2F13007F9B209290DD89A
:1089B000394930460BF00CFE064638460BF0B4FD44
:1089C000014630460BF0FCFC0646E9E72E2A17D19B
:1089D000314F234614F8010B3038C2B2092A0FD8A0
:1089E0000BF0A2FD39460BF0A7FE014630460BF016
:1089F000E7FC2949064638460BF0EAFD0746E8E75A
:108A00001A7802F0DF02452A39D15A782D2A02D18C
:108A10000233012704E02B2A14BF0133023300275D
:108A2000013B002413F8012F303AD1B2092903D8B1
:108A30000A2101FB0424F5E7B4F59A7F28BF4FF41F
:108A40009A74A0464FF07E53B8F1070F07D9184625
:108A500012490BF0BDFDA8F108080346F4E704F045
:108A6000070434B118460C490BF0B2FD013C034633
:108A7000F7E719462FB130460BF05EFE04E04FF0E9
:108A80007E5130460BF0A4FD014628460BF0A0FDB8
:108A9000BDE8F081000080BF0000204120BCBE4C3A
:108AA00030B5054687B00C4603A800210C220EF015
:108AB00056FF284600210BF047FF20B128462849E1
:108AC0000BF07EFC03E0284625490BF077FC254996
:108AD0000BF07EFD0BF042FF054680EAE070694630
:108AE000A0EBE5700BF04EF8002DACBF20232D233A
:108AF00068468DF80C300EF076FF012807D1302340
:108B00008DF80D308DF80E308DF80F300CE0022806
:108B100005D130238DF80D308DF80E3004E0032898
:108B200004BF30238DF80D30694603A80EF03EFFD8
:108B300003A80EF058FF0338C5B22A4603A9204601
:108B40000EF07CFF00236355204607490EF02EFFF0
:108B500003AB204659190EF029FF204607B030BD5F
:108B60006F12033A00007A44A6BD010870B50646AC
:108B7000B6FBF2F40846154614B12046FFF7F6FF9F
:108B800005FB1464024B1B5D00F8013B70BD00BF88
:108B9000A8BD01082DE9F04F81468A4616461C46BD
:108BA00089B000253178002900F0DB80252902D02A
:108BB0000136484674E072784FF00008302A0CBF46
:108BC000B278B71CA2F1300312BF4FF0000BF71CB4
:108BD0004FF0010B092B19D8A2F13003D9B20929A2
:108BE00005D80A2202FB083817F8012BF4E7A2F196
:108BF0006103052B02D8A2F1570305E0A2F141035E
:108C0000052B03D8A2F137030A2BEADD6C2A30D1F9
:108C10003A787E1C642A00F083800BD8252A3DD048
:108C200003D8002A00F09D80BCE7582A0CD0632AA4
:108C300019D0B7E7732A22D002D86E2A37D0B1E70D
:108C4000752A5CD0782AADD1271D2068A2F158047E
:108C500062424FF01001624155E02CD9582A32D0BF
:108C6000632A2AD13E4648462178271DD047013540
:108C70000FE0642A63D00ED9732A14D13E462368CC
:108C800048460093514642460023FFF712FE271D37
:108C900005443C4686E7252ADFD13E464846252145
:108CA000D04701357EE70AD86E2A06D13E462368B2
:108CB00004341D6076E7002A53D03E4672E7752AD9
:108CC00026D0782AF9D1A2F1580304F1040C5A42B3
:108CD0002068CDF80CC04FF010015A4105ABFFF7EA
:108CE00095FDDDF80CC03E46644605AB0093484652
:108CF000514642465B46FFF7DCFD054452E72068DB
:108D0000271D0A21002205ABFFF7A7FD3C46ECE733
:108D100004F1040CCDF80CC020680A210022DDE724
:108D20002068271D002808DA2D238DF814304042D2
:108D30000DF115030A210022E6E705ABFAE72068EA
:108D400004F1040C00280ADA2D238DF81430404277
:108D50000DF11503CDF80CC00A210022BFE705ABC9
:108D6000F8E7284609B0BDE8F08F0EB40FB505ABA3
:108D700053F8042B0190064901A80393FFF70AFF5B
:108D8000019B00221A7004B05DF804EB03B0704739
:108D9000A98800080FB413B50B4904AB08680B4948
:108DA00053F8042B09680193FFF7F4FE0446084BBF
:108DB000186809F04CFC0028F9D0204602B0BDE844
:108DC000104004B0704700BFCC000020C800002055
:108DD000C80F002080EAE073A3EBE0738B4206DB50
:108DE000002801DD401A704702D008447047002077
:108DF00070472DE9F84321F0004520F00046074672
:108E00008846284631460BF09FFD08B9344600E0FD
:108E10002C46204600210BF06FFD60B928463146F4
:108E20000BF074FD08B9304600E0284621460BF0EF
:108E300083FC044600E00024204625490BF0C8FBD3
:108E400024490BF0BBFA21460BF0C2FB22490BF080
:108E5000B5FA21460BF0BCFB20490BF0AFFA2146D6
:108E60000BF0B6FB1E490BF0A9FA1E4900F10049B0
:108E700020460BF0ADFB1C490BF0A2FA21460BF08B
:108E8000A7FB4FF07E510BF09BFA014648460BF0D2
:108E900053FC2946044630460BF056FD20B12146CE
:108EA00012480BF08BFA0446404600210BF02EFDD1
:108EB00020B121460E480BF081FA044638460021C5
:108EC0000BF024FD08B104F100442046BDE8F8830E
:108ED00039094E3DE3B59E3E88FA163E45FE7F3F7A
:108EE000A7DFA83499FB243F69A2163EDB0FC93FD8
:108EF000DB0F494070B504460BF030FD20304028B0
:108F000057D820462C490BF01FFD28B120462B498D
:108F10000BF054FA0446F4E7204629490BF0F6FC1E
:108F200028B1204625490BF04BFA0446F4E72046C9
:108F300024490BF009FD30B1224920460BF03EFADE
:108F4000014620480AE020461F490BF0DFFC40B1F3
:108F50001C4920460BF034FA01461B480BF02EFA50
:108F60000446214620460BF033FB054620462946A1
:108F70000BF02EFB0021064628460BF029FB134977
:108F80000BF01CFA014628460BF022FB10490BF0AF
:108F900017FA014628460BF01BFB0E490BF00EFAA0
:108FA000014630460BF014FB014620460BF008FA50
:108FB00070BD002070BD00BFDB0F4940DB0FC94012
:108FC000DB0F49C0DB0FC93FDB0FC9BF92E7413957
:108FD0009730083C15A82A3E08B503490BF0F0F974
:108FE000BDE8084086E700BFDB0FC93F064B10B560
:108FF0001A881C4622EA00009042188002D0012004
:1090000009F0AEFA208810BDA4190020064B10B557
:109010001A881C4610439042188002D0012009F0A3
:109020009FFA208810BD00BFA4190020024A93684F
:1090300023EA000090607047E8100020024A93681D
:1090400018439060704700BFE810002008B5104B2F
:109050001A780023D9B2914207D20E49002051F864
:109060002310013309680880F4E7322009F01DFA63
:10907000094B1B685A0309D5084B9B685B0305D451
:10908000BDE8084040F2DC5009F00FBA08BD00BF4F
:10909000F82F0020C82F00207C310020E81000208D
:1090A0002DE9F34103F0C0FE4B4A6C2313704FF4DB
:1090B000FC635380BE231371EF2382F8DD37002356
:1090C0001946164682F8DE37F25C0133B3F5FC6FC1
:1090D00081EA0201F8D1404B404A83F8DE17404B49
:1090E00004275A6002F188325A600020013F17F0CD
:1090F000FF075ED03A4B34223A4CDA6004F17848EC
:10910000A8F5FC38C8F3090353B100234FF400500D
:1091100056F80880019303F05DFB0428E6D11CE0BB
:109120004FF4302003F056FB0428DFD12C4D4FF4D0
:1091300030202B6943F002032B616C612B6943F0F3
:1091400040032B6103F046FB41F6FD732A690428B6
:1091500003EA02032B61D8D0C8E7214D4FF4005039
:109160002B6943F001032B611FFA88F3238003F07E
:1091700031FB042813D1A31C0193019B4FEA18482B
:10918000A3F800804FF4005003F024FB41F6FE7377
:109190002A69042803EA02032B6106D0A6E741F6F8
:1091A000FE732A6913402B61A0E70F4B04349C42E5
:1091B000A4D10B4A0428136943F08003136102D140
:1091C00008F0BDFB10B9052009F0E2F903F016FE26
:1091D00002B0BDE8F08100BFE81000202301674520
:1091E0000020024000F80108E0FF010810B50E4C15
:1091F000206809F0A1F820680022047A02FB02F33B
:10920000193B634303F6C4135343192193FBF1F352
:10921000064921F812300132072AEFD1BDE810408B
:10922000034909F041B800BF40100020980F00200A
:10923000281200202DE9F04108F081FB10B904202C
:1092400009F0A6F9C04C03F0EFFDC0494FF4FC62F1
:1092500020460EF079FB94F8B4374FF4CC71022B12
:1092600084BF002384F8B43794F8B427B84D01FBC9
:1092700002F3E01800F53B702344286093F84003A4
:1092800001FB0242022803F54E7384BF00201872CE
:1092900092F84033AF4A13700C2202FB0343AE4AEC
:1092A00003F2B673136046F20903A26813401BB9B8
:1092B0004FF40050FFF7C2FEA368DF0703D54FF459
:1092C0000050FFF7B3FEA3685E0409D50820FFF73E
:1092D000ADFE4FF40050FFF7A9FE0120FFF7A6FEF8
:1092E000A368180706D54FF40050FFF79FFE012032
:1092F000FFF79CFEA368990413D54FF40040FFF7D5
:1093000095FE914B93F88431012B03D14FF400600B
:10931000FFF78CFE4FF48030FFF788FE4020FFF708
:1093200085FEA3685A0603D54FF48030FFF77EFE12
:10933000A36803F40852B2F5085F0AD11B0508D5EB
:10934000814B93F88431012B03D14FF40060FFF778
:109350006DFE94F8DE217C4B2AB193F8E22112B124
:10936000002283F8E2214FF0000C67467B4E7C4BD5
:109370001E6004EB0C03B3F8F6E14FEA5E0101F066
:1093800077314FEA9E0303F03333C1EB0E00C11A6D
:109390004FEADE0303F01133CB1A03EB231303F080
:1093A0000F32FF2392FBF3F31EF00108C3EB0323FC
:1093B00018BF0137A2EB030318BFFFB2012B0ADD70
:1093C000022B40F0BE80B8F1000F00F0BA801EF012
:1093D000BC0F00F0B6800CF1080CBCF1280FC8D10E
:1093E000013F012F00F2AD80FFF700FF3022002186
:1093F0005C480EF0B4FA5C4F5C4BD5F800801F60FF
:109400005B4B002108F17900C3F8008008F0D2FF1F
:10941000584B80F001001870574B07F128021A6072
:10942000564B07F1DC021A6098F8000001F096FE36
:109430002868534B00F5C5721A6004F085FC514B47
:1094400094F8D61107F196021A6064224A434E4BF3
:10945000C8325A6000229A60DA601A615A619A61D1
:10946000DA6183F8202083F82120484B2D6807F12A
:109470002E021A60464B05F219121A60454B05F28E
:1094800089121A60444B07F108021A60434BDFF857
:1094900040811F60424B07F1A2021A6007F1AC0342
:1094A000C8F800303F4BB4F864011E600BF038F888
:1094B000C8F80800B4F866010BF032F895F85C3093
:1094C00008F1040288F8043095F87830C8F80C00E8
:1094D00088F8053094F8E131286E88F81030324B66
:1094E000C8F814501A6005F16403C8F818302F4901
:1094F0000BF06EF801464FF07C500BF01DF9B5F8FB
:109500001641C8F81C0020460BF00EF8014628480A
:109510000BF012F927490BF05BF8274A274B15602F
:10952000274A186005F168031360264A05F21115F1
:109530001560254A1760254ABDE8F041136003F025
:109540005DBC02F069F94FE7E810002000F801085F
:10955000181000203431002040100020701200202C
:10956000C8240020CC0E002028120020000F00206C
:10957000040F002008000020400700208C05002078
:10958000100F0020382E0020D4240020F01F0020CF
:10959000102E00203C0900209C300020A03000202C
:1095A000500800201409002068200020DB0F4940EB
:1095B000000061444C3D0F44100700204C0800207F
:1095C000040700203C08002044080020000600207A
:1095D000C019002008B5FFF763FDFFF72BFEBDE8BB
:1095E0000840012008F0BCBF426A806A131A584242
:1095F000584170474171704743799B070AD5436AC8
:109600008269D154436A01690133B3FBF1F201FB72
:10961000123343627047437913F001031FBFC368DD
:1096200003F1FF32C369006A1DBF181A1040C0B2AF
:1096300018467047437910B513F0010304460DD066
:10964000FFF7E9FF58B1236A6269E168D05C013332
:10965000B3FBF1F201FB1233236210BD184610BDBB
:1096600090F83B3210B57BB990F83A3290F8394215
:10967000A34209D2B0F8401201229A400A430133B2
:10968000A0F84022DBB2F3E710BD8379DB0748BFC7
:10969000B1FA81F1D0F8343148BF49095A681B89C1
:1096A00009B1136170475361704710F80A3C0133E8
:1096B000DBB20A2B84BF10F8131C054A00F80A3CE1
:1096C00082BF002322F8113000F80A3C704700BF27
:1096D00044230020334A70B5136C9068194440F657
:1096E0008C23081A98429160D060516013463BD990
:1096F000127893F9451010468A420BD1111F0829A0
:1097000008D893F84610182901D8013103E083F8EE
:10971000442002E0002183F8461093F94440214997
:10972000A24219D191F84740B4B10C3100249442BF
:1097300006DA51F8046F1C4D25F814600134F6E781
:109740000C2805D01849002421F810400130F7E713
:10975000164801780131017083F84520002201216B
:109760001A7083F8471070BD92F84710C9B140F2E3
:10977000DA51A0F2EF248C4208D811780B2905D8D1
:109780000B1D0131117042F8230070BD002283F8D7
:109790004720074B03F13002002143F8041F934296
:1097A000FAD170BDF400002044230020BC05002045
:1097B00000010020024A136C013319441164704700
:1097C000F4000020024B53F820301B6819807047CA
:1097D000C82F0020074BA1F57A7153F820301A6882
:1097E0001B8959434FF47A7391FBF3F189B21180CD
:1097F000704700BFC82F00201FB50123ADF8083007
:10980000ADF80410002301A9ADF80A30ADF80C3012
:10981000ADF8062002F0EFFF05B05DF804FB38B5A7
:10982000A0F513746379A579DB0745D594F8383230
:1098300005F00105F3B1226B1068838DC3F34E036D
:10984000838494F83C3223B1B4F842320133A4F853
:109850004232917A6A00FFF7CFFF012384F83B324E
:10986000002384F8393284F83A3284F83832A4F884
:10987000403238BD94F83B322046012B04BF94F8A7
:10988000393284F83A32FFF7EBFE94F83B22236B2F
:109890003AB9012284F83B221868997A05FA02F253
:1098A00007E0002284F83B2295421868997A08BFA5
:1098B0000222BDE838409FE738BD10B5A0F512740C
:1098C00094F83C22BAB9A36A616A994228D0591C1B
:1098D000A069A162C35C2069DBB25B0043F4007342
:1098E0008142A4F83E324FF00A0384F83D3228BF8B
:1098F000A262012312E094F93D327BB1B4F83E122A
:1099000020464B08A4F83E3201F00101FFF7BDFEEE
:1099100094F83D32013B84F83D3201E084F83C325A
:1099200094F83832002B4ED194F839320133DBB23F
:10993000092B84F8393203D12046BDE810408FE668
:109940000A2B40D194F83B322BB9B4F8403243F0A3
:109950000103A4F840326379D9071CD5B4F840025A
:10996000820501D4C30705D4B4F844320133A4F806
:10997000443210E0E36AC0F347000BB198470AE0B5
:10998000E3696269D054E369E1680133B3FBF1F242
:1099900001FB1233E361012284F8382294F83B2260
:1099A0000023012A84F839320DD1A27984F83B32A0
:1099B000236B12F0010F1868997A0CBF0222002263
:1099C000BDE8104018E710BDF0B5046D8279A38999
:1099D000467923F4005312F0020F4FEA03434FEA93
:1099E00013430CBF00214FF4005112F0040FA38168
:1099F00014BF4FF4806E4FF0000E16F0010F876811
:109A0000054614BF04200020B307238A48BF40F056
:109A100008029BB223F4405343EA01032382A18945
:109A200048BF90B289B221F4B05121F00C014EEA46
:109A3000010140EA0102A281A38A87B023F44073A6
:109A40001B041B0CA38201A802F07AFE039B049E58
:109A5000254A944218BF1E46A389192272431BB29D
:109A6000002BB4BF7E00BE00B2FBF6F66427B6FB47
:109A7000F7F00001010907FB1163A28912B2002A65
:109A8000B7BFD9001A013231B1FBF7F2A7BF3232AA
:109A9000B2FBF7F302F007021043A8BF03F00F0375
:109AA000AA79A8BF184380B212F0010F20812B6D54
:109AB00006D00E498B4202BF042001F548410861DF
:109AC00012F0080F9A8A0BBF22F0080292B2120419
:109AD00042F0080208BF120C9A829A8992B242F4AC
:109AE00000529A8107B0F0BD0038014000440040A8
:109AF0002DE9F04F504C4FF4147685B080469146D6
:109B00001D4606FB0046274608B94C4B02E00128DB
:109B100004D14B4B33631033C6F834314FF4147314
:109B200003FB08F3474AFC18FA50032262712246ED
:109B300003F59C733B44E162A36100214FF4807004
:109B4000D4F8343134324FF0010B62612162E161AB
:109B5000A162616284F83C1284F83912A4F84212BE
:109B6000A4F84412C4F80890A571E060206184F85C
:109B700038B284F8468258681B890222ADF80C304E
:109B800003A910238DF80E308DF80F20019205F0F7
:109B90004AFA236B019A597B58681B898DF80E107D
:109BA00003A9ADF80C308DF80F2005F03CFA3046D3
:109BB0005946FFF76AFD322008F077FC224BD4F8B3
:109BC00034A11B681A46B2FBF9F1B1F5803F03D30B
:109BD000012AF8D95208F6E71C4A5046B3FBF2F2C4
:109BE00089B2D2B203F098FA4FF4147000FB08F077
:109BF000174B07EB000800F512703C180022C8F85C
:109C000048325046214603F0CFFAD8F8307015F0AC
:109C1000010F0CBF022200223868B97AFFF7ECFD71
:109C20000C4B3846C8F84C32211D002203F0BCFA18
:109C3000304605B0BDE8F08FE019002004B60108F9
:109C400024B601086C9E01085400002040420F0019
:109C5000BB9800081F98000803460A4690F8460281
:109C6000D96A9B7944E71FB50123ADF8083000237A
:109C7000ADF80C30ADF80A30084BADF804101B7885
:109C800001A9012B08BF0323ADF8062008BFADF8DA
:109C90000C3002F0B0FD05B05DF804FBF0000020D0
:109CA00038B510F80E2C044650F8043C52B9012285
:109CB00000F80E2C20F80C1C997A18680222BDE8D6
:109CC0003840D0E730F80C2C20F80A1C891A89B2E9
:109CD00020F8081C074A10F80F0C002522F8101075
:109CE00004F80E5C1868997A2A46FFF7BCFF04F85E
:109CF000065C38BD44230020044B53F820301BB1D0
:109D000007289CBF1B681980704700BF1C020020F9
:109D10002DE9F7438E460546DFF8A092114699F8E3
:109D2000A0440068164698467246631C89F8A03421
:109D300003F09EF92B8901A9ADF8043018238DF8A2
:109D40000630686802238DF8073005F06CF9AB7AAD
:109D500009F2A447240127442A6849460C2B00F243
:109D6000F680DFE813F00D00F400F400F400510079
:109D7000F400F400F4008A00F400F400F400C200DF
:109D8000138CDFF83CC223F001031B041B0C13846B
:109D9000138CB2F804E0108B624520F073004FEA98
:109DA00000404FEA10409BB21FFA8EFE40F0700058
:109DB00014D00CF5006C624510D00CF5406C624577
:109DC0000CD00CF5806C624508D00CF5806C6245B7
:109DD00004D023F0020343F0030307E023F00E0353
:109DE0002EF4407E43F003034EF4807EA2F804E09C
:109DF0001083A2F834801384138B23F008031B0410
:109E00001B0C43F0080336E0138CDFF8B4C123F0D9
:109E100010031B041B0C1384138CB2F804E0108B8A
:109E2000624520F4E6404FEA00404FEA10409BB202
:109E30001FFA8EFE40F4E04008D00CF5006C62453D
:109E400004D023F0200343F0300307E023F0E003C5
:109E50002EF4406E43F030034EF4806EA2F804E01E
:109E60001083A2F838801384138B23F400631B043F
:109E70001B0C43F40063138369E0138CDFF840C1CB
:109E800023F480731B041B0C1384138CB2F804E0BE
:109E9000908B624520F073004FEA00404FEA10407B
:109EA0009BB21FFA8EFE40F0700008D00CF5006CDB
:109EB000624504D023F4007343F4407307E023F4B5
:109EC00060632EF4405E43F440734EF4805EA2F86B
:109ED00004E09083A2F83C801384938B23F0080362
:109EE0001B041B0C43F0080330E0138CDFF8D0C0D8
:109EF00023F480531B041B0C1384108CB2F804E071
:109F0000938B20F4005023F4E6431B0400041B0C45
:109F1000000C62451FFA8EFE43F4E04340F44050CB
:109F200003D00CF5006C624503D12EF4804E4EF444
:109F3000804EA2F804E09383A2F840801084938BB3
:109F400023F400631B041B0C43F4006393832B7BFB
:109F500043B1B2F844306FEA43436FEA53439BB2D4
:109F6000A2F8443013889BB243F001031380AB7A0C
:109F70000C2B19D8DFE803F0071818180B1818185D
:109F80000F18181813000B1902F134000AE00B190E
:109F900002F1380006E00B1902F13C0002E00B1957
:109FA00002F14000C3F8A40438460C44A4F8AC64A1
:109FB000C4F8A82403B0BDE8F08300BFE019002076
:109FC000002C014004F0FEBE04F0FCBE04F0FABE1A
:109FD0002DE9F84F4668D1F808A0D0F808904F68EE
:109FE0000D68D0F800805146304614460AF0F0FA69
:109FF0003946834648460AF0EBFA014658460AF0CD
:10A00000DDF92946206048460AF0E2FA51468146C9
:10A0100040460AF0DDFA014648460AF0CFF93946D3
:10A02000606040460AF0D4FA2946074630460AF0F6
:10A03000CFFA014638460AF0C1F9A060BDE8F88FB2
:10A040002DE9F04106460D464068496814460AF07D
:10A05000B7F9A9688046B0680AF0B2F929680746DE
:10A0600030680AF0ADF9C4F804802060A760BDE84C
:10A07000F0812DE9F04106460D4608467168144608
:10A080000AF0A6FAB168804628460AF0A1FA2946E5
:10A09000074630680AF09CFAC4F804802060A76084
:10A0A000BDE8F0812DE9F04F87B00393904B8146D6
:10A0B0001B889346980737D540F2E632109B8D48AF
:10A0C000DC89B0F900301B1B03F2F315954203D86D
:10A0D000002BB8BF5B4201E04FF4FA73B0F90220E5
:10A0E00040F2E630121B02F2F314844203D8002A35
:10A0F000B8BF524201E04FF4FA729342B8BF134620
:10A100000522C3F5FA7393FBF2F30A22643B53432F
:10A1100099F81C20D2105343642293FBF2F31344AA
:10A1200023EAE373DBB200E06423C8460093CB1C50
:10A1300002930025029B022D13F8016F6E4F0293CC
:10A140004FEA450A05D1B7F904301B365E43761154
:10A1500049E06A4B37F9152033F9153003EB420219
:10A16000CBF100039A4203DB5A451346A8BF5B4676
:10A17000634A32F90A40039A1B1B32F91540234403
:10A18000019306F0F1F8019B88B15E4A1846545DD0
:10A190000AF0CAF95C490AF0CFFA0146204609F0F4
:10A1A000D3FA59490AF014FA0AF0D8FB0346504A88
:10A1B0001288D10713D437F90A401B366643920739
:10A1C0004FEA26160FD599F812409DF900206343F7
:10A1D0005343642293FBF2F306EB231603E099F852
:10A1E00008405C432611494B042433F90A3098F89F
:10A1F000017093FBF4F4341B6743454E022DAB5DB5
:10A2000003FB07F701934FF0640397FBF3F74FEA63
:10A21000E7170AD138460AF087F9311D1E22F36884
:10A22000FEF778FB0AF09AFB07463A4A384B11884A
:10A2300003F1100E01FB04F298F80B605EF82500A4
:10A24000D21206FB0206344AB6F5001FA8BF4FF42F
:10A2500000169642B8BF164603F11C0252F82500BC
:10A2600042F825404FF6FF720909B2FBF1F1201ABE
:10A27000484399F850404EF825604FEA850C761314
:10A2800080118CB1CDF810C005930AF04DF9059BF3
:10A29000224603F1280101EBC501DB68FEF73AFB1A
:10A2A0000AF05CFBDDF810C098F815301B4A5843E3
:10A2B000019BB91943431846642390FBF3F31B1227
:10A2C000194422F80A10013502F108014CF8017016
:10A2D000032D02F1140102F120024CF801604CF848
:10A2E000023008F101087FF425AF07B0BDE8F08F18
:10A2F000A4190020B8310020E0100020C433002051
:10A30000743100208C9E010800002041FC0F0020C9
:10A31000441F0020F82100200000E0FF841F0020DF
:10A320002DE9F04F054690F850008DB00991069246
:10A330000A9318B13228A8BF322000E001200AF0A9
:10A34000F3F80146A9480AF0F7F9A94B0446188822
:10A35000002808BF01200AF0E7F8A64907900AF094
:10A3600037F90190019920460AF02AF80146019830
:10A370000AF0E2F9A04B08901B889A0724D59F4960
:10A38000B1F90030B1F9020083EAE37280EAE071CA
:10A39000A2EBE372A1EBE07191420C46B8BF144608
:10A3A000B4F5E17F12DA914203DD0028D8BF4042C4
:10A3B00003E0002BCCBF184658420AF0B5F890498C
:10A3C0000AF0BAF9064603E0002601E04FF07E5697
:10A3D0004FF0000804950024CDF808806300059331
:10A3E000884B33F914000AF09FF887490AF0F0F817
:10A3F0000AF0B4FA0AF098F884490AF0E9F87F4BB9
:10A40000039033F914000AF08FF87B4B07461B8842
:10A410009B077ED0014609F0D3FF7D4B804633F980
:10A4200014000AF081F80146404609F0C9FF0AF01D
:10A4300095FA069B5B42984203DB069B8342A8BFCA
:10A440000346744A0599885E0A9A1B1A32F9140069
:10A4500018440AF069F8804605F086FF70B16E4B2B
:10A4600040466E4914F803900AF066F901464846E2
:10A4700009F06AF969490AF0ABF88046287F0AF0CA
:10A480004FF867490AF0A4F88246287A0AF048F89B
:10A49000014640460AF09CF862490AF099F80AF031
:10A4A0005DFA81460AF100400AF058FA814505DB61
:10A4B00050460AF053FA4845A8BF48460AF034F817
:10A4C000DFF884A10290019940460AF081F85AF819
:10A4D000241009F075FF54494FEA840B80460AF0B6
:10A4E00015FA38B9404651490AF02EFA20B1DFF882
:10A4F0003C8101E0DFF830814AF80B80A87C0AF04B
:10A500000FF8014640460AF063F849490AF060F83E
:10A510008046394BB3F800A01AF0010F40F0968046
:10A52000384B059A4FEA840BD35EDFF81491002B69
:10A53000B8BF5B42B3F5206F03DD002349F8243038
:10A5400029E03C4938460AF043F8049B0B905878C0
:10A5500009F0E6FF0B9A014610460AF0EDF8039960
:10A5600009F02CFF01990AF033F859F8241009F08A
:10A5700027FF314981460AF0C9F938B948462F49C1
:10A580000AF0E2F920B1DFF8B49001E0DFF8A8901A
:10A590002B4A42F80B90049BD87A09F0C1FF284B54
:10A5A00053F824100AF014F826490AF011F81AF0AA
:10A5B000020F81464CD03846029909F0FFFE014651
:10A5C00030460AF005F80146029809F0F9FE4146C6
:10A5D0000746484609F0F2FE0146304609F0F8FF0A
:10A5E0000146404609F0ECFE814631E083F9223E07
:10A5F000D80F0020BD378635A4190020E0100020B8
:10A600000000E143FC0F00200000A03ECDCC4C40F8
:10A61000C4330020743100208C9E010800002041CA
:10A620000000A0406F12033C0000F0C10000F041A8
:10A630000AD7A33D0000A043000040C300004043F0
:10A64000B81F00200AD7233CB01F0020C146029F3C
:10A65000DFF820A20AF18002105D09F065FF0146D3
:10A66000039809F0B5FF7B4909F0B2FF014638466F
:10A6700009F0A4FE0AF1840B5BF824100746039846
:10A6800009F09CFE01990AF057F8039B0AF18C022D
:10A690004BF8243052F824B00392594609F08EFE4C
:10A6A0000146089809F094FF0146584609F088FED3
:10A6B000039A834642F824000AF19402105D09F0DF
:10A6C00033FF0146584609F083FF634909F080FFD4
:10A6D00083464946384609F073FE594609F06EFE36
:10A6E0000DF04AFB059B0AF14002D0520AF14802E4
:10A6F000384603920AF032F9039A0AF1540742F8F5
:10A70000240048460AF02AF947F824000BF10040DB
:10A710000AF024F9049B0AF16007013347F824008A
:10A7200004930CB9012459E6099A4C4B9479B3F976
:10A730000430640028345C43494B6411B3F90400CD
:10A7400009F0F2FE4FF07A5109F042FF0DF014FBD0
:10A75000201A09F0E9FE002CB8BF6442322C0646EC
:10A7600003DD0023CAF8183027E007980AF0F6F84E
:10A7700020F0030009F0D8FE0746687B09F0D0FE00
:10A780000146304609F024FF36490446384609F0B0
:10A79000D3FF0146204609F01BFF0AF0DFF8DAF884
:10A7A00018301844304B9842A8BF18462F4B984297
:10A7B000ACBFCAF81800CAF81830DAF818306FF0D1
:10A7C000FF005B13B3F5807FA8BF4FF480739842FE
:10A7D000B8BF184609F0A8FE074630460AF0BEF892
:10A7E000EB785843801109F09FFE214B04461B78FB
:10A7F000032B11D9B5F84E50B5F5FA7F0CD20AF0FB
:10A80000ADF86B42984203DBA8420346A8BF2B4633
:10A81000184609F089FE04463946204609F0D0FD65
:10A820000AF09CF800B209F07FFE0DF0A5FAAAF834
:10A83000440020460AF092F8CAF8500038460AF060
:10A840008DF80023CAF85C00CAF868300DB0BDE886
:10A85000F08F00BFA69B443BF7CC9238E01000205D
:10A86000FC0F002000803B45FEFFFF0F020000F0C0
:10A87000F82F0020441F00202DE9F04F834699B0A7
:10A88000894C94F89770254647B1012F40F05184C8
:10A89000D4F8D870D4F8DC60002415E107F0DEFDB0
:10A8A0000646C4F89800D4F8A000301A09F038FE23
:10A8B0007E4909F08DFE7E4BC4F89C005B6804F174
:10A8C000A400C4F8A060984704F1A406002800F092
:10A8D000E480784B30461A78314602F051F9B4F8EA
:10A8E000AA30002B43D03B46D4F8AC00B5F8AA20E0
:10A8F0007149B2F5C87F04BF002241F823204FEA16
:10A90000830C36F913E051F80C20674F724441F87C
:10A910000C20002126F8131020F813100133032B0C
:10A92000E4D1B7F8AA30012B1CD1D7F8B0304FF4DE
:10A93000C87EC83393FBFEF20280D7F8B420C83239
:10A9400092FBFEF24280D7F8B8305C4AC83393FBE2
:10A95000FEF312889B1A8380ABF80010ABF802104C
:10A96000FEF738FEB4F8AA30013BA4F8AA30544BE5
:10A970001B685B077DD5B4F8BC204B4B322A13D142
:10A98000D3F8AC201188A3F8BE1051889288A3F8A0
:10A99000C010A3F8C220BBF80020A3F8C420BBF865
:10A9A0000220A3F8C62001E0002A40D0D4F8AC1061
:10A9B0000020B5F8BC304FEA800E322B414B04BF6B
:10A9C000002243F8202036F910C053F80E20364FED
:10A9D000624443F80E20002326F8103021F810308E
:10A9E000013003281A46E4D1B7F8BC30012B19D145
:10A9F0000C2087F8D42087F8D53007F08FFDD7F8E2
:10AA0000AC30B7F8BE201A80B7F8C0205A80B7F82B
:10AA1000C2209A80B7F8C430ABF80030B7F8C6301F
:10AA2000ABF80230B4F8BC30013BA4F8BC3094F869
:10AA3000D6301D4AEBB1D2F8C830322193FBF1F386
:10AA4000D2F8AC50002082F8D6002B80D2F8CC305F
:10AA500093FBF1F36B80D2F8D030184A93FBF1F3FB
:10AA600012889B1AAB80ABF80000ABF80200FEF72F
:10AA7000B1FDD4F8AC20B4F8A43011885B1AA4F866
:10AA8000A4305188B4F8A6305B1AA4F8A630928896
:10AA9000B4F8A8309B1AA4F8A83094F89730013382
:10AAA00084F89730ECE600BF441F0020BD378635A0
:10AAB0004C210020CA330020F41F00201C0000207D
:10AAC0007C3100200C200020DFF8DC8208F1A40299
:10AAD00032F81400B04A08F1E00522F8140000B280
:10AAE00009F022FD394609F073FDAC4A45F824000F
:10AAF00032F9140009F018FD314609F069FD08F13A
:10AB0000EC0545F824000134032CDDD128462A4603
:10AB100008F1F801FFF794FA284608F5827106AAB1
:10AB2000FFF78EFA06A80246D8F89C10FFF7A1FAA4
:10AB300006984FF07C5109F04BFD4FF07C510646D2
:10AB4000079809F045FD4FF07C510546089809F03B
:10AB50003FFD31460446304609F03AFD2946074696
:10AB6000284609F035FD0146384609F029FC214602
:10AB70000746204609F02CFD0146384609F020FC26
:10AB80004FF07C5109F024FD01464FF07E5009F052
:10AB900015FCD8F81491D8F8183149460193029061
:10ABA00009F016FD01990390204609F011FD039A62
:10ABB0000146104609F004FCD8F81C710390394690
:10ABC000284609F005FD039A0146104609F0F6FBF8
:10ABD000D8F810A103905146304609F0F9FC039AC9
:10ABE0000146104609F0ECFB01990590029809F026
:10ABF000EFFC39460390304609F0EAFC039A01461F
:10AC0000104609F0DDFB51460390284609F0E0FCB0
:10AC1000039A0146104609F0D3FB494603902046AB
:10AC200009F0D6FC039A0146104609F0C7FB4946D5
:10AC30000490284609F0CCFC01990390304609F0B5
:10AC4000C7FC039A0146104609F0B8FB3946039049
:10AC5000029809F0BDFC039A0146104609F0B0FBCA
:10AC600051460390204609F0B3FC039A0146104672
:10AC700009F0A6FB51460390029809F0A9FC494649
:10AC80008246304609F0A4FC0146504609F096FB86
:10AC900001990646284609F09BFC0146304609F01A
:10ACA0008DFB39460546204609F092FC01462846B0
:10ACB00009F084FB059BDDF810C0C8F81431C8F812
:10ACC0001001C8F818C1039A03F1004109A8C8F897
:10ACD0001C2102F100420CF1004C09910B9201463B
:10ACE0000CAACDF828C0FFF7ABF92D48D8F8101101
:10ACF00012AAFFF7BEF90FAE09A8294915AAFFF756
:10AD000067F915A812A93246FFF79AF90CA831463F
:10AD100015AAFFF75DF93246214815A9FFF790F90A
:10AD20001198D8F8201109F00FFE1E4B1A7810B1B7
:10AD300042F0080201E022F008021B4C1A70D4F81D
:10AD4000243104F596771B7883B3D4F828913846DC
:10AD5000494612AAFFF78DF9D4F8388104F1E000D2
:10AD6000414615AAFFF785F912A815A93A46FFF73B
:10AD700067F904F59E70494612AAFFF77AF9304642
:10AD8000414615AAFFF775F912A815A904F59E7298
:10AD9000FFF756F916E000BFCA100020FC0F002094
:10ADA000909E0108E0180020441F002004F1E003F9
:10ADB00004F59E7593E8070087E8070096E807000A
:10ADC00085E80700D4F8E000D4F8E480014609F0F3
:10ADD000FFFB41460546404609F0FAFB014628467E
:10ADE00009F0EEFAD4F8E87005463946384609F01D
:10ADF000EFFB0146284609F0E3FA9A49074609F0B5
:10AE0000A3FD994E002520B93846984909F07EFDEA
:10AE100030B1C4F80451C4F80851C4F80C5112E020
:10AE200006F5827206F5967006F59E71FFF7D0F86A
:10AE3000D6F89C108E4809F07FFC014606F582701A
:10AE40000246FFF716F9B4F84831874D01339BB23B
:10AE5000B3F57A7FA4F848314ED1D5F81001D5F872
:10AE60001491014609F0B4FB49460646484609F0EC
:10AE7000AFFB0146304609F0A3FAD5F81881064623
:10AE80004146404609F0A4FB0146304609F098FAD5
:10AE9000D5F81C7106463946384609F099FB01463B
:10AEA000304609F08DFA0DF0A5F901464FF07E50BD
:10AEB00009F042FCD5F81411064609F089FBD5F8D3
:10AEC00018118146304609F083FBD5F81C118046E5
:10AED000304609F07DFB31460746D5F8100109F0F0
:10AEE00077FB0023C5F81001C5F81491C5F8188147
:10AEF000C5F81C71A5F84831D4F81081D4F8186150
:10AF00004046314609F064FBD4F81471D4F81C5162
:10AF100039460446284609F05BFB0146204609F005
:10AF20004DFA014609F04CFA4FF07E51044609F003
:10AF30000BFD50B920464F4909F0E8FCE0B9204626
:10AF40004FF07E5109F000FD08B14FF07E542046CD
:10AF500009F08CF90CF070FF09F0DCF900210446CF
:10AF600009F0F2FC48B14449204609F027FA0021D3
:10AF700009F0EAFC88B923E0404C04F100493E495D
:10AF8000484609F01BFA0021824609F0DDFC90B129
:10AF90002046002109F0D8FC30B12046364909F09E
:10AFA0000DFA4FF0010902E04FF001095046344913
:10AFB00009F0ACFC0FE02046002109F0C5FC08B107
:10AFC000204600E048462C4909F0F8F92D494FF099
:10AFD000010909F0B9FC00B981465FFA89F353B160
:10AFE00028464146FDF705FF014609F0E9F94FF013
:10AFF000000A05467DE03946404609F0E9FA29464F
:10B000008146304609F0E4FA0146484609F0D8F98D
:10B01000014609F0D5F931460190304609F0D8FAD9
:10B0200081463946384609F0D3FA494609F0C8F94D
:10B03000014609F0C5F901464FF07E5009F0BEF90E
:10B0400000218246019809F057FC20B150460021AA
:10B0500009F052FCC0B951460198FDF7CAFE82467C
:10B0600014E000BFB81E8D3F441F00203D0A673F1B
:10B070006F12833A000080BFDB0FC93FDB0FC9BFEF
:10B0800035FA0E3C35FA0EBC4FF0000A2946404610
:10B0900009F09EFA31468046384609F099FA014691
:10B0A000404609F08DF9014609F08AF9294606461D
:10B0B000284609F08DFA0146484609F081F9014613
:10B0C00009F07EF901464FF07E5009F077F9002132
:10B0D0000546304609F010FC20B12846002109F051
:10B0E0000BFC28B929463046FDF783FE054600E0F3
:10B0F00000251549504609F06BFA0CF03DFE134E41
:10B1000011493080204609F063FA0CF035FE1049F1
:10B11000708005F1004009F05BFA09F01FFC80B275
:10B120000C4B10F4004F18BF00F5B47018800023CA
:10B1300000E00123084A002182F89710002B7FF4D9
:10B140009FAB19B0BDE8F08F4D3D0F447431002026
:10B15000E12E6542D8100020441F002001380A4B20
:10B16000042804D8DFE800F00507090B0D00074AA2
:10B1700008E0074A06E0074A04E0074A02E0074AF7
:10B1800000E0074A1A6070474C000020BD09010822
:10B19000A5A00008990C0108D10601088D0301083B
:10B1A00021A3000808B508480CF01DFCC0B209280E
:10B1B0000246054B04DC01302021C0B29954F6E769
:10B1C00000221A5408BD00BF812D002008B5074891
:10B1D0000CF009FCC0B21428044B04D8421C2021F6
:10B1E0001954D0B2F7E700221A5408BD812D00206F
:10B1F0002DE9F74F07F032F9A64C804626686568BE
:10B20000A768861BF643451BC71BED43FF43F60F9C
:10B21000ED0FFF0F2EB93FB9002D00F08782B94620
:10B220002CE04FF0000929E0B14627E003EB8A0B40
:10B23000BBF802301A050ED413F4805F1DBF964A86
:10B240009BF801101268954A954B14BF52F82120C3
:10B25000126843F82A20BBF80230D80516D49905A5
:10B260000AD5904B1B7813F0040F0CBF8E4A8F4AFF
:10B270008B4B126843F82A2009F10109207B5FFA01
:10B2800089FA8B4982450B68D0D326E0894A50461B
:10B29000594605F00DFF884B1B885A0603D55046CA
:10B2A0005946864A16E0580703D550465946844AFF
:10B2B00010E0190703D550465946824A0AE09A071A
:10B2C00003D550465946804A04E0DB07D4D55046A2
:10B2D00059467E4A05F0ECFECEE7DFF808E200931F
:10B2E000BEF906307822A3F57A7353434FF47A728D
:10B2F00093FBF2F3F34603F22B13019300225FFA60
:10B3000082FE864517D2009B03EB820EBEF802E058
:10B310001EF4806F0DD040F2671ADFF88491019B14
:10B3200039F822E09E449EFBFAFC0AFB1CEE29F849
:10B3300022E00132E3E74DB308F5C333A033636085
:10B34000637B544A13BB9373614B1B6813F0020F6A
:10B350000AD0DFF894E19EF800E0BEF1000F03D0C0
:10B360004FF0010E82F80EE0DA0506D5594BDB7876
:10B370001BB1A37B43F00203A3734A4B1B7813F06A
:10B38000050F02BFA37B43F00403A37394F80EE000
:10B39000BEF1000F03D13F4B5B7B002B4FD094F8E5
:10B3A0000DC01CF0010FACF10C031DD1BCF1030F5B
:10B3B00007D8DFF8E8901EF0040F3B4A08BF4A4662
:10B3C00000E0364AACF1040CBCF1070F05D8DFF8F9
:10B3D0001CC11EF0010F18BF6246DBB2032B0ED852
:10B3E0001EF0020F3C4B06E0DBB2032B06D82F4BBE
:10B3F0002A4A1EF0020F18BF1A4600E0274A4FF0F3
:10B40000000C5FFA8CF383420DD20B6803EB8C03C4
:10B410005B881B0642BFD2F80090214B43F82C906A
:10B420000CF1010CEDE785B1BEF1000F08D0637B94
:10B43000184A0133DBB2142B06D1002304E025B1F6
:10B44000637B002BF3D100E05373002E52D0234ACC
:10B450003223B2F90250B2F90020002DB8BF6D427C
:10B46000002AB8BF524295FBF3F592FBF3F2EDB21E
:10B47000D3B2AB4238BF2B46194A13B192FBF3F358
:10B4800000E0134643442360E37B024A83BB01236D
:10B490002FE000BF902000200C2E0020A4B6010851
:10B4A000820D0020C933002058A7010848A70108D1
:10B4B000A81900209C9E0108A4190020A29E010842
:10B4C000A89E0108AE9E0108B49E0108BA9E01081C
:10B4D0007C310020D424002060A70108E010002067
:10B4E000400D0300B83100202C19002068A7010886
:10B4F0000023D3738F4D904B2D78E27BADB9002F95
:10B5000000F00F818D4B267B1A788D4B02F00402E0
:10B5100093F800C08B4BD2B2D3F800E00B68002147
:10B52000894D03EB86060F46B5E01AB9874A1A61C2
:10B53000002508E0864AFAE70A68AB00D618768844
:10B54000760604D40135EBB28342F5D3D7E7814EBA
:10B55000B6F90060192E25DD12F803E094F814C046
:10B560000EF00F09E14526690CDCDFF8CCC19CF830
:10B5700015C0BCEB1E1FDEBFD6F800C0DFF8D8E157
:10B5800043F80EC012F803E094F816C00EF00F094D
:10B59000E14533DBDFF8A0C19CF815C0BCEB1E1FF2
:10B5A0002CDC26E0193629DA12F803E094F814C0EE
:10B5B0000EF00F09E14526690CDCDFF87CC19CF830
:10B5C00017C0BCEB1E1FA2BFD6F800C0DFF888E191
:10B5D00043F80EC012F803E094F816C00EF00F09FD
:10B5E000E1450BDBDFF850C19CF817C0BCEB1E1F18
:10B5F00004DBD6F800E0584E43F806E0554EB6F9A5
:10B600000260192E1BDD12F803C094F814E00CF050
:10B610000F09F14526690CDCDFF81C9199F81590AB
:10B62000B9EB1C1FDEBFD6F80090DFF82CC143F841
:10B630000C90D25C02F00F0CF4451EDD82E7193647
:10B6400080DA12F803C094F816E00CF00F09F14507
:10B6500026690CDBDFF8E09099F81590B9EB1C1F18
:10B66000DEBFD6F80090DFF8F0C043F80C90D25C53
:10B6700002F00F0CF445FFF665AF94F817E0BEEB4F
:10B68000121FA2BF3668344A9E505BE758880005F7
:10B6900004D404330435B342F8D122E04AB101EBBB
:10B6A0000C0A06209AFBF0F900FB19A001280DDC1A
:10B6B00001E057B9012793F801900EEB89003EF89D
:10B6C00029A090F80290C07803E017460020814638
:10B6D0008246013125F802AC85F800906870C9B245
:10B6E000D7E7174A1378013B13F0FF0308BF06237F
:10B6F0001370124B1B785B0741BFBBF906304FF448
:10B700007A72A3F57A7303EBC30348BF93FBF2F39A
:10B71000124A46BF0133DBB2012392FBF3F34344E9
:10B72000A36003B0BDE8F04F03F08ABB03B0BDE8EF
:10B73000F08F00BF3B0E002090200020C933002076
:10B74000200000200C2E0020840D002064A701089A
:10B75000A4B60108E0100020820D0020400D030077
:10B7600010B50446B0F9000006F0CBFCB4F90200B5
:10B7700006F0C7FCB4F90400BDE8104006F0C1BCF7
:10B7800010B50446006806F0BCFC606806F0B9FC21
:10B79000A068BDE8104006F0B4BC2DE9F74F0120C9
:10B7A00006F07CFD002480B3012C2ED84FF04C0A0B
:10B7B0000AFB04F7DFF85C8008EB070B0BF1480687
:10B7C000B57815B10134E4B2EDE790F9003090F8A6
:10B7D00004E018460E4B03228DE8240001212A467E
:10B7E00053F82E30FCF74CFA814650B158462946A2
:10B7F00052460CF0B4F801231C4448F80790B3708B
:10B80000E4B2012006F030FDCDE703B0BDE8F08FD3
:10B81000C09E0108A820002000212A2210B511484E
:10B820000CF09DF8104B0022194610480424105CBF
:10B83000013283F8F401052083F8F94182424FF088
:10B84000000483F8F80183F8FB4183F8FA0103F15F
:10B850000803EAD10123A1F8F631522381F8F2312D
:10B8600010BD00BFDA120020E8100020CDBD010895
:10B8700070B50646441E14F8011F89B1094D2846CB
:10B880000CF0A3F80028F6D005F1080398423FBF5A
:10B89000054B401BC018A31B38BF80F88831EAE76E
:10B8A00070BD00BF52D30108E810002007B51C4B43
:10B8B00003F19C02C3F898201A4A92F890215AB1D9
:10B8C000012A14D1032183F89E10072183F8A020B8
:10B8D00083F89F100C2208E0022183F89E100321B8
:10B8E00083F8A02083F89F10072283F89C200E4A3B
:10B8F0000E4B40201A6006F0D1FC70B101220023EB
:10B9000090F9000040218DE80C00094A4FF4E13322
:10B91000FCF7B6F9003018BF012003B05DF804FB56
:10B92000A8200020E810002031C3000824000020D7
:10B93000BDC400082DE9F04FB84C8BB005468946D0
:10B94000164600210C2204F1A4009B460CF007F8D7
:10B950000021142204F1B0000CF001F8B04F0023D4
:10B9600084F8C430AF4B97F800A003F11802BAF185
:10B97000010F88BF1346C4F8C830FAF7E9FD8046C6
:10B9800090B1A94BA94AC4F8B030A94BC4F8B4305F
:10B99000A84BC4F8BC30A84BC4F8C03001231371C5
:10B9A00084F8C430022339E0192006F07EFD6820B7
:10B9B0001521424607F022FAA8B1A04B9B4AC4F8D1
:10B9C000B0309F4BC4F8B4309E4BC4F8B8309E4B97
:10B9D000C4F8BC30984BC4F8C0300123537184F8CC
:10B9E000C43004231AE0BAF1030F40F0BF83FAF722
:10B9F0006BFD002800F0BA83944B8C4AC4F8B03039
:10BA0000934BC4F8B430934BC4F8BC308A4BC4F8A1
:10BA1000C0300123937184F8C43007238E4900207D
:10BA20000B708E4B00911A689A4642F001021A6020
:10BA30008B4A10709046082D31D8DFE805F036307B
:10BA400036121E21122C2C004FF0000C0AAB03F80A
:10BA500018CD532061460122CDF804C007F08EF9BD
:10BA600038BB704B397803F11802012988BF13469F
:10BA7000C4F8C830FAF76CFD70BB3B78012B73D962
:10BA800000210AAB03F8181D1820012207F076F9EF
:10BA9000002840F088803B78032B00F09480012D33
:10BAA00040F2A880002588F800503B78012BD8D8B8
:10BAB000CAE79DF81030DDF804C0E52BD1D1694B01
:10BAC00084F8CCC0C4F8A430674BC4F8A830042371
:10BAD00088F80030022385E006210A4604AB68207E
:10BAE00007F04CF99DF8151001F001029DF81310B4
:10BAF00001F001014B0043EA82019DF8112002F0A0
:10BB000001030B430AD05BB2012B01D1002302E0F9
:10BB1000022B0FD1012384F8CD3012E00C210DEB64
:10BB200001036820012207F029F99DF80C3013F079
:10BB30000F0303D1032006F02BFD02E0042BE9D113
:10BB4000E4E74A4BC4F8A430494BC4F8A83094F851
:10BB5000CD30002B0CBF6F236E2384F8AC30012353
:10BB600088F8003003233DE000220AAB03F8182DCB
:10BB70001C200D21012207F001F9002880D09DF83A
:10BB800010302A2B02D01A2B7FF47AAF394A84F86E
:10BB9000CE30C4F8A420384A022388F80030C4F814
:10BBA000A82004231EE09DF81030FB2B7FF473AF18
:10BBB000324BC4F8A430324BC4F8A830012388F8C3
:10BBC000003005230EE0FAF77FFC00283FF467AF52
:10BBD0002C4BC4F8A4302C4BC4F8A830012388F8AF
:10BBE00000300823009A5370DAF8003043F0020363
:10BBF000CAF800303B78012B05D107F089FD234BB3
:10BC00004FF400525A61042E00F20A82DFE816F067
:10BC100040001102A3004000B10100BFA820002095
:10BC2000CB330020E09E0108C963000824000020F7
:10BC30003D5E0008395C000890C1793D69640008E8
:10BC4000155F0008E15E0008C15E00088962000817
:10BC5000EF610008D161000850000020DC180020CE
:10BC6000CA330020D15C0008F55F00083D6400087D
:10BC70007F5E000819610008555F0008AD5C000890
:10BC8000AF5F0008295C00082D6200080010014029
:10BC90000A2006F00AFC7720A021012203AB07F05E
:10BCA0006DF8002857D01E210122772007F0A6F852
:10BCB0004FF42F6006F0EEFB0025A5F160014FF078
:10BCC0000008C9B2022204AB77208DF810808DF8ED
:10BCD000118007F053F89DF811309DF8102043EAC9
:10BCE0000222C04B03F1D0016A520235102DE4D17B
:10BCF000B3F8DE10424601F00F0601F47F41A3F8CD
:10BD0000DE104346012522F001002044B0F8D000A7
:10BD1000002818BF002512F0010F03D0C0B2434025
:10BD2000082002E083EA1023FAE713F4004F18BF5B
:10BD300083F4C05301384FEA4303F6D10132102A8D
:10BD4000E1D13143A74AA4F8DE1025B9C3F3033388
:10BD50009E4200F0E68194F8E060A24D002E40F093
:10BD6000FD81DFF8B88207F0D3FC4FF4804A282326
:10BD700003A940468DF80E300093ADF80CA003F0F7
:10BD800052F94FF40052C8F81020974806F04AFCC8
:10BD90000E21022003F032F90822CDF810A004A8E9
:10BDA0004FF0010A8DF815208DF814608DF816A05B
:10BDB00000F034FE009B4FF0030C02A88DF8083011
:10BDC0008DF809C0CDF800C08DF80A608DF80BA081
:10BDD00007F024FC142006F068FB52467720D0219F
:10BDE00003AB06F0CBFF4246002800F0A2809DF88E
:10BDF0000C30DDF800C0552B85F8FB30A5F804C1E8
:10BE000040F09780D121524603AB772006F0B6FF71
:10BE10009DF80C30772003F00F021B0985F8FC20F9
:10BE200085F8FD30162204ABAA2106F0A7FF9DF885
:10BE300010209DF8113043EA0223A5F8E4309DF864
:10BE400012209DF8133043EA0223A5F8E6309DF84E
:10BE500014209DF8153043EA0223A5F8E8309DF838
:10BE600016209DF8173043EA0223A5F8EA309DF822
:10BE700018209DF8193043EA0223A5F8EC309DF80C
:10BE80001A209DF81B3043EA0223A5F8EE309DF8F6
:10BE90001C209DF81D3043EA0223A5F8F0309DF8E0
:10BEA0001E209DF81F3043EA0223A5F8F2309DF8CA
:10BEB00020209DF8213043EA0223A5F8F4309DF8B4
:10BEC00022209DF8233043EA0223A5F8F6309DF89E
:10BED00024209DF8253043EA0223A5F8F83041F2EA
:10BEE0007073A5F8083146F67813A5F80A313F4B70
:10BEF000C5F80C313E4BC5F810313E4BC5F8143136
:10BF00003D4BC5F818313D4BC5F81C3195F8E03074
:10BF10004BB9F9F7C1FE42F6E06006F0BBFAD8F87B
:10BF20000860C6F38036364BDE71012384F8E030BA
:10BF300014E13449D4F820010B6823F480430B60EA
:10BF4000294B2849984209D0D1F82401984207D0BA
:10BF5000D1F82811994209D1022302E0002300E020
:10BF6000012304EB83030021C3F820114FF4005395
:10BF7000536194F82C611B4D002E40F0E980142091
:10BF800006F093FA05F22D137620D021012206F057
:10BF9000F5FE95F82D31582B4BD105F59873882176
:10BFA0001822762006F0EAFE7620F421312206F0EF
:10BFB00025FF012385F82C31134BA5F80861C5F83E
:10BFC0001031124BC5F80C3145F6D813A5F80A31DB
:10BFD0000F4BC5F814310F4BC5F818310E4BC5F88F
:10BFE0001C31B5E0A8200020C5600008995C00085D
:10BFF000095E0008735C0008BD5D00084D5B000829
:10C000002400002000040140495B00084B5B00084D
:10C01000695C0008715D0008E558000800100140E7
:10C02000012E06D0534B544A9E70136843F004030C
:10C030001360514D2B689A0702D5D4F8A430984765
:10C04000002384F84C314FF47A73C4F85031D4F89B
:10C05000B0309847494B97F800A003F11802BAF1A5
:10C06000010F94BF9A4692464F46454E00233370C7
:10C070000FB1022F6ED14FF000080AAB03F8188DF4
:10C080001E200A210122DFF82891C4F854A106F0ED
:10C0900075FE98B19DF81030482B61D1394B0222C2
:10C0A000C9F85831384BC9F85C3103233370314B30
:10C0B000DA702B6843F008032B6001E080464FE004
:10C0C000324B93F854210AB184F8C42093F85521D7
:10C0D0000AB12F490A7093F8563103B133702B68B7
:10C0E0001B0718D564269BFBF6F5284608F01CFABA
:10C0F000074606FB15B000B208F016FA254908F00D
:10C1000067FA0146384608F05BF9234908F060FAFF
:10C11000C4F8600102E00023C4F860314FF0010868
:10C1200024E042F21073A2F80831A2F80A311B4B46
:10C130000326C2F80C311A4BC2F81031194BC2F861
:10C140001431194BC2F81831184BC2F81C3169E789
:10C15000042667E7012FB3D91F4686E7022661E769
:10C16000012FADD9002786F8008084E740460BB048
:10C17000BDE8F08F50000020DC180020109F01085F
:10C18000CC3300208BF0000829ED0008E8100020D7
:10C19000CA3300208988883C000020415F5C000889
:10C1A000615D0008555C0008515D000829570008D2
:10C1B000A82000200120002106F0B8BF174AF0B5E2
:10C1C000164692F86431D2F868E1042B10D85C1C52
:10C1D0000EEBC3039D1CE4B208D09A88D10705D5A5
:10C1E000104203D008E00131052907D12346ECE7CE
:10C1F00086F864310020F0BD9F7800210C2202FBFC
:10C2000001F3064D05F5B67C1CF803209742EAD1F0
:10C210002B4485F86441D3F87001F0BDA8200020BC
:10C220008A6810B50C6A036814430A6923F4FF4353
:10C2300014434A6923F0700314438A691443CA699A
:10C2400014434A6A14438A6A224313430360CB6847
:10C2500043600B6883604B68C36010BD084BDA68AD
:10C26000D10709D4DA68520708D4DB6813F0100F3D
:10C2700014BF03200420704701207047022070473C
:10C280000020024003788B4286BF024B33F8110036
:10C2900000207047502200200022134670B5234929
:10C2A00014180C44247E83EA0423082413F4004F5A
:10C2B0004FEA430318BF83F4815304F1FF3418BFDE
:10C2C00083F0010314F0FF049BB2EFD10132192A6D
:10C2D000E5D100F1190200F11A050A440D44167E59
:10C2E0002A7E02EB062292B29A421ED10F4B93F89D
:10C2F0003950E2B2AA4215D2431C03EB4203DBB22F
:10C30000CA1801330B44127E1B7E03EB02239BB23F
:10C310004FF4AF6253431B1303F5487321F81430F5
:10C320000134E6E7012381F83A3070BD5022002045
:10C3300003788B420BD9074B89001A78064B1944B6
:10C34000C86B02B1400800F5777080B270470020DA
:10C35000704700BF482100205022002007299DBFC0
:10C36000034B03EB8101B1F86C000020704700BF64
:10C3700050220020034B03EB4101B1F88C00C008B0
:10C38000704700BF5022002008B5084B03EB810125
:10C39000D1F8AC0008F0C4F8054908F019F90549CE
:10C3A00008F00EF808F000FB80B208BD5022002013
:10C3B0000000203F00005C44014B33F8110070473F
:10C3C000B8310020024B03EB4101B1F8F400704793
:10C3D00050220020024B03EB4101B1F8F4007047FA
:10C3E000502200200020704770B5054606F036F850
:10C3F000314CD4F80C31C4F80C01C31AB3F5FA5F10
:10C40000C4F8103182BF002384F8143184F8153148
:10C4100094F814312BB9A12D02BF274A012182F8CB
:10C42000151194F81511244A29B1D118EDB2013330
:10C430000D7682F8143194F8145194F81631AB4209
:10C4400039D11D4B93F81731052B02D0062B03D0A1
:10C450002CE00020FFF720FF637E1E2B26D100205A
:10C460000246C1B26B1E994219DA21440B7E0821A3
:10C47000DBB283EA0206F60744BF83F01803C3F376
:10C48000460301F1FF3154BF5B0843F0800311F014
:10C49000FF01C2F34702ECD101301A46E1E7234421
:10C4A0001B7E9A4202D10320FFF7F6FE002384F898
:10C4B000153184F8143170BD5022002010B50446A7
:10C4C00005F0CCFF41F288310E4BE4B2D3F81821CD
:10C4D000C3F81801821A8A42C3F81C2184BF0022C3
:10C4E00083F8202193F8202106490F2A134418BF0E
:10C4F000013283F8214112BF81F82021012381F804
:10C50000313110BD5022002010B5044605F0A6FFC1
:10C5100041F288310E4BD3F83421C3F83401821A2A
:10C520008A42C3F8382184BF002283F83C2193F863
:10C530003C210749142A134418BF013283F83D41B6
:10C5400012BF81F83C21012381F8523110BD00BF98
:10C550005022002038B5044605F080FF274A2749BD
:10C56000D2F85431C2F85401C31AB3F57A6F84BFBC
:10C57000002382F8583192F8583133B9A82C3BD1B6
:10C5800081F85931A1F85A3106E0022B02D181F825
:10C590005C4101E0242B02D8D11881F85D4192F86A
:10C5A0005C1101330231DBB249008B42134D82F83A
:10C5B000583118DAB5F85A31E0B283EA002008237E
:10C5C00010F4004F4FEA400018BF80F4815003F18F
:10C5D000FF3318BF80F0010013F0FF0380B2EFD1EA
:10C5E000A2F85A0138BD01318B4201BF002385F802
:10C5F0005831012385F8593138BD00BF5022002041
:10C6000010B5044605F02AFF40F6AC510F4AD2F8A7
:10C610008431C31A8B42C4BF002382F8883192F858
:10C620008831D11881F8894123B90F2C0DD10749E0
:10C63000C1F884010133DBB2192B044982F8883137
:10C640000CBF0123002381F8A23110BD502200202D
:10C650004FF6FE73026813400360002303604360DB
:10C660008360C360284B984201D1284A27E0284BB9
:10C67000984201D1254A2AE0264B984201D1234A0B
:10C680002DE0254B984201D1204A30E0234B9842BF
:10C6900001D11E4A33E0224B984204D11B4A536811
:10C6A00043F470032EE01F4B984204D1174A53689D
:10C6B00043F0706326E01C4B984204D11B4A536838
:10C6C00043F00F031EE01A4B984204D1174A5368F7
:10C6D00043F0F00316E0174B984204D1134A536815
:10C6E00043F470630EE0144B984204D10F4A536830
:10C6F00043F4704306E0114B984204D10B4A53684F
:10C7000043F4702353607047080002400000024069
:10C710001C00024030000240440002405800024029
:10C720006C00024080000240080402400004024005
:10C730001C040240300402404404024058040240F9
:10C740001F4A10B5536803F00C03042B03D0082BC9
:10C7500004D01C4B14E01C4B1B6811E0536851685B
:10C76000C3F38343C90303F1020301D4174906E06D
:10C77000516811F4003F1449096818BF49084B4338
:10C78000036053681249C3F30313CC5C0368E340AE
:10C7900043605468C4F302240C5D23FA04F48460FB
:10C7A0005468C4F3C2240C5DE340C3605268C2F312
:10C7B00081320A44127CB3FBF2F3036110BD00BF67
:10C7C0000010024000127A002C00002000093D00F9
:10C7D000409F010810B50446FFF740FD012806D12F
:10C7E0001CB1FFF73BFD013CF8E7052010BD002C14
:10C7F00008BF052010BD0A88F0B54B888E88B1F8B7
:10C8000008E0CC88002A3AD1028C43F0010322F0E0
:10C8100001021204120C0284058B078CADB225F0C4
:10C82000F30545EA0E1189B241EA06027A49BFB220
:10C83000884212D001F5006188420ED0B0F1804FDD
:10C840000BD0A1F59831884207D001F5806188426C
:10C8500003D001F58061884202D127F0020701E090
:10C8600027F00A071F4302830784038B23F00C037E
:10C870001B041B0C0383038B9BB21C4344E0042A60
:10C8800044D1028C22F010021204120C0284018B9B
:10C89000058C21F440721205120D42EA0E325E49F7
:10C8A00092B242EA06228842ADB292B212D001F5AB
:10C8B000006188420ED0B0F1804F0BD0A1F59831C5
:10C8C000884207D001F58061884203D001F580617C
:10C8D000884207D125F0200141EA03139BB243F0BF
:10C8E000100304E025F0A00143F010030B43028382
:10C8F0000384038B23F440631B041B0C0383038B0F
:10C900009BB243EA0424A4B20483F0BD082A028C3B
:10C910003ED122F480721204120C0284828B3E4DAE
:10C9200092B222F0F307018C47EA0E1292B2A842AB
:10C9300089B242EA060212D005F50065A8420ED07F
:10C94000B0F1804F0BD0A5F59835A84207D005F57A
:10C950008065A84203D005F58065A84207D121F47F
:10C96000007141EA03239BB243F4807304E021F495
:10C97000206143F480730B4382830384838B23F011
:10C980000C031B041B0C8383838B9BB21C4341E071
:10C9900022F480521204120C0284858B018C25F43F
:10C9A00040752D052D0D45EA062545EA0E321A4D36
:10C9B00089B2A84292B212D005F50065A8420ED005
:10C9C000B0F1804F0BD0A5F59835A84207D005F5FA
:10C9D0008065A84203D005F58065A84207D121F4FF
:10C9E000005141EA03339BB243F4805305E047F61C
:10C9F000FF5543F480530D402B4382830384838B84
:10CA000023F440631B041B0C8383838B9BB243EA98
:10CA10000424A4B28483F0BD002C0140016830B529
:10CA2000CD43154B1C682C401C605A682A405A6044
:10CA3000027902F1804202F58232146821431160CA
:10CA400002689C68D5432C409C60D9682940D96015
:10CA50004179102909BF996801F180431143996018
:10CA600015BF03F58233D96819680A4316BF0A4314
:10CA7000DA601A6030BD00BF00040140054B1A683F
:10CA80005B69034004D0104214BF012000207047AE
:10CA90001846704700040140CA78F0B5D40648BF74
:10CAA0008C780D8802F00F0348BF234315F0FF0F69
:10CAB0001DD0016800240126A64006EA0507B742FA
:10CAC00011D14FEA840E0F2606FA0EF621EA06016E
:10CAD000282A03FA0EF641EA060101D1476102E075
:10CAE000482A08BF07610134082CE4D10160FF2DFA
:10CAF0001FD94168002404F108070126BE4006EA58
:10CB00000507B74211D14FEA840E0F2606FA0EF63A
:10CB100021EA0601282A03FA0EF641EA060101D1AC
:10CB2000476102E0482A08BF07610134082CE2D1BE
:10CB30004160F0BD0F4B1A6842F001021A6059685B
:10CB40000D4A0A405A601A6822F0847222F4803238
:10CB50001A601A6822F480221A605A6822F4FE02CF
:10CB60005A604FF41F029A60044B4FF000629A60C3
:10CB7000704700BF001002400000FFF800ED00E029
:10CB80002DE9F8435B4C0368013AC4F8A43183886B
:10CB90000D46A4F8A831072A42D8DFE802F0040ABB
:10CBA000101822292F35B4F8A4310B80B4F8A6311F
:10CBB00013E0B4F8A6310B80B4F8A43105E0B4F862
:10CBC000A4315B420B80B4F8A6315B4205E0B4F8B7
:10CBD000A6315B420B80B4F8A4316B80B4F8A83165
:10CBE0001DE0B4F8A4315B420B80B4F8A63112E02A
:10CBF000B4F8A6310B80B4F8A4310CE0B4F8A43139
:10CC00000B80B4F8A63105E0B4F8A6315B420B8086
:10CC1000B4F8A4315B426B80B4F8A8315B42AB80BE
:10CC2000354B1B79002B62D1B5F9000007F07CFC75
:10CC30008046B5F9020007F077FC0746B5F9040015
:10CC400007F072FCD4F8AC110646404607F0C0FC71
:10CC5000D4F8B8118146384607F0BAFC0146484678
:10CC600007F0AEFBD4F8C4118146304607F0B0FCA3
:10CC70000146484607F0A4FB0BF07EF8D4F8B0114B
:10CC80002880404607F0A4FCD4F8BC118146384601
:10CC900007F09EFC0146484607F092FBD4F8C81105
:10CCA0008146304607F094FC0146484607F088FB71
:10CCB0000BF062F8D4F8B4116880404607F088FCA5
:10CCC000D4F8C0118046384607F082FC0146404641
:10CCD00007F076FBD4F8CC110746304607F078FC15
:10CCE0000146384607F06CFB0BF046F8A880BDE81B
:10CCF000F88300BF502200202C00002038B50F4BD5
:10CD00001B689C890E4B186880F31000201A07F0EE
:10CD10000BFC0C4907F05CFC0546204607F004FCC0
:10CD20000146284607F008FD07F018FE6428A8BF52
:10CD3000642020EAE070C0B238BD00BFC8180020EF
:10CD4000D81800200000C84244F6FB71084B1A684E
:10CD5000137803EB431300FB03135078C0EB003050
:10CD6000B3FBF0F39078B3FBF0F080B2704700BFF4
:10CD7000C818002008B50A480A2290F8D13100EB03
:10CD80004303B3F8E01100F5F87089B220F8081CED
:10CD900005F06CFC80B2FFF7D7FF024B188008BD8E
:10CDA00050220020CC180020114BD3F8783203EB2E
:10CDB0004002117E11B1022910D00BE0022805D9E2
:10CDC000032807D10B4A1268D20401D5D8897047CD
:10CDD000988A7047084B33F810007047507E00EB7C
:10CDE000800000EB800000F2EE2080B2704700BFB0
:10CDF000502200207C310020B831002008B505F019
:10CE00002DFB074B022283F88022064AC3F87C02DE
:10CE10001268C3F88C22012283F8A52208BD00BF46
:10CE200050220020A031002008B505F017FB084B68
:10CE3000022283F88022D3F88C2200F5B71000F587
:10CE4000587002F2DC52C3F87C02C3F88C2208BD91
:10CE50005022002042F20102034B1B681A420CBF11
:10CE600001200020704700BF7C3100200F4B10B51F
:10CE700093F8A8221C46012A0CD007D3022A0CD111
:10CE80000B4AD36883F00803D36006E0084B0822FE
:10CE90001A6102E0064B08225A6105F0DFFA00F53C
:10CEA000F42000F59070C4F8AC0210BD50220020B0
:10CEB000000C0140026D70B515880446ADB2A9069C
:10CEC00013D5036B8BB9C36A1BB1908880B29847A6
:10CED0000BE0E169928840694E1CD2B2E66142548F
:10CEE000E169E268914228BFE3612B0613D5636ACA
:10CEF000A26A9A42236D0AD0511CA069A162825C89
:10CF00009A802369994206D30023A36270BDDA6830
:10CF100022F08002DA6070BD026B0346C16810B572
:10CF2000406942B11A6C8C1A013A08BF0A46005D8A
:10CF30001A64C0B210BD1A6A805C01328A4228BFEE
:10CF40000022C0B21A6210BD436B13B190F84400C6
:10CF50007047836A406A1B1A584258417047036BF6
:10CF600013B15B68016C01E0C369016A8B423CBF8D
:10CF7000C2689B18581AC0B27047836A8169426BB5
:10CF80001944D160416A994297BF0169CB1ACB1A03
:10CF9000536096BF0023536083624FF0000380F814
:10CFA0004430136888BF816243F001031360704707
:10CFB000436A8269D154436A02690133934228BFAC
:10CFC00000234362436B1BB11B68DB0705D4D4E726
:10CFD000026DD36843F08003D36070474171FCF762
:10CFE000F3BC8160FCF7F0BC2DE9F04105460E462C
:10CFF000078A83899BB21F40002F37D0B7FA87F288
:10D000004FF00043D340DB4399B21F40A2F11B0312
:10D010002982042BF0D8DFE803F0221F1C1903003B
:10D02000746A24B1013C0023A4B2736201E0AC8DA8
:10D03000A4B2D6F82080B8F1000FDDD0D8F80030C7
:10D04000404621469847D8F80480F4E73068A98E16
:10D0500008E07068298F05E0B068A98F02E0F068E9
:10D06000B5F84010036889B29847C5E7BDE8F0817C
:10D07000254B10B55A43254B254C1B680139B3FB92
:10D08000F2F20388013AA04289B292B29BB212D066
:10D0900004F50064A0420ED0B0F1804F0BD0A4F58F
:10D0A0009834A04207D004F58064A04203D004F570
:10D0B0008064A04202D123F070039BB2154CA042C1
:10D0C00006D004F58064A0421CBF23F440739BB2D9
:10D0D00003800F4B8185984202850FD003F50063D2
:10D0E00098420BD003F54063984207D003F5806364
:10D0F000984203D003F58063984201D10023038650
:10D100000123838210BD00BF40420F005400002065
:10D11000002C01400010004073B505460068FFF781
:10D12000A7FF2A680124138800269BB243F001035D
:10D130001380EB7A01A88DF804308DF805408DF846
:10D1400006608DF8074006F069FAEB7A1B2B0BD1CD
:10D15000192301A88DF804308DF805408DF806607C
:10D160008DF8074006F05AFA02B070BD0C4B800AE9
:10D1700098420CD004D8B0F5801F0CD10120704724
:10D18000084B984205D04933984206D003E002206C
:10D19000704703207047FE2070470020704700BF93
:10D1A00001001000020010002DE9F8430468074652
:10D1B000204688469146FFF7D9FF03284BD8BA7A14
:10D1C0009108B8F1000F06D1A589AEB202258D40B5
:10D1D00026EA0505A5810A2303FB00131F4A42F82E
:10D1E0002380043342F82390B8F1000F07D0BD7AB2
:10D1F000A189AD080223AB400B439BB2A381282336
:10D20000434303F120011144EFF31286502585F3C7
:10D21000128803F10C051C331544134455F8047FA0
:10D2200017B10F60296804319D42F7D100230B60CC
:10D23000F3B283F31188282303FB0020036A23B190
:10D24000A3899BB243F0010304E0A38923F0010307
:10D250001B041B0CA381BDE8F88300BFFC2F00203A
:10D26000004827E600250020004823E6542500203A
:10D2700000481FE6A82500200B4B4FF400525A60CF
:10D280004FF6FE730948D0F8DC2011680B4013609C
:10D29000D0F8CC20D0F8D0309A4201D0A8306CE63B
:10D2A000012380F8EC307047000002400025002088
:10D2B0002DE9F0431D46A64B8DB09842884617468F
:10D2C0009DF850605CD1A34BA34AA449C3F8A820A1
:10D2D00003F1FC02C3F8BC2003F5FE72C3F8C020C2
:10D2E0004FF48072C3F8B420C3F8B8209C4AC3F846
:10D2F000B070C3F8D820A2F54842543AC3F8F420DD
:10D30000C3F8F020C3F8F800C3F8DC10954B9A6915
:10D3100042F480429A615A6942F001025A61022342
:10D320008DF803304FF40073ADF80030330701D5AA
:10D330001C230FE0AC0706D518238B4869468DF8EF
:10D34000023001F070FEE8070AD54FF48063ADF8B3
:10D3500000304823844869468DF8023001F063FEAE
:10D360000E238DF804300022012301A88DF805302A
:10D370008DF806208DF807307C4C06F04FF9A1E0BF
:10D380007B4B98424ED1734B734ADF655A654FF41D
:10D3900080721A665A6603F53F729A6603F57F72C9
:10D3A000DA66744AC3F8A400C3F89C20C3F8A0202E
:10D3B0006C4B3107DA6942F40032DA615A6942F0A3
:10D3C00001025A614FF002038DF803304FF004035D
:10D3D000ADF8003001D51C230EE0AA0706D51823AE
:10D3E000614869468DF8023001F01DFEEB0709D552
:10D3F0000823ADF8003048235B4869468DF80230B9
:10D4000001F011FE26238DF804300022012301A82B
:10D410008DF805308DF806208DF80730564C06F053
:10D42000FDF84FE0554B984240F0ED80494B4A4A99
:10D430009F601A6003F2FC425A6103F2FC529A6147
:10D440004FF48072DA601A614D4A18659A64DA64A2
:10D45000444B3407DA6942F48022DA619A6942F077
:10D4600008029A614FF002038DF803304FF4806395
:10D47000ADF8003001D51C230FE0A80706D518230E
:10D48000404869468DF8023001F0CDFDE9070AD524
:10D490004FF40063ADF8003048233A4869468DF8F0
:10D4A000023001F0C0FD27238DF804300022012353
:10D4B00001A88DF805308DF806208DF8073006F0AC
:10D4C000ADF8244C4FF00009012384F84430C4F82F
:10D4D0002090C4F81C90C4F82890C4F82490C4F894
:10D4E0002C806571A760A6712046FCF76DFAEA07EB
:10D4F00052D5206B002847D0E36CCDF80C900193F7
:10D500004FF480530A9380230693E368CDF8149078
:10D510000493202309936369CDF81C900293CDF8FE
:10D520002090CDF82C90FFF793F801A9206BFEF71F
:10D5300077FE226B216D136843F0010313608B8A21
:10D540009BB243F040038B8253689BB2236423E079
:10D550000038014000250020549F0108440002408B
:10D56000580002400010024000080140A825002099
:10D57000004400400444004054250020004800407E
:10D5800004480040000C01404FF6DF72236D1A8002
:10D59000DA6842F02002DA60AB072CD5606B28B362
:10D5A000A36C002501934FF480530A9380230693C4
:10D5B0002369029504931023039305950795089515
:10D5C00009950B95FFF744F8606B01A9FEF728FE5B
:10D5D000636B1A6842F002021A60226D5D605D6042
:10D5E000938A9BB243F08003938204E0226DD36858
:10D5F00043F08003D360226D204693899BB243F4AD
:10D600000053938100E000200DB0BDE8F08300BF1F
:10D6100010B506F089FF0021044607F095F908B11E
:10D62000204601E004F10040054907F085F805496E
:10D6300006F0CEFFFBF7D0FC034B186010BD00BF17
:10D640008096184B35FA8E3C40000020F8B59C4B74
:10D6500004461B68187818B1012800F06A819AE224
:10D66000242C984D0CD006D80A2C00F0D9800D2C13
:10D6700000F0D68048E12A2C06D02C2C04D043E1BF
:10D6800028706870A87050E18F4B69782F7800205F
:10D690008C4A58542FBB1978D770472921D1597813
:10D6A00050291ED19978472907D1D978472904D123
:10D6B0001979412901D10121D1709978824A5229E1
:10D6C00003D1D1784D2900F0688299787E4A4729A4
:10D6D00007D1D178532904D11279562A04BF0322E5
:10D6E000EA70EA78774E022A39D0032A4CD0012A10
:10D6F00040F08580BA1E072A00F28180DFE802F040
:10D7000004080F131A257F2A06F090F9686076E066
:10D710001B78532B73D16B685B426B606FE006F034
:10D7200085F9A8606BE01B78572B68D1AB685B422A
:10D73000AB6064E01B78302B644B1A788CBF42F0EE
:10D74000020222F002021A7059E0002006F0CEF91F
:10D75000287354E0002006F0C9F9E8814FE0072F54
:10D7600006D0082F4BD1012006F0C0F9708246E0A8
:10D77000012006F0BBF941F2184358434FF47A7385
:10D78000B0FBF3F030823AE0022F07D0032F0AD12A
:10D79000002006F0ABF94E4B187030E0002006F088
:10D7A000A5F930752BE02AD93A1F9210337D01324A
:10D7B000D2B2013B02EB8303DBB2102B1FD8F91E60
:10D7C000C2F1010201EB8202D2B2012A0BD0042A7B
:10D7D00011D100205E1E06F089F93E4B00229855BB
:10D7E0003D4B9A5507E03D4A5E1E0020935506F0DA
:10D7F0007DF93B4B98553B4A136801331360314B1D
:10D800002A2C18BF9A7807F101074FF000000CBFCF
:10D81000012254402F7068700CBF5A759C7084E0D0
:10D82000687D002848D0304B13F8012D2F495A70DD
:10D830008B42F9D1244A234C13785278402B85BF70
:10D84000373B1B011B01DBB298BF03F0F003402AFA
:10D850008CBF373A303AD2B21344AA78DBB29A423C
:10D8600027D121230B702249E0780B68012803F1AE
:10D8700001031E4A0B600AD002281CD172231370C8
:10D88000228A1C4B1A80628A1B4B1A8013E0672382
:10D8900013700E4B1B789F070ED5184B62681A60E9
:10D8A000A2685A60227B164B1A70E289154B1A80C7
:10D8B00002E03F230B70002000236B7535E000BFB2
:10D8C0003C070020FC2B0020A8310020E01800209D
:10D8D0005C1000208D1000207D1000205D100020C5
:10D8E0006D100020982D0020600200204C020020C6
:10D8F000A42D0020E218002044100020E818002089
:10D90000E6180020E41800206B78687D0E2B9FBF7E
:10D91000A54A591C5170A54A98BFD454A24A18B9B7
:10D9200093785C40947000E00020003018BF012024
:10D93000F8BD9D4B0022997D082900F22C81DFE87B
:10D9400001F0050B0F15202B475D6700B52C40F04B
:10D950002281DA75012239E0622C08BF022235E00B
:10D9600003229A751C765C769C7614E104229A75E3
:10D970005A7E997E2244D2B25A760A449A76DC764E
:10D9800009E105229A755A7E997E2244D2B25A76CE
:10D990000A449A769C83FEE006229A755A7E997E06
:10D9A0002244D2B25A760A449A769A8B02EB042425
:10D9B000A4B2B4F5AC7F82BF7B4A0121D1750022AD
:10D9C0009C83DA83002C40F0E68007229A75E2E01F
:10D9D0005A7E997E2244D2B25A760A449A76DA8BDB
:10D9E000B2F5AC7F3EBF7049891881F82040013202
:10D9F000998B92B29142DA83E7D9CCE008229A75EA
:10DA00005B7EA34200F0C780674B0122DA750DE010
:10DA1000674D9A7515F8012D6A70664A9542F9D1DD
:10DA2000997E614AA14206D03F232B70624A536817
:10DA300001335360AFE06148016801310160D07D7E
:10DA400010B13E232B70A6E021212970D17E06293A
:10DA500041D004D8022907D0032923D0F8BD1229C8
:10DA600059D0302967D0F8BD5021546A29705449E3
:10DA70004C60946A0C60116B4FF47A7491FBF4F172
:10DA8000504C218092F878114F4A19B1117841F029
:10DA9000020102E0117821F002011170012283F8E5
:10DAA000792169E05321297092F82510CE0705D518
:10DAB00092F82420D51E6A426A4100E0024602F034
:10DAC000010183F87811002A56D13F490A7822F0E3
:10DAD00002020A7050E04F21297092F82B10CC07F7
:10DAE00005D592F82A20D11E4A424A4100E002465A
:10DAF00002F0010183F8781122B933490A7822F043
:10DB000002020A7093F84F10304A1170B3F84C10AB
:10DB10002F4A118030E05621546B29702D490C801A
:10DB200042F21074916B91FBF4F12B4C2180012196
:10DB300082F87A1120E04921297092F82410274AAE
:10DB4000102988BF10211170254914780022A242A3
:10DB50000ED20E7A234D56554E7A234D5655CE7A17
:10DB6000224D565511F80C6F214D56550132EEE7F6
:10DB700020490A6801320A6093F879310A4A002B79
:10DB80003AD092F87A31BBB3002182F8791182F849
:10DB90007A111846F8BD0020F8BD1279432A7FF4A7
:10DBA00094AD0222EA7090E5FC2B0020A831002001
:10DBB000600200204C0200201C070020A42D002041
:10DBC000E8180020E4180020E0180020E6180020E3
:10DBD0004A000020E2180020441000205C100020C1
:10DBE0001C2C00205D1000206D1000207D100020F6
:10DBF0008D100020982D0020F8BD0449044B0968C1
:10DC0000002218705A6199611A777047A03100207C
:10DC10001C070020F8B5101A0D461F4606F084FCBC
:10DC20000446781B06F080FC174B079E196806F027
:10DC3000CFFC21460546204606F0CAFC2946074689
:10DC4000284606F0C5FC0146384606F0B9FB0AF046
:10DC5000D1FA0E4906F0BCFC06F0A6FE069B29464A
:10DC6000186004F10040FBF7C4F8094906F0B0FC65
:10DC7000084906F0A5FB06F071FE0028BCBF00F5C0
:10DC80000C40A0303060F8BD400000202C7D8E3F5D
:10DC9000A00CB34500A00C4644F25063984203DD4B
:10DCA000A0F50C40A0387047034B9842BCBF00F56C
:10DCB0000C40A030704700BFB0B9FFFFF7B5036854
:10DCC000174C184D23600B68174E63600068FFF710
:10DCD0009FFC95E80300154B0196009394E80C0017
:10DCE000FFF798FF3668124B60681E606B68114F33
:10DCF000C01A06F019FC104B196806F069FC06F012
:10DD00002DFE2A68236878609B1A3B600B4B1E60CF
:10DD10000B4B1B68DA880B4B1A8003B0F0BD00BFB9
:10DD2000A82E0020E8180020B42E0020B02E0020DD
:10DD3000F02E0020B82E002040000020E82E002009
:10DD4000100F0020E42E002070B50446407906F044
:10DD5000E7FB1E4906F0F0FC1D4D1E4E2860E07BDF
:10DD600006F0DEFB194906F0E7FCEE606860A0797A
:10DD700006F0D6FB184906F0DFFC184D2860207C21
:10DD800006F0CEFB114906F0D7FC6860A07E06F0D5
:10DD9000C7FB134906F0D0FCEE60A860E07906F0FE
:10DDA000BFFB0D4906F0C8FC0E4D2860607C06F0F4
:10DDB000B7FB064906F0C0FC6860E07E06F0B0FBE9
:10DDC000074906F0B9FCEE60A86070BD0000C842CB
:10DDD000C02E00200000FA4400002041D02E002078
:10DDE00000007A44F42E002010B50C4C23789B07D9
:10DDF00013D50B4B1B78042B0FD90A4A0A4B10681A
:10DE0000526818605A60FFF703FC084B1A88084BE9
:10DE10001A80237843F00103237010BDE01800201E
:10DE2000E6180020E818002048100020D810002034
:10DE3000042F0020164B13B51B681B0325D5154B6B
:10DE4000154C1B7815498DF80030154B20681B7850
:10DE50008DF8013006F0BCFB06F0A6FD11498DF8E7
:10DE60000200606806F0B4FB06F09EFD8DF803002A
:10DE7000A06806F099FD0C4B8DF804001B780A2071
:10DE800069468DF80530FAF7EBF802B010BD00BF17
:10DE90007C3100206E3100209031002000002041B4
:10DEA0008C31002000007A4472310020054A13783A
:10DEB00083F001031370044A00231360034A1360C4
:10DEC000B8E700BF72310020883100208431002083
:10DED000094A137818441346C0B210F0800F18BFD7
:10DEE00080381070054A19781378994201BF0023D1
:10DEF0001370014A13707047092F0020082F00206B
:10DF000010B50A4B0A4A1B7842609C18094A046003
:10DF100012789A4225BFD31A0B60C3F18003002305
:10DF20002EBF4B600B604A6010BD00BF092F002060
:10DF30000A2F0020082F00201FB5684602A9FFF70E
:10DF4000DFFF044B02981B6803440398184405B094
:10DF50005DF804FBB00500202DE9F04F89B0019376
:10DF600000238246994602910392039A934205DA6E
:10DF7000029A52F8232001339144F6E7019B4D4663
:10DF8000002B56D101F088F9002852D101987DE08C
:10DF90000222404E8DF81C201A0C4FF480578DF849
:10DFA0001D2006201A0A8DF81E208DF81F3001F062
:10DFB00097F97761062005F085FB374B0122376121
:10DFC000D0461A7077612646002007A9042205F082
:10DFD00043FB029F4FF0000B039B9B451EDABC46A0
:10DFE00057F8042B4FEA8B03002A48D0B24236D3AD
:10DFF00032465AF803100020CDF814C0049305F0FF
:10E000002BFB049BDDF814C05AF8032032444AF875
:10E010000320DCF800309E1BCCF800601D4B4FF451
:10E0200080521A611D4A2D1B13681C44019B146009
:10E0300053B34DB3194B1B68DCB22A19B2F5807F7C
:10E04000174A88BFC4F58074D26898BF2C469342A3
:10E050009ED3144A00231370134A137014E0002057
:10E06000D8F8001005F0F8FA57F8043CD8F800206A
:10E07000F61A1344C8F80030002347F8043C0BF1AB
:10E08000010B08F10408A7E7C5EB090009B0BDE8DA
:10E09000F08F00BF000C0140AD050020B00500204E
:10E0A0000C000020082F0020092F002030B50B4C59
:10E0B0000B4D22782B7885B09A420CD0684602A985
:10E0C000FFF71EFF0123684602A90222FFF744FF63
:10E0D00000232B70237005B030BD00BF092F002036
:10E0E000082F002030B50E4D0E4C2A78237885B0CD
:10E0F0009A4211D0684602A9FFF702FF002302A945
:10E1000002226846FFF728FFFFF7E2FE20782B780F
:10E110001B1A5842584100E0012005B030BD00BF35
:10E12000092F0020082F002038B50E4C4FF48055E1
:10E1300045F2082001F0D4F86561062005F0C2FA26
:10E14000094B01222561C7201A70656105F0BAFAF2
:10E15000064A002325611370054A1370054A1360AF
:10E1600038BD00BF000C0140AD050020082F002085
:10E17000092F0020B005002001480249FEF734BFF6
:10E18000000800407430002001480249FEF72CBF0F
:10E19000000400404C3000204FF080400149FEF761
:10E1A00023BF00BF2430002001480249FEF71CBFF6
:10E1B000002C0140FC2F002001480249FEF714BF4B
:10E1C000002C0140FC2F00200028114AB8BF40421B
:10E1D00090FBF2F330B50F4C3C2504FB0300684381
:10E1E0000D4D90FBF2F22D682D7B25B903EB8303D7
:10E1F00003EB830301E0C3EB031302EB830304FB94
:10E2000002020B804FF47A7392FBF3F24A8030BD26
:10E2100080969800806967FFD0180020022803D0FC
:10E22000431E584258417047064B1B681B7823B168
:10E23000054B1868C0F3C0407047044B1878C0F312
:10E24000800070478C050020DC0F0020C9330020BF
:10E2500010B50A4C5E280146206805D15D2104F006
:10E2600002FA20683E2105E05D2903D104F0FBF9A4
:10E2700020683D21BDE8104004F0F5B9782D00205C
:10E28000A0F17D03012B70B504460D460A4E05D85A
:10E2900030687D2104F0E7F984F0200430682146DD
:10E2A00004F0E1F935B12B881C4404EB142404F08C
:10E2B000FF042C8070BD00BF9419002010B5054CE0
:10E2C000206804F0CDF918B1206804F0C6F9F6E72B
:10E2D00010BD00BF6419002010B50446C0B2FFF79E
:10E2E000B7FFC4F30720BDE81040B1E7024B5E2141
:10E2F000186804F0B8B900BF782D002038B505467D
:10E30000054C5E21206804F0AEF920682946BDE87E
:10E31000384004F0A8B900BF782D002013B504469A
:10E3200001A90068FFF750FF1320FFF7E7FFBDF9D1
:10E330000400FFF7D1FF1B20FFF7E0FFBDF9060047
:10E34000FFF7CAFF2320FFF7D9FF2368002BB4BFD4
:10E3500053204E20FFF7C0FF01A96068FFF734FF8C
:10E360001220FFF7CBFFBDF90400FFF7B5FF1A201D
:10E37000FFF7C4FFBDF90600FFF7AEFF2220FFF74D
:10E38000BDFF6368002BB4BF57204520FFF7A4FFF3
:10E3900002B010BD674B73B51878FFF73FFF664DAD
:10E3A00004462B78834220D0C8B1644B1B68E3B18C
:10E3B00093F9000002230093614B04211B680022A3
:10E3C0005B78003318BF012301934FF41653F9F71C
:10E3D00057FC5C4B186040B101232B7005E0594E8F
:10E3E0003068F9F739FC34602C70574B574D18786A
:10E3F000FFF714FF2B780446834218D088B1544BA2
:10E400001B68A3B10022012493F9000008214FF4F6
:10E41000964300940192F9F733FC4E4B186028B9EB
:10E4200005E04C4E3068F9F717FC34602C704A4B0D
:10E430004A4D1878FFF7F2FE2B78044683422E46A9
:10E4400043D0002838D0464B1A68002A3DD0D379F3
:10E4500092F90000002B4FF00202424C08BF022349
:10E460000092002254F8233001921021F9F708FCA1
:10E470003D4B0546186040B33C4C94F84A30022BA3
:10E480000BD094F89620022A01D14C3405E023B138
:10E49000002A04F14C0418BF0024354B1C6044B121
:10E4A000204600214C2209F05AFA0223256084F804
:10E4B0004A300123337008E02B4E306804F0E2FD4F
:10E4C0003068F9F7C9FB34602C702A4B2A4D187854
:10E4D000FFF7A4FE2B780446834229D000B3274BD4
:10E4E0001B682BB3264A93F9000012680323527865
:10E4F0002021002A0CBF08220922009301924FF428
:10E5000061430022F9F7BCFB1E4B186080B11E4A24
:10E51000012313702B701D4B1A681D4B1A6007E006
:10E52000184E3068F9F798FB174B34601C702C704C
:10E5300002B070BD94050020C0100020900500209E
:10E54000D0180020782D002095050020F01800201C
:10E550007419002064190020A00500207A190020F9
:10E560009C050020C09E01087C190020A8200020E6
:10E5700080190020AC05002090190020A80500207B
:10E58000A40500209419002098190020A031002033
:10E590009C190020642928BF6421F8B501FB00F50F
:10E5A000642495FBF4F40646E4B20027FBB2A342D0
:10E5B00004D29F2000F0CFFE0137F7E7B4420BD220
:10E5C000142195FBF1F5C4EB8410663DC4EB80008B
:10E5D0002844C0B200F0BFFE0134E4B2B44201D21C
:10E5E0009A20F7E7F8BD2DE9F74303F037FF924C87
:10E5F0006368C31A002BC0F2628300F5433303F54E
:10E60000A07363608D4B1D78237AC5F38005EB1AE8
:10E6100018BF012325724DB1002B00F05083884BA9
:10E620005A789A7001225A701A702BE0844A2BB1E2
:10E63000D37843F00203D37093785370D67806F002
:10E64000020101F0FF0339B97D498968411A0029A7
:10E6500003DB06F0010300E0012303F00107784922
:10E6600017707BB1F2070DD50A7905230132D2B2BA
:10E67000B2FBF3F303EB8303D31A724ADBB20B71E1
:10E68000D35C4B706E4EDFF8088233787BB3F3783F
:10E6900023F00203F3706C4B0344AE20B36000F030
:10E6A0007EFE08B100F080FE88F80000002800F02F
:10E6B0000683B02000F073FE402000F070FE0020C2
:10E6C00000F06DFE102000F06AFE4FF48067013FFD
:10E6D0000020BFB200F03AFE002FF8D1384600F01B
:10E6E000D2FE7278594B53F8220000F04FFE98F892
:10E6F0000030002B00F0E3827378062B00F2AC822E
:10E70000DFE813F00700AA02180078006501820113
:10E71000E6014F494F4A504B5048FAF726FB01207B
:10E7200000F0B1FE4D4800F031FE022000F0ABFEDB
:10E730004B48A7E14B4F3B689B0735D5DFF8548129
:10E740000A23B8F80010DFF85091B1FBF3F203FB95
:10E75000121399F8001092B29BB200913F484249BF
:10E76000FAF703FBFCF732FD012000F08CFE3B487A
:10E7700000F00CFE3D4B99F800201868B8F8003006
:10E78000067902FB163164234B43C17802208E1BAD
:10E790005643B3FBF6F6F6B200F075FE314615208F
:10E7A000FFF7F8FE032600E001263B681F0540F155
:10E7B00053822F4B2F491F68642397FBF3F209689C
:10E7C00003FB1273009125482B49FAF7CEFAFCF7A8
:10E7D000FDFC304600F057FE204800F0D7FDFEF764
:10E7E0008DFA0746701C00F04EFE15203946FFF7E3
:10E7F000D1FE31E20120214F00F045FE204800F01B
:10E80000C5FD3B68980749D51E4A1448B2F9021065
:10E81000B2F900300091B2F904201B4901921B4A61
:10E82000FAF7A3FAFCF7D2FC022000F02CFE0B480A
:10E8300000F0ACFD032632E0782D0020C933002023
:10E84000CC2D0020D2BD0108404B4C00749F010824
:10E85000D7BD0108E0BD0108DDB60108812D00200B
:10E86000E7BD01087C310020F2BD0108C818002076
:10E87000D4180020D81800200ABE0108DC18002097
:10E880001FBE0108CA10002035BE010844BE0108A1
:10E890003D020020CC1800204800002002263B68E2
:10E8A000D9071AD5794A7A48B2F90210B2F900307C
:10E8B0000091B2F9042077490192774AFAF755FAA4
:10E8C00006F10108FCF782FC304600F0DCFD5FFA3F
:10E8D00088F86F4800F05AFD46463B681A0718D57D
:10E8E0006E4A6B48B2F90210B2F900300091B2F9E9
:10E8F0000420684901926A4AFAF737FA771CFCF754
:10E9000065FC304600F0BFFDFFB2614800F03EFDFF
:10E910003E46644A5F49B2F90030B2F902205C48D1
:10E920000092614A614FB2F90020B9460192604AF3
:10E93000FAF71BFAFCF74AFC304600F0A4FD5448F5
:10E9400000F024FD52493868FAF7AAF8504809F057
:10E950004AF806F101085FFA88F8C1B2092909D816
:10E960004B1CDBB2214420224A720021E218917232
:10E970001946F3E7464FD9F804003944FAF790F8FE
:10E98000FCF724FC404600F07EFD384600F0FEFC1B
:10E990003946D9F80800FAF783F8384609F023F821
:10E9A0000236F6B2C1B2092909D84A1C6318D2B29C
:10E9B000202159720021A31899721146F3E73944B6
:10E9C0000020FAF76DF8FCF701FC304657E000260E
:10E9D000384F3B78B34240F23F810E2E00F03C812D
:10E9E0007008013000F04FFD304605F0A5F83B7887
:10E9F000B34206D9202000F0AEFC701CC0B205F076
:10EA00009BF80236F6B2E3E72B4E2C4996F8B42772
:10EA10001F48FAF7AAF9012000F035FD1C4800F064
:10EA2000B5FC274B27491F7819483A46FAF79DF954
:10EA3000022000F028FD164800F0A8FC0C2303FB80
:10EA40000766214996F8B72796F8B6371048FAF7BF
:10EA50008CF9FCF7BBFB032000F015FD0C4800F01F
:10EA600095FC96F8BC1796F8BA2796F8BB37084875
:10EA700000911649FAF779F9FCF7A8FB042000F099
:10EA800002FD034800F082FCE6E000BFFC0F00201E
:10EA9000812D002035BE010848BE0108021000206B
:10EAA0004ED3010874310020D8100020040E00203D
:10EAB0004CBE010844210020E810002050BE01088F
:10EAC000343100205CBE01086DBE01087EBE010825
:10EAD0007C4B1B681B0640F1BB80236A616A7A4A43
:10EAE0008B421CBF536292F828304FF001011CBFCB
:10EAF000013303F003034FF0000018BF82F8283001
:10EB000000F0CDFC94F82830704A0026D05C00F06C
:10EB100022FC0220012100F0C2FC6D4B3620F35C88
:10EB20000136C3EBC30393FBF0F0C0B2062828BF45
:10EB300006206038C0B200F00EFC102EEDD1654BFF
:10EB400065491B78654813F0020F654B1A7814BFAE
:10EB500059234E23FAF709F9FCF738FB022000F09D
:10EB600092FC5E4800F012FC5E495F4B4E680A68FA
:10EB70005A4892FBF3F25D4996FBF3F3FAF7F5F886
:10EB8000FCF724FB032000F07EFC544800F0FEFB61
:10EB9000574B58491A885148FAF7E7F8FCF702FB37
:10EBA000042000F070FC4D4800F0F0FB524B53493C
:10EBB0001A884A48FAF7D9F8FCF7F4FA04210A202F
:10EBC00000F06DFC454800F0E1FB4D49E26A434826
:10EBD000FAF7CBF84B4EFCF7E5FA052000F053FCB2
:10EBE0003E4800F0D3FB7268B36847493B48FAF7E8
:10EBF000BCF8FCF7D7FA05210A2000F050FC374892
:10EC000000F0C4FB3369F2684049D21A3348FAF77E
:10EC1000ACF8FCF7C7FA062000F035FC2F4800F0EE
:10EC2000B5FBB2683A492D48FAF79FF8FCF7BAFAF3
:10EC300006210A2000F033FC284800F0A7FB3549E4
:10EC40001522264808F0FAFEFCF7ACFA072016E772
:10EC5000F37843F00203F370002D30D12E4B0021E6
:10EC600093F820301220052B97BF2C4A3F259B1884
:10EC70001D7F00F014FC284600F06DFB13200021DE
:10EC800000F00DFC264B1B78002B264B18BF722082
:10EC90001B7808BF2120002B18BF522000F05BFB1F
:10ECA0001420002100F0FBFB94F83050074B585D16
:10ECB000013505F0030500F04EFB84F8305003B039
:10ECC000BDE8F0837C310020782D002090BE010843
:10ECD0008D100020E018002095BE0108812D002035
:10ECE000E6180020E818002080969800A6BE0108CB
:10ECF000E2180020B3BE010844100020BBBE01088A
:10ED0000C2BE01081C070020C9BE0108D2BE01080E
:10ED1000D9BE01084C020020D4240020749F0108B1
:10ED20003B0E0020A00E002037B5044603211E2014
:10ED300006226B4604F022F878BB9DF801309DF85E
:10ED40000000174D43EA002000B205F0EDFB2968F2
:10ED500005F03EFC05F002FE9DF8033020809DF892
:10ED6000020043EA002000B205F0DEFBA96805F0CE
:10ED70002FFC05F0F3FD9DF80530A0809DF8040000
:10ED800043EA002000B205F0CFFB696805F020FCE3
:10ED900005F0E4FD6080012000E0002003B030BDFC
:10EDA0003400002010B5054C23681869FDF766FE95
:10EDB00018B123681A69024B5A6110BDFC2100206A
:10EDC0000004014038B50D4B0D4D99680D4B1A6884
:10EDD0001C465288114203D003F040FB286007E034
:10EDE00003F03CFB2B68984282BFC01A064B1860A8
:10EDF00023685A68054B5A6138BD00BF000C0140BA
:10EE0000AC2D002018070020000000200004014065
:10EE1000084A13689B020BD5074B002119704FF667
:10EE2000FE730649086803400B604FF400135360FB
:10EE3000704700BF00000240C83300206C00024051
:10EE40002DE9F047664D6B686649581C0A788E4676
:10EE500002F0FF060AB10346F6E737466B60687CAE
:10EE6000EB6895F81080AA7C39B2202900F09C80CC
:10EE7000DFF880C10CEB8103DC789B783CF8211033
:10EE8000C3F1FF039BB2002B65D04FF03C0CB1FBEC
:10EE9000FCF9C3F1FF0363431B12B9F1050F5DD801
:10EEA000DFE809F0030B1A293A4AE01A4143B1FBA3
:10EEB000FCF0DAB21044C0B251E0B1FBFCF00CFB44
:10EEC000101189B2DAB2C1F13C01E31A4B43B3FB32
:10EED000FCFC204694442CE0B1FBFCF00CFB101130
:10EEE000E21A89B24A43B2FBFCF25FFA83F8424469
:10EEF000D2B2204632E0B1FBFCF90CFB191189B209
:10EF0000E01AC1F13C014843B0FBFCF05FFA83F822
:10EF10004044C0B2224621E0B1FBFCF80CFB1811C2
:10EF2000D8B289B2E31A01FB03F2B2FBFCFC224621
:10EF300084445FFA8CF412E0B1FBFCF80CFB18116E
:10EF400089B2D8B2C1F13C01E31A4B43B3FBFCF2E6
:10EF50000244D2B203E02246204600E044464FEA93
:10EF6000042C4CEA004C4CEA020C17234FF0010829
:10EF700008FA03F806F1170118EA0C0FA1EB0301D8
:10EF8000DFF8748014BF4FF011094FF0090989B2FE
:10EF900013F1FF3308F80190E8D218360137B6B202
:10EFA000BFB2114BA0465FE7EB6001238EF8003043
:10EFB00040F22A33AA740D4A69810D4985F8108000
:10EFC00068742E81536000238B840B889BB243F0BE
:10EFD00001030B80136843F001031360BDE8F08761
:10EFE000AC2D0020C8330020BC2D00206C00024056
:10EFF00000040040820D00206102002001F00303A4
:10F0000001F0FC0101F1804101F5803110B59B0058
:10F010008C680F229A4024EA02028A608A6898402B
:10F0200002438A6010BDF0B5B1F800E000234EFA4B
:10F0300003F2D50725D58E784FEAD30CF40648BFE6
:10F04000CC7806F00F0203F0070748BF2243BF0049
:10F0500050F82C500F24BC4025EA0404BA40224347
:10F06000282E40F82C2005D1C46801229A4024EAB9
:10F07000020205E0482E04D1C46801229A402243CE
:10F08000C2600133102BD2D1F0BD2DE9F0437A4A92
:10F0900087B01368904693B11A681AB177498869A6
:10F0A00002438A619A889868ADF8002002228DF8A0
:10F0B0000320694604228DF80220FFF7B4FF3220B6
:10F0C00003F0F3F9002111221E2003F097FE012125
:10F0D00060221E2003F092FE642003F0E6F9002473
:10F0E00002A8FFF721FE274626460A250221012213
:10F0F0001E2003F083FE322003F0D7F902A8FFF7A9
:10F1000013FEBDF90820BDF90A1014448A42A8BFB5
:10F110000A46BDF90C300F4493421E44A8BF134663
:10F1200013F5805F09DD564A013DD36883F0100373
:10F13000D360DBD14FF0010901E04FF000091E2040
:10F140000021122203F05AFE0A25022101221E206C
:10F1500003F054FE322003F0A8F902A8FFF7E4FD03
:10F16000BDF90820BDF90A10A41A8A42A8BF0A46B0
:10F17000BDF90C307F1A9342A6EB0306A8BF1346D5
:10F1800013F5805F07DD3E4A013DD36883F010032D
:10F19000D360DAD101E04FF00009204605F0C4F950
:10F1A0000146384805F0C8FA374D20F00040286085
:10F1B000384605F0B9F90146324805F0BDFA20F0AD
:10F1C00000406860304605F0AFF901462F4805F071
:10F1D000B3FA20F00040A860002170221E2003F046
:10F1E0000DFE012120221E2003F008FE1E20022118
:10F1F000002203F003FE642003F057F9B9F1000F79
:10F2000004D14FF07E532B606B60AB60D8F80030B8
:10F21000194E1A7B62B31A7D52B3184900258A69C8
:10F22000012442F001028A61187B197DFFF7E6FE96
:10F23000174803F0F7F93368164A1B6904A85361AD
:10F2400004930C238DF815308DF814508DF816406A
:10F25000FDF7E4FB336801A85B7D8DF806508DF85F
:10F26000043003238DF805308DF8074004F0D6F9FB
:10F2700007B0BDE8F08300BFFC2100200010024071
:10F28000000C014000406F463400002001C05E4683
:10F29000A5ED0008000401400F4B73B518781C461B
:10F2A00098B105230D4D8DF800304FF480560023A2
:10F2B0008DF8013001A86E616946022204F0CCF994
:10F2C0002E619DF8050000F0010000F001002070A3
:10F2D00080F0010002B070BDAD050020000C0140BF
:10F2E000064B70B506461C461D68FFF7D5FF18B9DA
:10F2F00023685B1BB342F8D970BD00BFA03100206A
:10F30000F7B503238DF80430030C8DF805308DF824
:10F310000700030A06200F4614468DF80630FFF753
:10F32000DFFF78B1084D4FF4805601A904226E61C9
:10F33000002004F091F938460021224604F08CF9AF
:10F3400020462E6103B0F0BD000C01400246402172
:10F350003C2003F053BD70B500EB8000094CA0F1D8
:10F36000A1059C3825440444074B15F8010F1E786D
:10F370007040FFF7EBFFA542F6D13046BDE8704084
:10F38000E4E700BF989F0108CD33002010B5441E6C
:10F3900014F8010F10B1FFF7DEFFF9E710BD0246C8
:10F3A00080213C2003F02ABD10B5D420FFF7F7FFE1
:10F3B0008020FFF7F4FFA820FFF7F1FF3F20FFF7C1
:10F3C000EEFFD320FFF7EBFF0020FFF7E8FF402020
:10F3D000FFF7E5FF8D20FFF7E2FF1420FFF7DFFFC7
:10F3E000A120FFF7DCFFC820FFF7D9FFDA20FFF7E5
:10F3F000D6FF1220FFF7D3FF8120FFF7D0FFCF20E9
:10F40000FFF7CDFFD920FFF7CAFFF120FFF7C7FFB5
:10F41000DB20FFF7C4FF4020FFF7C1FFA420FFF768
:10F42000BEFFA620FFF7BBFFAF20FFF7B8FFA62067
:10F43000FFF7B5FFAE20FFF7B2FF2020FFF7AFFFC9
:10F440000020FFF7ACFFB020FFF7A9FF4020FFF737
:10F45000A6FF0020FFF7A3FF1020FFF7A0FF4FF447
:10F460008064013C0020A4B2FFF770FF002CF8D1AB
:10F470008120FFF794FFC820FFF791FFAF20FFF72F
:10F480008EFF012010BD08B55038C0B2FFF787FFCE
:10F490000020FFF784FFBDE8084010207FE710B58B
:10F4A00004465039C8B2FFF77AFF04EB440040002D
:10F4B00000F00E00FFF773FF06206043BDE8104028
:10F4C000C0F3031010306AE7012828BF01202DE99E
:10F4D000F04F0646734F142000FB0671724BD1F8B3
:10F4E000A4421E765C61714BD1F8B422DD69B1F89B
:10F4F000AC822A43DA61A288B1F8AEA222F440724B
:10F50000D1F8A852120489B0120C4AEA0809A28064
:10F5100003A9C5F8109002228DF80E002846019329
:10F52000ADF80C908DF80F20FFF77DFD019B009743
:10F530001F464FF0080BAA6818EA020F03D10A20F1
:10F5400002F0A8FFF7E70A20C5F8148002F0A2FF36
:10F55000C5F810800A2002F09DFFBBF1010BEAD133
:10F56000C5F814A00A2002F095FFC5F814800A20FF
:10F5700002F090FFC5F810800A2002F08BFF0222F3
:10F58000C5F810A0284603A98DF80F201C228DF87D
:10F590000E20ADF80C90FFF746FD454A03A89442B3
:10F5A0003A690BBF42F4001242F480023A613A61B8
:10F5B0000BBF3A693A6922F4001222F480023A61E0
:10F5C000A38823F440731B041B0CA38023889BB2E5
:10F5D00043F001032380A588FDF7B2F80599354B68
:10F5E00025F03F05B1FBF3F32D042D0C1D43ADB207
:10F5F000A5802288002522F001021204120C22802C
:10F600002D4A03A8B1FBF2F100298AB208BF0122FA
:10F6100042F400414FF4967253434FF47A7293FBD5
:10F62000F2F301339BB22384A1832388009A9BB217
:10F6300043F001032380238823F4816323F0020332
:10F640001B041B0C23804FF480432381142303FBF2
:10F65000062696F8B13201248DF80C308DF80D5045
:10F660008DF80E508DF80F4003F0D8FF96F8B032A9
:10F670009DF80F208DF80C308DF80D508DF80E5040
:10F680001AB103A803F0CAFF08E05A0903F01F03E8
:10F690009C4002F12003094A42F8234009B0BDE82A
:10F6A000F08F00BF989F0108AC2D00200010024091
:10F6B0000054004040420F00804F120000E100E083
:10F6C00038B500240B4D6059254403F0D1FD69681D
:10F6D00011B10948F9F75EFBA96811B10748F9F7BC
:10F6E00059FB0748103403F0C3FDB4F5F07FE9D1AE
:10F6F00038BD00BF64A2010812BF010818BF01088D
:10F7000031C9010870B50546284608F06CF906466F
:10F7100058B91A4B1A485A791A4BBDE8704003EB96
:10F720008203D3F8DC11F9F735BB28461649324677
:10F7300008F062F960B9154803F09AFD144C54F8CA
:10F74000041F19B11348F9F725FBF8E7124805E043
:10F750000024124B53F8241021B91148BDE8704021
:10F7600003F086BD2846324608F046F901340028E9
:10F77000EFD1024B0B4D5C71C6E700BFE8100020D3
:10F780001EBF010864A201082ABF01082FBF01089B
:10F7900040A4010842BF010831C9010844A401087E
:10F7A000BABC010804BA0108F0B585B0044608F0F7
:10F7B0001AF9082826D1621EE01D1F4912F8013FE0
:10F7C00009681944497801F00301022908BF203B68
:10F7D00082421370F1D1254604F1080715F8016B38
:10F7E0001648314608F0F1F820B12846314608F0B5
:10F7F000ECF810B1F7F7E8FC1CE0BD42EED1204672
:10F80000FCF736F80E4803F033FD00230D4A04A937
:10F810001A4492F888210A440849595C0133082B9C
:10F8200002F80C1CF2D10023074801A98DF80C3016
:10F83000F9F7B0FA05B0F0BD5C00002052D3010822
:10F8400046BF0108E8100020D5C701082A4B2B4C01
:10F850001E6880B52068F8F7DBF93046F8F7D8F96C
:10F86000206841798D0703D441F0020102F0ECFEDB
:10F87000234B08221A61234D10221A612B689A0328
:10F8800041BF06236371E37923F0010344BF43F0D2
:10F890000203E371206802F0E3FE90B1184F0823E1
:10F8A0007B61164B186802F0D8FE8046FDF7CEFE4D
:10F8B00008B101F0C7FC3046414602F0D4FE0823EF
:10F8C0003B61304602F0CCFE78B10D4F4FF010088E
:10F8D000C7F814803046D4F8009002F0BEFE01460E
:10F8E000484602F0C0FEC7F810802B689B03D1D5B4
:10F8F000FEF779FECEE700BF50310020C82D002072
:10F90000000C01407C3100202DE9F041054608F053
:10F910006AF82C4B04469E6888B92B4803F0A8FC73
:10F920002A4B53F8241041B10123A340334202D0A3
:10F930002748F9F72FFA0134F2E7264821E0284654
:10F940002549224608F058F858B9244803F090FC9D
:10F95000234C54F8041F0029EFD01D48F9F71AFA78
:10F96000F7E72B7800262D2B03BF013504F1FF3478
:10F970004FF001084FF00008144B53F8267027B9D8
:10F980001848BDE8F04103F073BC284639462246CA
:10F9900008F032F898B90120B040B8F1000F03D058
:10F9A000F9F744FB104802E0F9F748FB0F4803F071
:10F9B0005FFC3946BDE8F0410D48F9F7EBB9013677
:10F9C000DAE700BFE81000204CBF0108ACA4010832
:10F9D00042BF010831C901082ABF010856BF01080A
:10F9E000A8A40108BABC010862BF01086BBF0108E6
:10F9F000D4C7010810B5084803F03AFC074B0024AF
:10FA00001C741C64064B1C7002F0D6FF03F0D4FD7E
:10FA1000044B1C6010BD00BF73BF0108C82D00203F
:10FA2000CE3300205031002070B5064600240B4B29
:10FA3000E518AA8816420AD0E1580948F9F7AAF948
:10FA40002846002103F0A5FB064803F011FC40F610
:10FA5000444314349C42EAD170BD00BF0CA9010894
:10FA60009FBF010831C9010808B50848F9F792F9A4
:10FA7000FEF75AFBFFF710FC18B9642002F015FDE1
:10FA8000F8E70348BDE80840F9F784B9A9BF0108C1
:10FA9000B6BF01082DE9FF410A48068885684488F9
:10FAA000B0F80480C768FEF747FACDF800800290EE
:10FAB000019731462A4623460348F9F76BF904B00B
:10FAC000BDE8F0810C000020BEBF0108F0B504784D
:10FAD0008BB005460CB1002436E04B4B19680E2361
:10FAE00003FB0411B1F91D51B1F91921B1F91B3111
:10FAF000009591F8205101F58C70019591F82151F4
:10FB000001F59071029590F90700039091F90210A8
:10FB10003E48049121460134F9F73CF9082CDCD128
:10FB200070E02D2B14D1072C1BDC284607F0B0FF0A
:10FB30000AAB661C03EB440424F8100C15F8013FD3
:10FB4000303B092BFAD934462B78002BE9D104E05D
:10FB5000A3F13002092A09D8E5E7082CBDF81820DE
:10FB600009D00BB0BDE8F040F7F72EBB202BF8D141
:10FB700001352646E7E7072AF3D840F2DC55BDF801
:10FB80001A00214BA0F2EE2189B2A9421B68E8D8E5
:10FB9000BDF81C10A1F2EE24A4B2AC42E1D8BDF82D
:10FBA0001E6004B237B2A742DBDB0DB2AF42D8DC35
:10FBB000A542D6DBBDF8247007F16404A4B2C82CBA
:10FBC000CFD8BDF826E00FFA8EF4112CC9DCBDF8B1
:10FBD0002050B42DC5D8BDF82240B42CC1D812B2E3
:10FBE0004FF00E0C0CFB0233A3F81901A3F81B1104
:10FBF000A3F81D6183F8205183F8214183F81F7118
:10FC000083F822E10BB0F0BD181000201BC00108E2
:10FC1000F0B504468FB0204607F0E5FEC5B21DBB27
:10FC2000AE4803F025FBAE4C94F8D21009B9AD48AC
:10FC300053E049B294F8D02094F8D130009194F870
:10FC4000D310A948019194F9D4100734029194F982
:10FC5000CE10039194F8CF10049129460135F9F79D
:10FC600099F8102DE0D1E2E72046A049052207F0DF
:10FC7000C3FE0546B8B929469D48702207F06FFEBD
:10FC800028469C4B19680E2303FB00130130002209
:10FC9000082883F8232183F8242183F8252183F879
:10FCA0002621F0D118E120469349042207F0A4FE52
:10FCB00005462046002D4AD1202107F086FE002867
:10FCC00000F00A81461C304607F08DFE2C460746A0
:10FCD0008A4B53F824502DB989480FB0BDE8F04045
:10FCE000F9F758B830462946FAB207F085FE0134D4
:10FCF0000028EDD17A4A164602F17001002382F8FD
:10FD0000D63082F8D23082F8D13082F8D030073243
:10FD10008A42F3D17B4901EBC40191F8A0229342BE
:10FD200010DAD1F8A472C3EBC302B0183A441768D2
:10FD300000F1D001C0F8D0709088013388809279AA
:10FD40008A71E7E729467048F9F724F895E06F498A
:10FD5000072207F051FE05462046002D49D12021FB
:10FD600007F033FE064607F03EFEC4B26CBB68489F
:10FD7000F9F710F8214667480134F9F70BF80E2C13
:10FD8000F8D15848F9F706F8002463482146F9F7F6
:10FD900001F80025574A012311680E2202FB0412C4
:10FDA000D2F82321AB4013425C4B5D495D4808BF4C
:10FDB00019460135F8F7EEFF0E2DEBD14948013415
:10FDC000F8F7E8FF082CE0D186E03046564907F006
:10FDD00063FE2C46002852D0022C55D007F058FE66
:10FDE00006AB43F824005049002007F055FE0134CB
:10FDF000F0E74D4907F050FE002460B1082C3ED0DA
:10FE000007F046FE06AB43F824004749002007F000
:10FE100043FE0134F1E7082C31D1069B0F2B2ED87D
:10FE2000DDF81CE0BEF1070F29D8089F0D2F26D85A
:10FE3000099E06F16402C82A21D80A9DFF2D1ED80A
:10FE40000B9864281BD80C99642918D8884216DAB4
:10FE50000D9C032C13D8224AC3EBC303134483F82D
:10FE6000D0E083F8D17083F8D26083F8D35083F860
:10FE7000D40083F8D51083F8D6402C4CCBE60FB0D5
:10FE8000BDE8F040F7F7A0B9069B072B20D80799EB
:10FE90000D291DD80278722A0DD06E2A18D1154A64
:10FEA0000E20126800FB032301228A40D3F823119D
:10FEB00021EA020209E00F4A0E20126800FB032328
:10FEC00001228A40D3F823110A43C3F8232101E019
:10FED000F7F77AF90D4C9EE60FB0F0BD43C001086C
:10FEE000E810002031C901086EC001088ABC010871
:10FEF000B811002018100020B5BC010844A4010866
:10FF0000BABC010864A20108C9BC01083BC00108D1
:10FF10001CBF01088AC00108BFBE01083ECC010811
:10FF200084CB01088FC0010893C0010804BA0108FE
:10FF30002DE9F743047805468CB9324D95F8AF1298
:10FF4000B5F8AC2295F8AE322F4800912146013425
:10FF5000F8F720FF102C05F10405EFD14EE007F073
:10FF600097FD0F28044636DC2846202107F02DFD9A
:10FF7000264EE4B2D6F84480451CA400002728464B
:10FF800007F086FD5FFA87F9B9F1010F83B208D057
:10FF9000B9F1020F0BD0B3F5B47F24D2726C1353B6
:10FFA0000AE0FF2B1FD8736C2344987004E0FF2BEA
:10FFB00019D8736C2344D87028462C2107F005FD0E
:10FFC000054608B1013502E0B9F1020F0BD1013746
:10FFD000032FD4D112E00E4800210F2203B0BDE858
:10FFE000F043F7F76EB808EB04000021042207F095
:10FFF000B6FC03B0BDE8F043F7F7E6B803B0BDE8E0
:020000040801F1
:10000000F08300BFE810002095C00108C82D002033
:1000100048BC01082DE9F04FAC498BB0044607F00D
:10002000A7FCAB49002820460CBF0125072507F097
:100030009FFCA8490028204608BF022507F098FC2D
:10004000002808BF0425E90740F1E780A24803F033
:100050000FF9002002F016FFA04CA14803F008F9A8
:10006000A04803F005F962799F4BA04803EB820397
:10007000D3F8DC11F8F78EFE9D48F8F78BFE264684
:100080000027D6F810800021404604F035FC20B14E
:100090009848F8F77FFE002669E039469648D6F87A
:1000A00014B0D6F818A0D6F81C90F8F773FE4046A6
:1000B000002104F02BFC10B1202003F0D1F806A998
:1000C0004046F8F7EDFC01468C48F8F763FE5846C9
:1000D000002104F01BFC10B1202003F0C1F806A998
:1000E0005846F8F7DDFC01468448F8F753FE5046C1
:1000F000002104F00BFC10B1202003F0B1F806A998
:100100005046F8F7CDFC01467C48F8F743FE4846D8
:10011000002104F0FBFB10B1202003F0A1F806A998
:100120004846F8F7BDFC013701467548F8F732FE3E
:100130000C2F06F11006A4D1AAE749B294F8D020FA
:1001400094F8D130009194F8D3106E48019194F94D
:10015000D4100734029194F9CE10039194F8CF1083
:10016000049131460136F8F715FE102E03D094F8AD
:10017000D2100029E1D1644803F07AF8574B634C60
:100180009F6854F8041F19B16148F8F703FEF8E7B7
:100190000E46604B53F826404CB10123B3403B421E
:1001A00003D05D482146F8F7F5FD0136F1E75B48DD
:1001B00003F05EF82146494B0AAA0B4493F88831B4
:1001C0001344574A8A5C0131082903F8102CF2D1F4
:1001D000002306A953488DF82030F8F7DBFD52487C
:1001E00003F046F85148F7F719FB514803F040F87F
:1001F0004E48F6F7EFFF4F4803F03AF84B48FFF749
:1002000097FE4D48F8F7C6FD4020FFF70DFC4B4820
:1002100003F02EF84548F7F7A3FBAA0739D548485D
:1002200003F026F8474803F023F8404802F06AFE3E
:10023000454803F01DF83D48F6F750FF434803F0EA
:1002400017F83A48F7F73CFA4148F8F7A3FD374862
:10025000F7F7CCF83F4803F00BF83448FFF736FCCB
:1002600000260E27774300243B4A0123926CA340CB
:100270003A44D2F80A2013421ED101340E2CF3D195
:100280000136082EEDD12C48F8F784FD8020FFF7C9
:10029000CBFB6B0716D5314802F0EAFF304802F07D
:1002A000E7FF224802F008FE2348F8F773FD4FF4F9
:1002B0008070FFF7B9FB05E0314622462948F8F780
:1002C00069FDDAE70BB0BDE8F08F00BFA9C00108F7
:1002D0001DC50108B0C00108B6C00108E810002023
:1002E000C4C00108D6C0010864A20108E2C0010828
:1002F000EDC00108FAC0010807C101081BBF0108D1
:10030000D5C701081FC101080FC10108A8A4010831
:100310003EC10108ACA401084CC1010859C1010843
:1003200052D3010865C101086EC1010804BA010871
:100330007DC1010889C1010831C9010897C10108BF
:10034000A4C10108B7C10108C5C10108CFC1010896
:10035000DEC10108ECC10108C82D0020F8C1010868
:1003600009C201081BC20108064B1B7803F00403F5
:1003700003F0FF001BB1044B1888C0F3C01000F05D
:1003800001007047C9330020A41900202DE9F04F67
:1003900089B00593B74B0026B3F90270B3F900306A
:1003A000002FB8BF7F42002BB8BF5B429F42B8BF4F
:1003B0001F4680468246B346B4463446B7F5FA7FB8
:1003C00004910292A8BF4FF4FA770196AA4D2B88A8
:1003D000990759D0A74B610033F91420A74B33F983
:1003E000143003EB4202029B5B429A4203DB029B06
:1003F0009342A8BF1346A24A31F90290059AC9EB6D
:10040000030332F9140003EB0009FFF7ADFF98B1C5
:100410009C4B48461B5D019304F086F89A4904F012
:100420008BF9019B0146184603F08EF9964904F0BA
:10043000CFF804F093FA814698F80830642203FB61
:1004400009F393FBF2F398F81C206FF0040C0CFBFB
:1004500002FC634504DB02EB820C9C45A8BF9C4672
:1004600042F21072894B53F8240048449042A8BFCE
:100470001046874A9042B8BF104643F8240098F8C7
:1004800012305843031301932D8805F00303012B09
:1004900036D0784B7F4933F914B07F4B9AF80190EE
:1004A00033F91400A60080EAE073A3EBE073B3F520
:1004B000206F51F824E016DC502303FB0BF292FB73
:1004C000F9F3042290FBF2F0181A8644BEF57A5F25
:1004D000724BA8BF4FF47A5E9E45ACBF41F824E052
:1004E00041F8243002E0002341F824308B597D2666
:1004F00093FBF6F69AF80B307343402693FBF6F61F
:10050000AA0711D507FB06F507FB0BF90198C7F5FC
:10051000FA7303FB0C9903FB00534FF4FA7199FB38
:10052000F1F293FBF1F505E0EB0759BF35465A466A
:100530006246019D63000393574B042033F814E097
:1005400057490FFA8EF393FBF0F9615C01FB09F157
:100550006FF04F0991FBF9F99144524A32F91410A6
:1005600022F814E098F850205B1A93FBF0F082B167
:10057000CDF818C0079203F0D7FF4B494B4B01EB66
:10058000C401079A1B68F8F7C5F904F0E7F9DDF82C
:1005900018C0474BDFF834E11B5D09EB05025843F7
:1005A000202390FBF3F30399D21A21F80E2041483F
:1005B0004149424A5B4241F8245040F8249042F8B5
:1005C00024300AF1010A75460CB90124FEE6294BD4
:1005D000304EB3F90440049BD6F808E09B790F3302
:1005E0005B0063432C4C5B11B4F90470002BA3EB4C
:1005F0000707B8BF5B42322B98F80D400BDC04FBB9
:1006000007E42F4BA342A8BF23462E4CA342ACBF06
:10061000B360B46001E00023B36098F8034004FBCA
:1006200007F3294C9B112478032C0CD9B8F84E40C1
:10063000B4F5FA7F07D26742BB4203DBA342A8BFEF
:10064000234600E03B46B4686FF0FF0644F34F34A6
:10065000B4F5807FA8BF4FF48074B442B8BF34466D
:1006600083601E190023AE808C60936009B0BDE8E2
:10067000F08F00BFE0100020A4190020C433002038
:10068000743100208C9E010800002041142E0020AF
:10069000F0D8FFFF541F0020FC0F002080C1FFFF97
:1006A000C41F00201C2E00206C1F0020501F0020A3
:1006B000D81F00208C1F0020981F0020A41F00209E
:1006C000FEFFFF0F020000F0F82F0020841F002023
:1006D0002DE9F04F87B00393A14B80461C8802910F
:1006E00004F00204A4B2019294B19E4BB3F902400B
:1006F000B3F90030002CB8BF6442002BB8BF5B4296
:100700009C42B8BF1C46B4F5007FA8BF4FF40074EC
:10071000C2460025934B944933F91520934B4FEA79
:10072000450B33F91530520083EAE376A6EBE37606
:10073000B6F5206F4FEA850951F8250011DC042633
:1007400093FBF6F3D31A0344B3F57A5F8848A8BF46
:100750004FF47A538342ACBF41F8253041F825006D
:1007600002E0002341F8253051F809709AF80B3067
:10077000FF119AF801605F43794B56431B88BF1104
:100780009B074FEAA61656D07A4B3BF903301A4422
:10079000019B5B429A4203DB019B9342A8BF134635
:1007A000754A3BF902209B1A039A32F915201A4424
:1007B0000492FFF7D9FD049A98B1704B10465B5D27
:1007C000049303F0B1FE6E4903F0B6FF049B0146AB
:1007D000184602F0B9FF6A4903F0FAFE04F0BEF8C9
:1007E000024642F21070674959F8013013448342BF
:1007F000A8BF034664488342B8BF034649F80130A6
:1008000098F8081098F81C004A4300EB8000D211B9
:1008100041428A4203DB8242A8BF0246114698F851
:100820001220761A53431B13FF1A6743664303EBE8
:10083000672701EB66264D494FF0040C3BF801E0B9
:10084000524A0FFA8EF393FBFCF0525D4243A6EB43
:10085000A2164F4A3BF902002BF802E098F850200C
:10086000181A90FBFCF08C467AB10591049203F0C3
:100870005BFE4849484B01EBC501049A1B68F8F739
:1008800049F804F06BF8DDF814C0444BDFF828E1B8
:100890005B5DF21958434311D21A2BF80E204048E1
:1008A0004049414A5B4249F8006049F8017049F803
:1008B00002300AF1010A76460DB901252AE7294BD3
:1008C000BCF90470B3F90440029B274D9B79D5F81D
:1008D00008E00F335B0063435B11002BA3EB0707BA
:1008E000B8BF5B42322B98F80D400BDC04FB07E4E9
:1008F0002E4BA342A8BF23462D4CA342ACBFAB60F6
:10090000AC6001E00023AB6098F8034004FB07F300
:10091000284C9B112478032C0CD9B8F84E40B4F520
:10092000FA7F07D26742BB4203DBA342A8BF23463C
:1009300000E03B46AC686FF0FF0544F34F34B4F57C
:10094000807FA8BF4FF48074AC42B8BF2C46836050
:100950001D190023B5808C60936007B0BDE8F08F4F
:10096000A4190020E0100020541F0020FC0F0020DC
:1009700080C1FFFFC4330020743100208C9E010829
:1009800000002041142E0020F0D8FFFFC41F0020DB
:10099000202E00206C1F0020501F0020D81F002098
:1009A0008C1F0020981F0020A41F0020FEFFFF0FB7
:1009B000020000F0F82F0020841F00202DE9F04FE6
:1009C00087B003939F4B0026B3F90280B3F9003040
:1009D000B8F1000FB8BFC8F10008002BB8BF5B42E8
:1009E0009845B8BF98468346B246B1463446B8F5F6
:1009F000FA7F0292A8BF4FF4FA7800900196924DC8
:100A00002B88990756D0022C54D08E4B610033F9B5
:100A100014208E4B33F9143003EB4202029B5B42ED
:100A20009A4203DB029B9342A8BF1346884A8F5E1B
:100A3000039ADB1B32F914001F18FFF795FC90B1E5
:100A4000844B384613F8049003F06EFD824903F09E
:100A500073FE0146484602F077FE7F4903F0B8FD79
:100A600003F07CFF07469BF8083064227B4393FB2E
:100A7000F2F39BF81C206FF0040909FB02F94B45C7
:100A800004DB02EB82099945A8BF994642F2107235
:100A9000724B53F8240038449042A8BF1046704A65
:100AA0009042B8BF104643F824009BF812305843D8
:100AB00003130193298801F00303012B01D1022CB8
:100AC0003DD1604B674D33F914A0009BA00093F813
:100AD00001E0654B55F8247033F9146086EAE6733B
:100AE000A3EBE673B3F5206F1CDC022C14D050236B
:100AF00003FB0AF292FBFEF3042296FBF2F69E1B26
:100B00003744B7F57A5F594BA8BF4FF47A579F42E5
:100B1000ACBF2F502B5007E08AEAEA73A3EBEA73CD
:100B2000642BE4DD00232B504E4B7D26C35893FBF2
:100B3000F6F6009BDB7A7343402693FBF6F68A07B2
:100B400013D5022C11D008FB06F508FB0AF7019813
:100B5000C8F5FA7303FB097703FB00534FF4FA72ED
:100B600097FBF2F193FBF2F508E0CB0704D5022CDA
:100B700002D0019D494601E0354651463A4B0427D3
:100B800033F914303A4A93FBF7F3A25C6FF04F0746
:100B9000534393FBF7F3022C4FEA440C01EB03079A
:100BA0000FD13846CDF810C003F0BEFC314B3249AE
:100BB0001E221B68F7F7AEFE03F0D0FE0746DDF8F5
:100BC00010C0294B2D4A3CF803103CF902000BB22F
:100BD0002CF802109BF85020181A042390FBF3F015
:100BE00082B1CDF814C0049203F09EFC2449214B3D
:100BF00001EBC401049A1B68F7F78CFE03F0AEFE0C
:100C0000DDF814C01F4B204A1B5D5843202390FB86
:100C1000F3F07B191B1A2CF802301C4B404243F8AE
:100C200024701B4B43F824501A4B43F82400009BBC
:100C300001340133032C00937FF4E1AE07B0BDE82B
:100C4000F08F00BFE0100020A4190020C433002062
:100C5000743100208C9E010800002041142E0020D9
:100C6000F0D8FFFF541F0020FC0F002080C1FFFFC1
:100C7000C41F0020501F0020481F0020242E0020E9
:100C80006C1F0020D81F0020841F00208C1F002014
:100C9000981F0020A41F00202DE9F04F89B0069373
:100CA000974B0C461B888146990703924DD540F21D
:100CB000E631129B934AD889B2F900301B1A03F22D
:100CC000F3158D4203D8002BB8BF5B4201E04FF40F
:100CD000FA73B2F90220101A40F2E63200F2F31170
:100CE000914203D80028B8BF404201E04FF4FA70A7
:100CF00099F84C503DB39842B8BF1846C0F5FA7009
:100D000003F012FC804903F017FD4FF07E5103F011
:100D100055FB0646642090FBF5F003F005FC014608
:100D2000304603F055FC4FF07E5103F049FB0021A3
:100D3000074603F0EBFD30B938464FF07E5103F023
:100D400003FE20B101E0002701E04FF07E57C846C6
:100D5000E31C04930024049B022C1A4612F8013F62
:100D60006A4E019304920AD1019DB6F904000A3536
:100D7000684303F0D9FB664903F0DEFC74E036F902
:100D8000140003F0D1FB8246039803F0C9FB5E49CF
:100D900003F0D2FC0146504603F01AFC5D4B82463C
:100DA00033F9140003F0C0FB0146504603F008FB82
:100DB000039B8246584203F0B7FB0546504629463E
:100DC0004FEA440B03F0A2FD48B9039803F0ACFBD3
:100DD00005465046294603F0B7FD00B955464E4A30
:100DE00032F90B0003F0A0FB0146284603F0E6FAB7
:100DF000069B824633F9140003F096FB01465046E9
:100E000003F0DEFA454903F097FC8246FFF7ACFA9F
:100E100028B1434B5146185D02F096FC8246384B90
:100E20001B88DA0705D55046D9F8441003F0D0FBEB
:100E30001AE0019D36F90B0014356843029303F064
:100E400073FB334903F078FC029B05469B070CD5E6
:100E5000D9F84810504603F0BBFB394603F0B8FB05
:100E60000146284603F0ACFA0546630005932D4B76
:100E70002D4E33F9140003F057FB2C4B196903F086
:100E8000A7FB0146284603F099FAD8F820108246BD
:100E900003F09EFB264B0546185D03F045FB01461B
:100EA000284603F095FB234903F046FC022C0190F1
:100EB00005D121491E223368F7F72CFD01903368D4
:100EC000504619460293DFF87CB003F081FBD8F856
:100ED0002C1003F07DFB114903F07AFB5BF8241022
:100EE00003F06EFA1549A500064603F00FFD58BB46
:100EF0003046134903F028FD38B3114E25E000BFFA
:100F0000A4190020B83100200000FA43E0100020AE
:100F100000004842C433002074310020000020410A
:100F20008C9E0108FC0F0020501F0020582100203B
:100F3000441F00200000C842481F002000007AC360
:100F400000007A43B81F0020374E4BF80560DFF8E9
:100F500004B1504655F80B1003F030FA029907908F
:100F600045F80BA04FF07E5003F0E6FB079B0146CF
:100F7000184603F02DFB99F85020034632B12B4957
:100F8000029B01EBC401F7F7C5FC0346D8F8381003
:100F9000184603F01DFB264B8246185D03F0C4FA89
:100FA0000146504603F014FB224903F0C5FB2249D9
:100FB000824603F0ABFC38B95046204903F0C4FC2C
:100FC00020B1DFF878A001E0DFF86CA0019831468D
:100FD00003F0F6F9514603F0F3F906F0CDFE184B95
:100FE000B0F57A7FA8BF4FF47A709842B8BF184620
:100FF000059A144B0134D052019803F0AFFC124B08
:1010000008F104085851304603F0A8FC0F4B585122
:10101000504603F0A3FC0E4B032C58517FF49BAEBB
:1010200009B0BDE8F08F00BF00007AC36C1F00203C
:10103000441F00200000C842000096C300009643F1
:1010400018FCFFFF841F00208C1F0020981F002029
:10105000A41F00202C2E0020044B00221A605A608E
:10106000034B00221A605A60704700BF142E002004
:10107000B01F002010B50B4C0123E3704FF48060CB
:10108000022384F82030F7F7C1FF074A074B526A62
:101090001B685278642101FB0233636123880133AA
:1010A000238010BDD4240020142E0020A031002065
:1010B00010B54B88DC0641BF2F4B14791B6853F8E1
:1010C000244044BF2D4B43F820404B889B0641BF32
:1010D000294B54791B6853F8244044BF274B43F8ED
:1010E00020404B881C070ED5254B0C781B78B3EBA2
:1010F000141FA1BF204BD4781B6853F82440A4BF11
:101100001E4B43F820404B889B070ED51D4B0C7897
:101110001B78B3EB141FDFBF174B54781B6853F8D1
:101120002440DCBF154B43F820404B88DC070FD52B
:10113000154C0B78247803F00F03A342DFBF0E4B4E
:1011400014781B6853F82440DCBF0C4B43F8204054
:101150004B885B070FD50B780C4903F00F03097818
:101160008B42A1BF044B92781B6853F82220A4BF86
:10117000024B43F8202010BD0C2E0020820D0020D1
:10118000A7200020A5200020A4200020A6200020C9
:10119000254A0023F0B515681C461A462348244901
:1011A00003700B702E1976884EB92F5D3FB903700E
:1011B00000230A704B7007781C461A460CE036056F
:1011C00048BF013204F1040403F1010348BFD2B265
:1011D000802CDBB2E6D1EAE7E0B2B8420CD215F8D7
:1011E0002400013406099E4200F00F00A8BF731CC2
:1011F0009042A8BF421CEFE78A704B70C2F34701D0
:1012000002F001020A444C1E0A490B480A70C3F35B
:10121000470203F00103134404700849501E084AB2
:1012200008701370F0BD00BFA81900209C2000209A
:101230003C2E0020A6200020A4200020A720002073
:10124000A5200020924B2DE9F04FDA68914D1A61EC
:101250002A6891B0DA60904A0295136843F020033F
:1012600013608E4B1A78012A0CBF002201221A70DB
:101270008B4B1A78910740F14D838A4909780429EC
:1012800040F248838849097801F0040101F0FF0029
:1012900011B922F001021A701B78DB0702D408B1E1
:1012A000FCF7A2FD8149CA78531C052293FBF2F298
:1012B00002EB82029A1A7E4BCA701F7892000023BA
:1012C000DFF81082DFF8109258F82310794C91FB68
:1012D000F9FE04F1080040F823E0774844F82310B1
:1012E00000FB0E1142F2107091FBF0F004F11006B9
:1012F00080B226F813004FF0140C04F114060CFB16
:10130000036C04F13C0A5AF823605CF802504CF874
:101310000210761B314405264AF8231091FBF6F1A2
:1013200009FB0E114434012F44F823104FEA830BBC
:10133000444605D10238B0F5797F98BF4BF80810C4
:101340000BB90123BCE7594E029BB2461868336DB6
:10135000C01A03F0E5F8594903F0EEF9029B4FF08B
:101360007E511B680746336503F0D0FA08B94FF089
:101370007E574B4BCAF854701B78514E13F0010343
:10138000504D12D00DAA00924F4B0EAA01920CCBD9
:1013900094E80300FCF73EFC0D9A6421B2FBF1F2E5
:1013A0000E9B328093FBF1F300E033802B809AF8A0
:1013B00058303E4D002B35D0696D4FF07E5003F014
:1013C000BBF90746EB6D2068C01A03F0ADF839464B
:1013D00003F0FEF803F0C2FA2B6E86B2606836B2F4
:1013E000C01A03F0A1F8394B196803F0F1F8394637
:1013F00003F0EEF803F0B2FAB5F9662000B28118F6
:10140000B5F964200220B31891FBF0F193FBF0F3DF
:1014100089B29BB2A5F86A10A5F86830A5F86610E5
:10142000A5F8643001238AF85830294B61681B887D
:10143000206803F030031D4E264DCAF86010CAF82C
:101440005C00002B00F0668206F17403009306F145
:1014500078030193F26E336FFCF7DCFB6B68306F3F
:10146000C01A03F061F8194B196803F0B1F803F0E2
:1014700075FAF36E2A68C6F880009B1AF3670C4B66
:101480001B78012B2AD0022B00F0E68042E200BF3D
:101490001C070020A0310020DC180020461000208E
:1014A000E0180020E6180020C93300203C2E002060
:1014B0000C0F0020402E0020806967FF00007A4456
:1014C0005A1900205C19002048100020400000201C
:1014D000A4190020E818002080969800D6F88430DF
:1014E000D6F8A0400293D6F8943004F1004003935C
:1014F000D6F89830776D059303F030FA8146204690
:1015000003F02CFAD6F89C30BB4C0493BB4B0690EE
:101510001B684FF0000B0793B94E4FEA4B0356F888
:101520002B80A6F11402404632F81B50089302F0BB
:10153000FBFF029903F04CF803F010FA401B1FFA6E
:1015400080FA283626F81BA00FFA8AFA504602F0D5
:10155000EBFF039903F03CF803F000FA86B20AEBC4
:10156000080002F0E1FF059903F032F8394603F074
:101570002FF8216802F024FF03F0F0F9484504DB5E
:10158000069B9842A8BF184600E0484602F0CCFFF0
:10159000206003F0E3F9079B304486B2987802F0AC
:1015A000BFFF984903F014F801464FF07E5003F056
:1015B000C3F8394602F004FF0146384603F0BCF890
:1015C00009906068D4F808A0C0EB080002F0ACFFF6
:1015D000394603F0B1F8514602F0F0FE099A01468F
:1015E000104602F0F5FF0146504602F0E9FE3135A3
:1015F000ADB2622D01462061C4F80480A0600ED90E
:10160000049802F0E5FF03F0A9F97F4AB0F5FA6FFC
:10161000A8BF4FF4FA609042B8BF104600E0002027
:1016200040F6B832064436B29642A8BF1646774A0C
:10163000089B9642B8BF1646754A54F8140B9E5242
:10164000142202FB0BF273495050BBF1000F40F023
:1016500061814FF0010B5FE7684BB6F8A8401F6847
:10166000736F3D8902935B089D4228BF1D4623B2DC
:101670009D4202DC1FFA85F90AE06749706D02F0AD
:10168000A7FF03F06BF920441FFA80F9A6F8A89091
:10169000DAF87860DAF8AC40341B2046FCF7FCFA44
:1016A00041F293130028D8BF40429842CCBF00209B
:1016B000012078B3204602F037FF584902F088FF36
:1016C000F7F718FC0446029802F02AFF014620466C
:1016D00002F07EFF03F042F940F6B83380B2AAF878
:1016E000B00000B29842A8BF1846484B9842ACBF21
:1016F0003018F01848F6A043984203DDA0F50C40DE
:10170000A03804E00028BCBF00F50C40A030CAF8A7
:10171000B40001E0CAF8B460DAF8B4300026C3F5CA
:101720000C502830039302F0FFFE3C4902F050FFBA
:101730000446F7F751FC0F902046F7F7DBFBDAF889
:10174000B830DAF8C4400593DAF8BC300E9004F1F2
:101750000040089303F002F90490204603F0FEF8DD
:10176000DAF8C030DAF854802A4C099007937300F5
:1017700048460A9302F0D8FE0EAB53F8261002F04A
:1017800027FFDFF8A0A005463AF9160002F0CCFECC
:101790000146284602F012FE03F0E0F805B2204BA5
:1017A000B5F57A7FA8BF4FF47A759D42B8BF1D4644
:1017B0000AF13C0AA8B22AF8160000B202F0B4FE00
:1017C0000599824602F004FF03F0C8F8089983B235
:1017D0005046069302F0FCFE414602F0F9FE2168F5
:1017E00002F0EEFD03F0BAF8049B98421CDB099B63
:1017F0009842A8BF184618E0480F0020100F00209C
:10180000B82E0020DB0FC94030F8FFFF48F4FFFF7F
:101810001A0F0020700F00200000C842D302373991
:1018200018FCFFFFA42E0020049802F07DFE20602B
:101830008346B87802F074FE384902F0C9FE0146CA
:101840004FF07E5002F078FF414602F0B9FD0146AC
:10185000404602F071FF0B906068D4F808A0281A87
:1018600002F062FE414602F067FF514602F0A6FD1B
:10187000DDF82CC00146604602F0AAFE0146504643
:1018800002F09EFD656001462061A060079802F0AD
:101890009FFE03F063F8069B1434034458469A46AF
:1018A00003F05CF840F6B832504400B29042A8BF52
:1018B00010461B4A0A9B9042B8BF1046194A1A4963
:1018C00098521422724342F801B00EB901264EE735
:1018D0003B792BB1039A642392FBF3F3134A1380F1
:1018E0003B88029A124C9A420DD9D4F8AC30A06FC2
:1018F000C01AFCF7D1F942F2107380EAE072A2EB51
:10190000E0729A4206DD0B4B01221A70B4F8C8202F
:10191000064B1A8011B0BDE8F08F00BFDB0FC94045
:1019200048F4FFFF1A0F0020480F0020080F002086
:101930003C2E00200C0F00200846F6F79FBA0E4BF5
:101940001A786C2A15D15A88B2F5FC6F11D11A7920
:10195000BE2A0ED193F8DD270020EF2A0BD113F811
:10196000012B5040054A9342F9D1B0FA80F040096A
:10197000704700207047704700F80108E0FF010839
:101980002DE9F04FD84C85B000214FF4FC62204681
:1019900005F0E5FFD54B04F53B721A60D44B0025EA
:1019A0001D70D44B04F2B6721A606C2323704FF48E
:1019B000807003236371F7F741FB202284F86821CC
:1019C0006E2284F87A210A224FF4167384F87B2160
:1019D0002B22A4F8643184F87D21FA232122A4F873
:1019E000663184F87E214FF4FA732322A4F86C3117
:1019F00084F87F2101234FF4C87284F85E3184F8A3
:101A0000693184F86A3184F87C31A4F8802184F843
:101A100084310022052384F8B457A4F87051A4F847
:101A20006E51A4F8725184F8545184F8555184F8D9
:101A30005651A4F85851A4F85A51A4F85C5184F8AE
:101A40005F51A4F88251A4F8865184F81D5284F89D
:101A50001C52C4F82022C4F8242284F8285284F8A6
:101A6000295284F82B3240F2DC53A4F8963140F22C
:101A70004C43A4F8983140F26C73A4F89A3140F2C8
:101A80007533A4F89C3140F64303A4F89E312346F5
:101A900084F82A5284F8905184F891510192032DD0
:101AA000CCBF0122002205F1010583F8A02114BF5B
:101AB0001E227522122D83F8A12103F10203EED11B
:101AC00040F27E4240F27E50A4F84021A4F8480142
:101AD00040F23A7240F2EA50A4F84221A4F84A01D6
:101AE00040F2DC5240F2B4504FF4FA63A4F8C6312D
:101AF000A4F8CA31A4F8CE31A4F8D231052384F871
:101B0000E031DFF8E881C823002501264FF47A7917
:101B10001E214FF0320A4FF0190BA4F8E4314FF4B4
:101B2000C87384F893110391A4F8E831A4F846210E
:101B30000292A4F84C0184F8E1B184F8925184F83F
:101B40009451A4F8C491A4F8C891A4F8CC91A4F835
:101B5000D09184F8D45184F8DE5184F8DF6184F8A0
:101B6000E26184F8E36184F8E66184F8EA5184F87C
:101B7000EC61A4F84491A4F84EA1A4F85031A4F863
:101B800052A184F8ED5184F8EE5184F8EF6184F8A5
:101B9000F051F9F741FED8F800300F202573587145
:101BA000222098710E2018743520039998762120F0
:101BB00058745320D9721973D87655215A20D97088
:101BC00018722D2178205973987219754A484FF46C
:101BD000FA71282783F807B0A3F84E104FF0640B72
:101BE00014210A229A741D705F705F759F709F7533
:101BF000DD7583F804A09D731D76DD735D7683F833
